Archive member included to satisfy reference by file (symbol)

libLoRa_pico_lib.a(LoRa-RP2040.cpp.obj)
                              CMakeFiles/main.dir/main.cpp.obj (LoRaClass::write(unsigned char))
libKISS.a(kiss.cpp.obj)       CMakeFiles/main.dir/main.cpp.obj (KissClass::EncodeFrame(aprs_frame*, ax25_frame*))
libi2c_sensor.a(i2c_sensor.cpp.obj)
                              CMakeFiles/main.dir/main.cpp.obj (initAM2315())
/usr/lib/gcc/arm-none-eabi/7.3.1/thumb/v6-m/libgcc.a(_dvmd_tls.o)
                              CMakeFiles/main.dir/__/pico-sdk/src/rp2_common/pico_divider/divider.S.obj (__aeabi_idiv0)
/usr/lib/gcc/arm-none-eabi/7.3.1/thumb/v6-m/libgcc.a(unwind-arm.o)
                              CMakeFiles/main.dir/main.cpp.obj (__aeabi_unwind_cpp_pr0)
/usr/lib/gcc/arm-none-eabi/7.3.1/thumb/v6-m/libgcc.a(libunwind.o)
                              /usr/lib/gcc/arm-none-eabi/7.3.1/thumb/v6-m/libgcc.a(unwind-arm.o) (restore_core_regs)
/usr/lib/gcc/arm-none-eabi/7.3.1/thumb/v6-m/libgcc.a(pr-support.o)
                              /usr/lib/gcc/arm-none-eabi/7.3.1/thumb/v6-m/libgcc.a(unwind-arm.o) (__gnu_unwind_execute)
/usr/lib/gcc/arm-none-eabi/7.3.1/../../../arm-none-eabi/lib/thumb/v6-m/libc.a(lib_a-abort.o)
                              /usr/lib/gcc/arm-none-eabi/7.3.1/thumb/v6-m/libgcc.a(unwind-arm.o) (abort)
/usr/lib/gcc/arm-none-eabi/7.3.1/../../../arm-none-eabi/lib/thumb/v6-m/libc.a(lib_a-atexit.o)
                              /usr/lib/gcc/arm-none-eabi/7.3.1/../../../arm-none-eabi/lib/thumb/v6-m/crt0.o (atexit)
/usr/lib/gcc/arm-none-eabi/7.3.1/../../../arm-none-eabi/lib/thumb/v6-m/libc.a(lib_a-calloc.o)
                              CMakeFiles/main.dir/__/pico-sdk/src/rp2_common/pico_malloc/pico_malloc.c.obj (calloc)
/usr/lib/gcc/arm-none-eabi/7.3.1/../../../arm-none-eabi/lib/thumb/v6-m/libc.a(lib_a-callocr.o)
                              /usr/lib/gcc/arm-none-eabi/7.3.1/../../../arm-none-eabi/lib/thumb/v6-m/libc.a(lib_a-calloc.o) (_calloc_r)
/usr/lib/gcc/arm-none-eabi/7.3.1/../../../arm-none-eabi/lib/thumb/v6-m/libc.a(lib_a-fini.o)
                              /usr/lib/gcc/arm-none-eabi/7.3.1/../../../arm-none-eabi/lib/thumb/v6-m/crt0.o (__libc_fini_array)
/usr/lib/gcc/arm-none-eabi/7.3.1/../../../arm-none-eabi/lib/thumb/v6-m/libc.a(lib_a-impure.o)
                              /usr/lib/gcc/arm-none-eabi/7.3.1/../../../arm-none-eabi/lib/thumb/v6-m/libc.a(lib_a-calloc.o) (_impure_ptr)
/usr/lib/gcc/arm-none-eabi/7.3.1/../../../arm-none-eabi/lib/thumb/v6-m/libc.a(lib_a-init.o)
                              /usr/lib/gcc/arm-none-eabi/7.3.1/../../../arm-none-eabi/lib/thumb/v6-m/crt0.o (__libc_init_array)
/usr/lib/gcc/arm-none-eabi/7.3.1/../../../arm-none-eabi/lib/thumb/v6-m/libc.a(lib_a-malloc.o)
                              CMakeFiles/main.dir/__/pico-sdk/src/rp2_common/pico_malloc/pico_malloc.c.obj (malloc)
/usr/lib/gcc/arm-none-eabi/7.3.1/../../../arm-none-eabi/lib/thumb/v6-m/libc.a(lib_a-mallocr.o)
                              /usr/lib/gcc/arm-none-eabi/7.3.1/../../../arm-none-eabi/lib/thumb/v6-m/libc.a(lib_a-callocr.o) (_malloc_r)
/usr/lib/gcc/arm-none-eabi/7.3.1/../../../arm-none-eabi/lib/thumb/v6-m/libc.a(lib_a-memmove.o)
                              CMakeFiles/main.dir/main.cpp.obj (memmove)
/usr/lib/gcc/arm-none-eabi/7.3.1/../../../arm-none-eabi/lib/thumb/v6-m/libc.a(lib_a-mlock.o)
                              /usr/lib/gcc/arm-none-eabi/7.3.1/../../../arm-none-eabi/lib/thumb/v6-m/libc.a(lib_a-mallocr.o) (__malloc_lock)
/usr/lib/gcc/arm-none-eabi/7.3.1/../../../arm-none-eabi/lib/thumb/v6-m/libc.a(lib_a-sbrkr.o)
                              /usr/lib/gcc/arm-none-eabi/7.3.1/../../../arm-none-eabi/lib/thumb/v6-m/libc.a(lib_a-mallocr.o) (_sbrk_r)
/usr/lib/gcc/arm-none-eabi/7.3.1/../../../arm-none-eabi/lib/thumb/v6-m/libc.a(lib_a-signal.o)
                              /usr/lib/gcc/arm-none-eabi/7.3.1/../../../arm-none-eabi/lib/thumb/v6-m/libc.a(lib_a-abort.o) (raise)
/usr/lib/gcc/arm-none-eabi/7.3.1/../../../arm-none-eabi/lib/thumb/v6-m/libc.a(lib_a-signalr.o)
                              /usr/lib/gcc/arm-none-eabi/7.3.1/../../../arm-none-eabi/lib/thumb/v6-m/libc.a(lib_a-signal.o) (_kill_r)
/usr/lib/gcc/arm-none-eabi/7.3.1/../../../arm-none-eabi/lib/thumb/v6-m/libc.a(lib_a-strcmp.o)
                              CMakeFiles/main.dir/main.cpp.obj (strcmp)
/usr/lib/gcc/arm-none-eabi/7.3.1/../../../arm-none-eabi/lib/thumb/v6-m/libc.a(lib_a-strlen-stub.o)
                              CMakeFiles/main.dir/main.cpp.obj (strlen)
/usr/lib/gcc/arm-none-eabi/7.3.1/../../../arm-none-eabi/lib/thumb/v6-m/libc.a(lib_a-__atexit.o)
                              /usr/lib/gcc/arm-none-eabi/7.3.1/../../../arm-none-eabi/lib/thumb/v6-m/libc.a(lib_a-atexit.o) (__register_exitproc)
/usr/lib/gcc/arm-none-eabi/7.3.1/../../../arm-none-eabi/lib/thumb/v6-m/libc.a(lib_a-freer.o)
                              /usr/lib/gcc/arm-none-eabi/7.3.1/../../../arm-none-eabi/lib/thumb/v6-m/libc.a(lib_a-malloc.o) (_free_r)
/usr/lib/gcc/arm-none-eabi/7.3.1/../../../arm-none-eabi/lib/thumb/v6-m/libc.a(lib_a-reent.o)
                              /usr/lib/gcc/arm-none-eabi/7.3.1/../../../arm-none-eabi/lib/thumb/v6-m/libc.a(lib_a-sbrkr.o) (errno)
/usr/lib/gcc/arm-none-eabi/7.3.1/../../../arm-none-eabi/lib/thumb/v6-m/libnosys.a(getpid.o)
                              /usr/lib/gcc/arm-none-eabi/7.3.1/../../../arm-none-eabi/lib/thumb/v6-m/libc.a(lib_a-signalr.o) (_getpid)
/usr/lib/gcc/arm-none-eabi/7.3.1/../../../arm-none-eabi/lib/thumb/v6-m/libnosys.a(kill.o)
                              /usr/lib/gcc/arm-none-eabi/7.3.1/../../../arm-none-eabi/lib/thumb/v6-m/libc.a(lib_a-signalr.o) (_kill)

Allocating common symbols
Common symbol       size              file

sf_table            0x100             CMakeFiles/main.dir/__/pico-sdk/src/rp2_common/pico_float/float_init_rom.c.obj
errno               0x4               /usr/lib/gcc/arm-none-eabi/7.3.1/../../../arm-none-eabi/lib/thumb/v6-m/libc.a(lib_a-reent.o)
_usbd_qdef_buf      0xc0              CMakeFiles/main.dir/__/pico-sdk/lib/tinyusb/src/device/usbd.c.obj
sd_table            0x100             CMakeFiles/main.dir/__/pico-sdk/src/rp2_common/pico_double/double_init_rom.c.obj
uart_char_to_line_feed
                    0x4               CMakeFiles/main.dir/__/pico-sdk/src/rp2_common/hardware_uart/uart.c.obj

Discarded input sections

 .text          0x00000000        0x0 /usr/lib/gcc/arm-none-eabi/7.3.1/thumb/v6-m/crti.o
 .data          0x00000000        0x0 /usr/lib/gcc/arm-none-eabi/7.3.1/thumb/v6-m/crti.o
 .bss           0x00000000        0x0 /usr/lib/gcc/arm-none-eabi/7.3.1/thumb/v6-m/crti.o
 .data          0x00000000        0x4 /usr/lib/gcc/arm-none-eabi/7.3.1/thumb/v6-m/crtbegin.o
 .fini_array    0x00000000        0x4 /usr/lib/gcc/arm-none-eabi/7.3.1/thumb/v6-m/crtbegin.o
 .text          0x00000000       0x6c /usr/lib/gcc/arm-none-eabi/7.3.1/../../../arm-none-eabi/lib/thumb/v6-m/crt0.o
 .data          0x00000000        0x0 /usr/lib/gcc/arm-none-eabi/7.3.1/../../../arm-none-eabi/lib/thumb/v6-m/crt0.o
 .bss           0x00000000        0x0 /usr/lib/gcc/arm-none-eabi/7.3.1/../../../arm-none-eabi/lib/thumb/v6-m/crt0.o
 .ARM.extab     0x00000000        0x0 /usr/lib/gcc/arm-none-eabi/7.3.1/../../../arm-none-eabi/lib/thumb/v6-m/crt0.o
 .ARM.exidx     0x00000000        0x8 /usr/lib/gcc/arm-none-eabi/7.3.1/../../../arm-none-eabi/lib/thumb/v6-m/crt0.o
 .debug_line    0x00000000       0x86 /usr/lib/gcc/arm-none-eabi/7.3.1/../../../arm-none-eabi/lib/thumb/v6-m/crt0.o
 .debug_info    0x00000000       0x26 /usr/lib/gcc/arm-none-eabi/7.3.1/../../../arm-none-eabi/lib/thumb/v6-m/crt0.o
 .debug_abbrev  0x00000000       0x14 /usr/lib/gcc/arm-none-eabi/7.3.1/../../../arm-none-eabi/lib/thumb/v6-m/crt0.o
 .debug_aranges
                0x00000000       0x20 /usr/lib/gcc/arm-none-eabi/7.3.1/../../../arm-none-eabi/lib/thumb/v6-m/crt0.o
 .debug_str     0x00000000       0x82 /usr/lib/gcc/arm-none-eabi/7.3.1/../../../arm-none-eabi/lib/thumb/v6-m/crt0.o
 .ARM.attributes
                0x00000000       0x1b /usr/lib/gcc/arm-none-eabi/7.3.1/../../../arm-none-eabi/lib/thumb/v6-m/crt0.o
 .group         0x00000000       0x18 CMakeFiles/main.dir/main.cpp.obj
 .group         0x00000000       0x18 CMakeFiles/main.dir/main.cpp.obj
 .text          0x00000000        0x0 CMakeFiles/main.dir/main.cpp.obj
 .data          0x00000000        0x0 CMakeFiles/main.dir/main.cpp.obj
 .bss           0x00000000        0x0 CMakeFiles/main.dir/main.cpp.obj
 .text._Z19SaveSettingsToFlashv
                0x00000000       0x54 CMakeFiles/main.dir/main.cpp.obj
 .ARM.extab.text._Z19SaveSettingsToFlashv
                0x00000000        0x0 CMakeFiles/main.dir/main.cpp.obj
 .ARM.exidx.text._Z19SaveSettingsToFlashv
                0x00000000        0x8 CMakeFiles/main.dir/main.cpp.obj
 .ARM.extab.text._Z12ShowSettingsv
                0x00000000        0x0 CMakeFiles/main.dir/main.cpp.obj
 .text._Z21ReadSettingsFromFlashv
                0x00000000       0x98 CMakeFiles/main.dir/main.cpp.obj
 .ARM.extab.text._Z21ReadSettingsFromFlashv
                0x00000000        0x0 CMakeFiles/main.dir/main.cpp.obj
 .ARM.exidx.text._Z21ReadSettingsFromFlashv
                0x00000000        0x8 CMakeFiles/main.dir/main.cpp.obj
 .ARM.extab.text._Z5setupv
                0x00000000        0x0 CMakeFiles/main.dir/main.cpp.obj
 .ARM.extab.text._Z10print_helpv
                0x00000000        0x0 CMakeFiles/main.dir/main.cpp.obj
 .text._Z20ConvertStringToValuePc
                0x00000000       0x44 CMakeFiles/main.dir/main.cpp.obj
 .ARM.extab.text._Z20ConvertStringToValuePc
                0x00000000        0x0 CMakeFiles/main.dir/main.cpp.obj
 .ARM.exidx.text._Z20ConvertStringToValuePc
                0x00000000        0x8 CMakeFiles/main.dir/main.cpp.obj
 .ARM.extab.text._Z10startRadiov
                0x00000000        0x0 CMakeFiles/main.dir/main.cpp.obj
 .ARM.extab.text._Z18ProcessSerialInputPc.part.0
                0x00000000        0x0 CMakeFiles/main.dir/main.cpp.obj
 .text._Z18ProcessSerialInputPc
                0x00000000       0x98 CMakeFiles/main.dir/main.cpp.obj
 .ARM.extab.text._Z18ProcessSerialInputPc
                0x00000000        0x0 CMakeFiles/main.dir/main.cpp.obj
 .ARM.exidx.text._Z18ProcessSerialInputPc
                0x00000000        0x8 CMakeFiles/main.dir/main.cpp.obj
 .text._Z17is_message_for_mePhS_
                0x00000000       0x90 CMakeFiles/main.dir/main.cpp.obj
 .ARM.extab.text._Z17is_message_for_mePhS_
                0x00000000        0x0 CMakeFiles/main.dir/main.cpp.obj
 .ARM.exidx.text._Z17is_message_for_mePhS_
                0x00000000        0x8 CMakeFiles/main.dir/main.cpp.obj
 .text._Z15compare_stringsPhS_
                0x00000000       0x3c CMakeFiles/main.dir/main.cpp.obj
 .ARM.extab.text._Z15compare_stringsPhS_
                0x00000000        0x0 CMakeFiles/main.dir/main.cpp.obj
 .ARM.exidx.text._Z15compare_stringsPhS_
                0x00000000        0x8 CMakeFiles/main.dir/main.cpp.obj
 .ARM.extab.text._Z16ComposeAprsFramePh
                0x00000000        0x0 CMakeFiles/main.dir/main.cpp.obj
 .ARM.extab.text._Z13ReadUSBSerialv
                0x00000000        0x0 CMakeFiles/main.dir/main.cpp.obj
 .ARM.extab.text.startup._GLOBAL__sub_I_lastRssi
                0x00000000        0x0 CMakeFiles/main.dir/main.cpp.obj
 .text._Z13getPacketDatai
                0x00000000       0x30 CMakeFiles/main.dir/main.cpp.obj
 .ARM.extab.text._Z13getPacketDatai
                0x00000000        0x0 CMakeFiles/main.dir/main.cpp.obj
 .ARM.exidx.text._Z13getPacketDatai
                0x00000000        0x8 CMakeFiles/main.dir/main.cpp.obj
 .text._Z8transmitv
                0x00000000       0x40 CMakeFiles/main.dir/main.cpp.obj
 .ARM.extab.text._Z8transmitv
                0x00000000        0x0 CMakeFiles/main.dir/main.cpp.obj
 .ARM.exidx.text._Z8transmitv
                0x00000000        0x8 CMakeFiles/main.dir/main.cpp.obj
 .bss.dcd       0x00000000        0x1 CMakeFiles/main.dir/main.cpp.obj
 .bss.dcdCount  0x00000000        0x2 CMakeFiles/main.dir/main.cpp.obj
 .bss.dcdLed    0x00000000        0x1 CMakeFiles/main.dir/main.cpp.obj
 .bss.dcdWaiting
                0x00000000        0x1 CMakeFiles/main.dir/main.cpp.obj
 .bss.lastRssiRaw
                0x00000000        0x1 CMakeFiles/main.dir/main.cpp.obj
 .bss.lastStatusUpdate
                0x00000000        0x4 CMakeFiles/main.dir/main.cpp.obj
 .bss.outboundReady
                0x00000000        0x1 CMakeFiles/main.dir/main.cpp.obj
 .bss.readLength
                0x00000000        0x4 CMakeFiles/main.dir/main.cpp.obj
 .bss.statRx    0x00000000        0x4 CMakeFiles/main.dir/main.cpp.obj
 .bss.statRxOngoing
                0x00000000        0x1 CMakeFiles/main.dir/main.cpp.obj
 .bss.statSignalDetected
                0x00000000        0x1 CMakeFiles/main.dir/main.cpp.obj
 .bss.statSignalSynced
                0x00000000        0x1 CMakeFiles/main.dir/main.cpp.obj
 .bss.statTx    0x00000000        0x4 CMakeFiles/main.dir/main.cpp.obj
 .data.dcdThreshold
                0x00000000        0x2 CMakeFiles/main.dir/main.cpp.obj
 .data.lastRssi
                0x00000000        0x4 CMakeFiles/main.dir/main.cpp.obj
 .data.statusIntervalms
                0x00000000        0x4 CMakeFiles/main.dir/main.cpp.obj
 .text          0x00000000        0x0 CMakeFiles/main.dir/__/pico-sdk/src/rp2_common/pico_stdlib/stdlib.c.obj
 .data          0x00000000        0x0 CMakeFiles/main.dir/__/pico-sdk/src/rp2_common/pico_stdlib/stdlib.c.obj
 .bss           0x00000000        0x0 CMakeFiles/main.dir/__/pico-sdk/src/rp2_common/pico_stdlib/stdlib.c.obj
 .text.set_sys_clock_48mhz
                0x00000000       0x3c CMakeFiles/main.dir/__/pico-sdk/src/rp2_common/pico_stdlib/stdlib.c.obj
 .text.set_sys_clock_pll
                0x00000000       0x78 CMakeFiles/main.dir/__/pico-sdk/src/rp2_common/pico_stdlib/stdlib.c.obj
 .text.check_sys_clock_khz
                0x00000000      0x170 CMakeFiles/main.dir/__/pico-sdk/src/rp2_common/pico_stdlib/stdlib.c.obj
 .text.setup_default_uart
                0x00000000       0x2c CMakeFiles/main.dir/__/pico-sdk/src/rp2_common/pico_stdlib/stdlib.c.obj
 .binary_info.__bi_ptr102
                0x00000000        0x4 CMakeFiles/main.dir/__/pico-sdk/src/rp2_common/pico_stdlib/stdlib.c.obj
 .rodata.__bi_102.5032
                0x00000000        0x8 CMakeFiles/main.dir/__/pico-sdk/src/rp2_common/pico_stdlib/stdlib.c.obj
 .comment       0x00000000       0x58 CMakeFiles/main.dir/__/pico-sdk/src/rp2_common/pico_stdlib/stdlib.c.obj
 .ARM.attributes
                0x00000000       0x32 CMakeFiles/main.dir/__/pico-sdk/src/rp2_common/pico_stdlib/stdlib.c.obj
 .text          0x00000000        0x0 CMakeFiles/main.dir/__/pico-sdk/src/rp2_common/hardware_gpio/gpio.c.obj
 .data          0x00000000        0x0 CMakeFiles/main.dir/__/pico-sdk/src/rp2_common/hardware_gpio/gpio.c.obj
 .bss           0x00000000        0x0 CMakeFiles/main.dir/__/pico-sdk/src/rp2_common/hardware_gpio/gpio.c.obj
 .text.gpio_irq_handler
                0x00000000       0x74 CMakeFiles/main.dir/__/pico-sdk/src/rp2_common/hardware_gpio/gpio.c.obj
 .text.gpio_get_pad
                0x00000000       0x28 CMakeFiles/main.dir/__/pico-sdk/src/rp2_common/hardware_gpio/gpio.c.obj
 .text.gpio_get_function
                0x00000000       0x14 CMakeFiles/main.dir/__/pico-sdk/src/rp2_common/hardware_gpio/gpio.c.obj
 .text.gpio_set_irqover
                0x00000000       0x24 CMakeFiles/main.dir/__/pico-sdk/src/rp2_common/hardware_gpio/gpio.c.obj
 .text.gpio_set_inover
                0x00000000       0x24 CMakeFiles/main.dir/__/pico-sdk/src/rp2_common/hardware_gpio/gpio.c.obj
 .text.gpio_set_outover
                0x00000000       0x24 CMakeFiles/main.dir/__/pico-sdk/src/rp2_common/hardware_gpio/gpio.c.obj
 .text.gpio_set_oeover
                0x00000000       0x24 CMakeFiles/main.dir/__/pico-sdk/src/rp2_common/hardware_gpio/gpio.c.obj
 .text.gpio_set_input_hysteresis_enabled
                0x00000000       0x28 CMakeFiles/main.dir/__/pico-sdk/src/rp2_common/hardware_gpio/gpio.c.obj
 .text.gpio_is_input_hysteresis_enabled
                0x00000000       0x14 CMakeFiles/main.dir/__/pico-sdk/src/rp2_common/hardware_gpio/gpio.c.obj
 .text.gpio_set_slew_rate
                0x00000000       0x20 CMakeFiles/main.dir/__/pico-sdk/src/rp2_common/hardware_gpio/gpio.c.obj
 .text.gpio_get_slew_rate
                0x00000000       0x14 CMakeFiles/main.dir/__/pico-sdk/src/rp2_common/hardware_gpio/gpio.c.obj
 .text.gpio_set_drive_strength
                0x00000000       0x20 CMakeFiles/main.dir/__/pico-sdk/src/rp2_common/hardware_gpio/gpio.c.obj
 .text.gpio_get_drive_strength
                0x00000000       0x14 CMakeFiles/main.dir/__/pico-sdk/src/rp2_common/hardware_gpio/gpio.c.obj
 .text.gpio_set_irq_enabled
                0x00000000       0x50 CMakeFiles/main.dir/__/pico-sdk/src/rp2_common/hardware_gpio/gpio.c.obj
 .text.gpio_set_irq_enabled_with_callback
                0x00000000       0x74 CMakeFiles/main.dir/__/pico-sdk/src/rp2_common/hardware_gpio/gpio.c.obj
 .text.gpio_set_dormant_irq_enabled
                0x00000000       0x40 CMakeFiles/main.dir/__/pico-sdk/src/rp2_common/hardware_gpio/gpio.c.obj
 .text.gpio_acknowledge_irq
                0x00000000       0x18 CMakeFiles/main.dir/__/pico-sdk/src/rp2_common/hardware_gpio/gpio.c.obj
 .text.gpio_debug_pins_init
                0x00000000       0x84 CMakeFiles/main.dir/__/pico-sdk/src/rp2_common/hardware_gpio/gpio.c.obj
 .text.gpio_set_input_enabled
                0x00000000       0x28 CMakeFiles/main.dir/__/pico-sdk/src/rp2_common/hardware_gpio/gpio.c.obj
 .text.gpio_init_mask
                0x00000000       0x68 CMakeFiles/main.dir/__/pico-sdk/src/rp2_common/hardware_gpio/gpio.c.obj
 .bss._callbacks
                0x00000000        0x8 CMakeFiles/main.dir/__/pico-sdk/src/rp2_common/hardware_gpio/gpio.c.obj
 .text          0x00000000        0x0 CMakeFiles/main.dir/__/pico-sdk/src/rp2_common/hardware_claim/claim.c.obj
 .data          0x00000000        0x0 CMakeFiles/main.dir/__/pico-sdk/src/rp2_common/hardware_claim/claim.c.obj
 .bss           0x00000000        0x0 CMakeFiles/main.dir/__/pico-sdk/src/rp2_common/hardware_claim/claim.c.obj
 .text.hw_claim_lock
                0x00000000       0x18 CMakeFiles/main.dir/__/pico-sdk/src/rp2_common/hardware_claim/claim.c.obj
 .text.hw_claim_unlock
                0x00000000       0x14 CMakeFiles/main.dir/__/pico-sdk/src/rp2_common/hardware_claim/claim.c.obj
 .text.hw_is_claimed
                0x00000000       0x18 CMakeFiles/main.dir/__/pico-sdk/src/rp2_common/hardware_claim/claim.c.obj
 .text.hw_claim_clear
                0x00000000       0x38 CMakeFiles/main.dir/__/pico-sdk/src/rp2_common/hardware_claim/claim.c.obj
 .text          0x00000000        0x0 CMakeFiles/main.dir/__/pico-sdk/src/rp2_common/pico_platform/platform.c.obj
 .data          0x00000000        0x0 CMakeFiles/main.dir/__/pico-sdk/src/rp2_common/pico_platform/platform.c.obj
 .bss           0x00000000        0x0 CMakeFiles/main.dir/__/pico-sdk/src/rp2_common/pico_platform/platform.c.obj
 .text.rp2040_chip_version
                0x00000000        0xc CMakeFiles/main.dir/__/pico-sdk/src/rp2_common/pico_platform/platform.c.obj
 .text          0x00000000        0x0 CMakeFiles/main.dir/__/pico-sdk/src/rp2_common/hardware_sync/sync.c.obj
 .data          0x00000000        0x0 CMakeFiles/main.dir/__/pico-sdk/src/rp2_common/hardware_sync/sync.c.obj
 .bss           0x00000000        0x0 CMakeFiles/main.dir/__/pico-sdk/src/rp2_common/hardware_sync/sync.c.obj
 .text.spin_lock_init
                0x00000000       0x18 CMakeFiles/main.dir/__/pico-sdk/src/rp2_common/hardware_sync/sync.c.obj
 .text.spin_lock_claim
                0x00000000       0x18 CMakeFiles/main.dir/__/pico-sdk/src/rp2_common/hardware_sync/sync.c.obj
 .text.spin_lock_claim_mask
                0x00000000       0x40 CMakeFiles/main.dir/__/pico-sdk/src/rp2_common/hardware_sync/sync.c.obj
 .text.spin_lock_unclaim
                0x00000000       0x24 CMakeFiles/main.dir/__/pico-sdk/src/rp2_common/hardware_sync/sync.c.obj
 .text.spin_lock_is_claimed
                0x00000000       0x10 CMakeFiles/main.dir/__/pico-sdk/src/rp2_common/hardware_sync/sync.c.obj
 .rodata.spin_lock_claim.str1.4
                0x00000000       0x1f CMakeFiles/main.dir/__/pico-sdk/src/rp2_common/hardware_sync/sync.c.obj
 .text          0x00000000        0x0 CMakeFiles/main.dir/__/pico-sdk/src/rp2_common/hardware_uart/uart.c.obj
 .data          0x00000000        0x0 CMakeFiles/main.dir/__/pico-sdk/src/rp2_common/hardware_uart/uart.c.obj
 .bss           0x00000000        0x0 CMakeFiles/main.dir/__/pico-sdk/src/rp2_common/hardware_uart/uart.c.obj
 .text.uart_init
                0x00000000       0xe8 CMakeFiles/main.dir/__/pico-sdk/src/rp2_common/hardware_uart/uart.c.obj
 .text.uart_deinit
                0x00000000       0x24 CMakeFiles/main.dir/__/pico-sdk/src/rp2_common/hardware_uart/uart.c.obj
 .text.uart_set_baudrate
                0x00000000       0x68 CMakeFiles/main.dir/__/pico-sdk/src/rp2_common/hardware_uart/uart.c.obj
 .text.uart_set_translate_crlf
                0x00000000       0x28 CMakeFiles/main.dir/__/pico-sdk/src/rp2_common/hardware_uart/uart.c.obj
 .text.uart_is_readable_within_us
                0x00000000       0x24 CMakeFiles/main.dir/__/pico-sdk/src/rp2_common/hardware_uart/uart.c.obj
 .comment       0x00000000       0x58 CMakeFiles/main.dir/__/pico-sdk/src/rp2_common/hardware_uart/uart.c.obj
 .ARM.attributes
                0x00000000       0x32 CMakeFiles/main.dir/__/pico-sdk/src/rp2_common/hardware_uart/uart.c.obj
 COMMON         0x00000000        0x4 CMakeFiles/main.dir/__/pico-sdk/src/rp2_common/hardware_uart/uart.c.obj
 .text          0x00000000        0x0 CMakeFiles/main.dir/__/pico-sdk/src/rp2_common/hardware_divider/divider.S.obj
 .data          0x00000000        0x0 CMakeFiles/main.dir/__/pico-sdk/src/rp2_common/hardware_divider/divider.S.obj
 .bss           0x00000000        0x0 CMakeFiles/main.dir/__/pico-sdk/src/rp2_common/hardware_divider/divider.S.obj
 .text.hw_divider_divmod_s32
                0x00000000       0x18 CMakeFiles/main.dir/__/pico-sdk/src/rp2_common/hardware_divider/divider.S.obj
 .text.hw_divider_divmod_u32
                0x00000000       0x18 CMakeFiles/main.dir/__/pico-sdk/src/rp2_common/hardware_divider/divider.S.obj
 .text.hw_divider_save_state
                0x00000000       0x1c CMakeFiles/main.dir/__/pico-sdk/src/rp2_common/hardware_divider/divider.S.obj
 .text.hw_divider_restore_state
                0x00000000       0x14 CMakeFiles/main.dir/__/pico-sdk/src/rp2_common/hardware_divider/divider.S.obj
 .ARM.attributes
                0x00000000       0x22 CMakeFiles/main.dir/__/pico-sdk/src/rp2_common/hardware_divider/divider.S.obj
 .text          0x00000000        0x0 CMakeFiles/main.dir/__/pico-sdk/src/common/pico_time/time.c.obj
 .data          0x00000000        0x0 CMakeFiles/main.dir/__/pico-sdk/src/common/pico_time/time.c.obj
 .bss           0x00000000        0x0 CMakeFiles/main.dir/__/pico-sdk/src/common/pico_time/time.c.obj
 .text.repeating_timer_callback
                0x00000000       0x1c CMakeFiles/main.dir/__/pico-sdk/src/common/pico_time/time.c.obj
 .text.alarm_pool_dump_key
                0x00000000       0x34 CMakeFiles/main.dir/__/pico-sdk/src/common/pico_time/time.c.obj
 .text.alarm_pool_create
                0x00000000       0x6c CMakeFiles/main.dir/__/pico-sdk/src/common/pico_time/time.c.obj
 .text.alarm_pool_destroy
                0x00000000       0x44 CMakeFiles/main.dir/__/pico-sdk/src/common/pico_time/time.c.obj
 .text.alarm_pool_cancel_alarm
                0x00000000       0x70 CMakeFiles/main.dir/__/pico-sdk/src/common/pico_time/time.c.obj
 .text.alarm_pool_hardware_alarm_num
                0x00000000        0x4 CMakeFiles/main.dir/__/pico-sdk/src/common/pico_time/time.c.obj
 .text.alarm_pool_add_repeating_timer_us
                0x00000000      0x200 CMakeFiles/main.dir/__/pico-sdk/src/common/pico_time/time.c.obj
 .text.cancel_repeating_timer
                0x00000000       0x84 CMakeFiles/main.dir/__/pico-sdk/src/common/pico_time/time.c.obj
 .text.alarm_pool_dump
                0x00000000       0x34 CMakeFiles/main.dir/__/pico-sdk/src/common/pico_time/time.c.obj
 .text.sleep_us
                0x00000000       0x30 CMakeFiles/main.dir/__/pico-sdk/src/common/pico_time/time.c.obj
 .rodata.alarm_pool_dump_key.str1.4
                0x00000000        0xf CMakeFiles/main.dir/__/pico-sdk/src/common/pico_time/time.c.obj
 .rodata.at_the_end_of_time
                0x00000000        0x8 CMakeFiles/main.dir/__/pico-sdk/src/common/pico_time/time.c.obj
 .rodata.nil_time
                0x00000000        0x8 CMakeFiles/main.dir/__/pico-sdk/src/common/pico_time/time.c.obj
 .text          0x00000000        0x0 CMakeFiles/main.dir/__/pico-sdk/src/common/pico_time/timeout_helper.c.obj
 .data          0x00000000        0x0 CMakeFiles/main.dir/__/pico-sdk/src/common/pico_time/timeout_helper.c.obj
 .bss           0x00000000        0x0 CMakeFiles/main.dir/__/pico-sdk/src/common/pico_time/timeout_helper.c.obj
 .text.check_per_iteration_timeout_us
                0x00000000       0x4c CMakeFiles/main.dir/__/pico-sdk/src/common/pico_time/timeout_helper.c.obj
 .text.init_per_iteration_timeout_us
                0x00000000       0x38 CMakeFiles/main.dir/__/pico-sdk/src/common/pico_time/timeout_helper.c.obj
 .text          0x00000000        0x0 CMakeFiles/main.dir/__/pico-sdk/src/rp2_common/hardware_timer/timer.c.obj
 .data          0x00000000        0x0 CMakeFiles/main.dir/__/pico-sdk/src/rp2_common/hardware_timer/timer.c.obj
 .bss           0x00000000        0x0 CMakeFiles/main.dir/__/pico-sdk/src/rp2_common/hardware_timer/timer.c.obj
 .text.hardware_alarm_unclaim
                0x00000000       0x10 CMakeFiles/main.dir/__/pico-sdk/src/rp2_common/hardware_timer/timer.c.obj
 .text.hardware_alarm_is_claimed
                0x00000000       0x10 CMakeFiles/main.dir/__/pico-sdk/src/rp2_common/hardware_timer/timer.c.obj
 .text.busy_wait_us_32
                0x00000000       0x6c CMakeFiles/main.dir/__/pico-sdk/src/rp2_common/hardware_timer/timer.c.obj
 .text.busy_wait_ms
                0x00000000       0x94 CMakeFiles/main.dir/__/pico-sdk/src/rp2_common/hardware_timer/timer.c.obj
 .text          0x00000000        0x0 CMakeFiles/main.dir/__/pico-sdk/src/common/pico_sync/sem.c.obj
 .data          0x00000000        0x0 CMakeFiles/main.dir/__/pico-sdk/src/common/pico_sync/sem.c.obj
 .bss           0x00000000        0x0 CMakeFiles/main.dir/__/pico-sdk/src/common/pico_sync/sem.c.obj
 .text.sem_init
                0x00000000       0x20 CMakeFiles/main.dir/__/pico-sdk/src/common/pico_sync/sem.c.obj
 .time_critical.sem_available
                0x00000000        0x8 CMakeFiles/main.dir/__/pico-sdk/src/common/pico_sync/sem.c.obj
 .time_critical.sem_acquire_blocking
                0x00000000       0x44 CMakeFiles/main.dir/__/pico-sdk/src/common/pico_sync/sem.c.obj
 .time_critical.sem_acquire_timeout_ms
                0x00000000       0x8c CMakeFiles/main.dir/__/pico-sdk/src/common/pico_sync/sem.c.obj
 .time_critical.sem_acquire_timeout_us
                0x00000000       0x78 CMakeFiles/main.dir/__/pico-sdk/src/common/pico_sync/sem.c.obj
 .time_critical.sem_acquire_block_until
                0x00000000       0x5c CMakeFiles/main.dir/__/pico-sdk/src/common/pico_sync/sem.c.obj
 .time_critical.sem_release
                0x00000000       0x4c CMakeFiles/main.dir/__/pico-sdk/src/common/pico_sync/sem.c.obj
 .time_critical.sem_reset
                0x00000000       0x40 CMakeFiles/main.dir/__/pico-sdk/src/common/pico_sync/sem.c.obj
 .comment       0x00000000       0x58 CMakeFiles/main.dir/__/pico-sdk/src/common/pico_sync/sem.c.obj
 .ARM.attributes
                0x00000000       0x32 CMakeFiles/main.dir/__/pico-sdk/src/common/pico_sync/sem.c.obj
 .text          0x00000000        0x0 CMakeFiles/main.dir/__/pico-sdk/src/common/pico_sync/lock_core.c.obj
 .data          0x00000000        0x0 CMakeFiles/main.dir/__/pico-sdk/src/common/pico_sync/lock_core.c.obj
 .bss           0x00000000        0x0 CMakeFiles/main.dir/__/pico-sdk/src/common/pico_sync/lock_core.c.obj
 .text          0x00000000        0x0 CMakeFiles/main.dir/__/pico-sdk/src/common/pico_sync/mutex.c.obj
 .data          0x00000000        0x0 CMakeFiles/main.dir/__/pico-sdk/src/common/pico_sync/mutex.c.obj
 .bss           0x00000000        0x0 CMakeFiles/main.dir/__/pico-sdk/src/common/pico_sync/mutex.c.obj
 .time_critical.recursive_mutex_enter_blocking
                0x00000000       0x50 CMakeFiles/main.dir/__/pico-sdk/src/common/pico_sync/mutex.c.obj
 .time_critical.recursive_mutex_try_enter
                0x00000000       0x54 CMakeFiles/main.dir/__/pico-sdk/src/common/pico_sync/mutex.c.obj
 .time_critical.recursive_mutex_enter_timeout_ms
                0x00000000       0xac CMakeFiles/main.dir/__/pico-sdk/src/common/pico_sync/mutex.c.obj
 .time_critical.mutex_enter_timeout_us
                0x00000000       0x84 CMakeFiles/main.dir/__/pico-sdk/src/common/pico_sync/mutex.c.obj
 .time_critical.recursive_mutex_enter_timeout_us
                0x00000000       0x90 CMakeFiles/main.dir/__/pico-sdk/src/common/pico_sync/mutex.c.obj
 .time_critical.mutex_enter_block_until
                0x00000000       0x68 CMakeFiles/main.dir/__/pico-sdk/src/common/pico_sync/mutex.c.obj
 .time_critical.recursive_mutex_enter_block_until
                0x00000000       0x74 CMakeFiles/main.dir/__/pico-sdk/src/common/pico_sync/mutex.c.obj
 .time_critical.recursive_mutex_exit
                0x00000000       0x44 CMakeFiles/main.dir/__/pico-sdk/src/common/pico_sync/mutex.c.obj
 .text          0x00000000        0x0 CMakeFiles/main.dir/__/pico-sdk/src/common/pico_sync/critical_section.c.obj
 .data          0x00000000        0x0 CMakeFiles/main.dir/__/pico-sdk/src/common/pico_sync/critical_section.c.obj
 .bss           0x00000000        0x0 CMakeFiles/main.dir/__/pico-sdk/src/common/pico_sync/critical_section.c.obj
 .text.critical_section_init_with_lock_num
                0x00000000       0x14 CMakeFiles/main.dir/__/pico-sdk/src/common/pico_sync/critical_section.c.obj
 .text.critical_section_deinit
                0x00000000       0x18 CMakeFiles/main.dir/__/pico-sdk/src/common/pico_sync/critical_section.c.obj
 .text          0x00000000        0x0 CMakeFiles/main.dir/__/pico-sdk/src/common/pico_util/datetime.c.obj
 .data          0x00000000        0x0 CMakeFiles/main.dir/__/pico-sdk/src/common/pico_util/datetime.c.obj
 .bss           0x00000000        0x0 CMakeFiles/main.dir/__/pico-sdk/src/common/pico_util/datetime.c.obj
 .text.datetime_to_str
                0x00000000       0x50 CMakeFiles/main.dir/__/pico-sdk/src/common/pico_util/datetime.c.obj
 .rodata.DATETIME_DOWS
                0x00000000       0x1c CMakeFiles/main.dir/__/pico-sdk/src/common/pico_util/datetime.c.obj
 .rodata.DATETIME_MONTHS
                0x00000000       0x30 CMakeFiles/main.dir/__/pico-sdk/src/common/pico_util/datetime.c.obj
 .rodata.datetime_to_str.str1.4
                0x00000000       0x19 CMakeFiles/main.dir/__/pico-sdk/src/common/pico_util/datetime.c.obj
 .rodata.str1.4
                0x00000000       0xad CMakeFiles/main.dir/__/pico-sdk/src/common/pico_util/datetime.c.obj
 .comment       0x00000000       0x58 CMakeFiles/main.dir/__/pico-sdk/src/common/pico_util/datetime.c.obj
 .ARM.attributes
                0x00000000       0x32 CMakeFiles/main.dir/__/pico-sdk/src/common/pico_util/datetime.c.obj
 .text          0x00000000        0x0 CMakeFiles/main.dir/__/pico-sdk/src/common/pico_util/pheap.c.obj
 .data          0x00000000        0x0 CMakeFiles/main.dir/__/pico-sdk/src/common/pico_util/pheap.c.obj
 .bss           0x00000000        0x0 CMakeFiles/main.dir/__/pico-sdk/src/common/pico_util/pheap.c.obj
 .text.ph_dump_node
                0x00000000      0x488 CMakeFiles/main.dir/__/pico-sdk/src/common/pico_util/pheap.c.obj
 .text.ph_create
                0x00000000       0x54 CMakeFiles/main.dir/__/pico-sdk/src/common/pico_util/pheap.c.obj
 .text.ph_clear
                0x00000000       0x30 CMakeFiles/main.dir/__/pico-sdk/src/common/pico_util/pheap.c.obj
 .text.ph_destroy
                0x00000000       0x14 CMakeFiles/main.dir/__/pico-sdk/src/common/pico_util/pheap.c.obj
 .text.ph_merge_two_pass
                0x00000000       0xc4 CMakeFiles/main.dir/__/pico-sdk/src/common/pico_util/pheap.c.obj
 .text.ph_dump  0x00000000       0xd4 CMakeFiles/main.dir/__/pico-sdk/src/common/pico_util/pheap.c.obj
 .rodata.ph_dump.str1.4
                0x00000000        0xf CMakeFiles/main.dir/__/pico-sdk/src/common/pico_util/pheap.c.obj
 .rodata.ph_dump_node.str1.4
                0x00000000       0x15 CMakeFiles/main.dir/__/pico-sdk/src/common/pico_util/pheap.c.obj
 .text          0x00000000        0x0 CMakeFiles/main.dir/__/pico-sdk/src/common/pico_util/queue.c.obj
 .data          0x00000000        0x0 CMakeFiles/main.dir/__/pico-sdk/src/common/pico_util/queue.c.obj
 .bss           0x00000000        0x0 CMakeFiles/main.dir/__/pico-sdk/src/common/pico_util/queue.c.obj
 .text.queue_init_with_spinlock
                0x00000000       0x24 CMakeFiles/main.dir/__/pico-sdk/src/common/pico_util/queue.c.obj
 .text.queue_free
                0x00000000        0xc CMakeFiles/main.dir/__/pico-sdk/src/common/pico_util/queue.c.obj
 .text.queue_try_add
                0x00000000       0x70 CMakeFiles/main.dir/__/pico-sdk/src/common/pico_util/queue.c.obj
 .text.queue_try_remove
                0x00000000       0x70 CMakeFiles/main.dir/__/pico-sdk/src/common/pico_util/queue.c.obj
 .text.queue_try_peek
                0x00000000       0x5c CMakeFiles/main.dir/__/pico-sdk/src/common/pico_util/queue.c.obj
 .text.queue_add_blocking
                0x00000000       0x74 CMakeFiles/main.dir/__/pico-sdk/src/common/pico_util/queue.c.obj
 .text.queue_remove_blocking
                0x00000000       0x74 CMakeFiles/main.dir/__/pico-sdk/src/common/pico_util/queue.c.obj
 .text.queue_peek_blocking
                0x00000000       0x60 CMakeFiles/main.dir/__/pico-sdk/src/common/pico_util/queue.c.obj
 .comment       0x00000000       0x58 CMakeFiles/main.dir/__/pico-sdk/src/common/pico_util/queue.c.obj
 .ARM.attributes
                0x00000000       0x32 CMakeFiles/main.dir/__/pico-sdk/src/common/pico_util/queue.c.obj
 .text          0x00000000        0x0 CMakeFiles/main.dir/__/pico-sdk/src/rp2_common/pico_runtime/runtime.c.obj
 .data          0x00000000        0x0 CMakeFiles/main.dir/__/pico-sdk/src/rp2_common/pico_runtime/runtime.c.obj
 .bss           0x00000000        0x0 CMakeFiles/main.dir/__/pico-sdk/src/rp2_common/pico_runtime/runtime.c.obj
 .text.runtime_install_stack_guard
                0x00000000       0x38 CMakeFiles/main.dir/__/pico-sdk/src/rp2_common/pico_runtime/runtime.c.obj
 .text.__assert_func
                0x00000000       0x34 CMakeFiles/main.dir/__/pico-sdk/src/rp2_common/pico_runtime/runtime.c.obj
 .text.panic_unsupported
                0x00000000        0xc CMakeFiles/main.dir/__/pico-sdk/src/rp2_common/pico_runtime/runtime.c.obj
 .rodata.__assert_func.str1.4
                0x00000000       0x43 CMakeFiles/main.dir/__/pico-sdk/src/rp2_common/pico_runtime/runtime.c.obj
 .rodata.panic_unsupported.str1.4
                0x00000000        0xe CMakeFiles/main.dir/__/pico-sdk/src/rp2_common/pico_runtime/runtime.c.obj
 .text          0x00000000        0x0 CMakeFiles/main.dir/__/pico-sdk/src/rp2_common/hardware_clocks/clocks.c.obj
 .data          0x00000000        0x0 CMakeFiles/main.dir/__/pico-sdk/src/rp2_common/hardware_clocks/clocks.c.obj
 .bss           0x00000000        0x0 CMakeFiles/main.dir/__/pico-sdk/src/rp2_common/hardware_clocks/clocks.c.obj
 .text.clocks_irq_handler
                0x00000000       0xc4 CMakeFiles/main.dir/__/pico-sdk/src/rp2_common/hardware_clocks/clocks.c.obj
 .text.clock_stop
                0x00000000       0x2c CMakeFiles/main.dir/__/pico-sdk/src/rp2_common/hardware_clocks/clocks.c.obj
 .text.clock_configure
                0x00000000      0x144 CMakeFiles/main.dir/__/pico-sdk/src/rp2_common/hardware_clocks/clocks.c.obj
 .text.clock_set_reported_hz
                0x00000000        0xc CMakeFiles/main.dir/__/pico-sdk/src/rp2_common/hardware_clocks/clocks.c.obj
 .text.frequency_count_khz
                0x00000000       0x44 CMakeFiles/main.dir/__/pico-sdk/src/rp2_common/hardware_clocks/clocks.c.obj
 .text.clocks_enable_resus
                0x00000000       0x34 CMakeFiles/main.dir/__/pico-sdk/src/rp2_common/hardware_clocks/clocks.c.obj
 .text.clock_gpio_init
                0x00000000       0x50 CMakeFiles/main.dir/__/pico-sdk/src/rp2_common/hardware_clocks/clocks.c.obj
 .text.clock_configure_gpin
                0x00000000      0x108 CMakeFiles/main.dir/__/pico-sdk/src/rp2_common/hardware_clocks/clocks.c.obj
 .bss._resus_callback
                0x00000000        0x4 CMakeFiles/main.dir/__/pico-sdk/src/rp2_common/hardware_clocks/clocks.c.obj
 .rodata.gpin0_src
                0x00000000        0xa CMakeFiles/main.dir/__/pico-sdk/src/rp2_common/hardware_clocks/clocks.c.obj
 .text          0x00000000        0x0 CMakeFiles/main.dir/__/pico-sdk/src/rp2_common/hardware_irq/irq.c.obj
 .data          0x00000000        0x0 CMakeFiles/main.dir/__/pico-sdk/src/rp2_common/hardware_irq/irq.c.obj
 .bss           0x00000000        0x0 CMakeFiles/main.dir/__/pico-sdk/src/rp2_common/hardware_irq/irq.c.obj
 .text.irq_is_enabled
                0x00000000       0x18 CMakeFiles/main.dir/__/pico-sdk/src/rp2_common/hardware_irq/irq.c.obj
 .text.irq_set_mask_enabled
                0x00000000       0x20 CMakeFiles/main.dir/__/pico-sdk/src/rp2_common/hardware_irq/irq.c.obj
 .text.irq_get_exclusive_handler
                0x00000000       0x50 CMakeFiles/main.dir/__/pico-sdk/src/rp2_common/hardware_irq/irq.c.obj
 .text.irq_add_shared_handler
                0x00000000      0x1c8 CMakeFiles/main.dir/__/pico-sdk/src/rp2_common/hardware_irq/irq.c.obj
 .text.irq_set_priority
                0x00000000       0x28 CMakeFiles/main.dir/__/pico-sdk/src/rp2_common/hardware_irq/irq.c.obj
 .text.irq_get_priority
                0x00000000       0x20 CMakeFiles/main.dir/__/pico-sdk/src/rp2_common/hardware_irq/irq.c.obj
 .text          0x00000000        0x0 CMakeFiles/main.dir/__/pico-sdk/src/rp2_common/hardware_irq/irq_handler_chain.S.obj
 .bss           0x00000000        0x0 CMakeFiles/main.dir/__/pico-sdk/src/rp2_common/hardware_irq/irq_handler_chain.S.obj
 .text          0x00000000        0x0 CMakeFiles/main.dir/__/pico-sdk/src/rp2_common/hardware_pll/pll.c.obj
 .data          0x00000000        0x0 CMakeFiles/main.dir/__/pico-sdk/src/rp2_common/hardware_pll/pll.c.obj
 .bss           0x00000000        0x0 CMakeFiles/main.dir/__/pico-sdk/src/rp2_common/hardware_pll/pll.c.obj
 .text.pll_deinit
                0x00000000        0x8 CMakeFiles/main.dir/__/pico-sdk/src/rp2_common/hardware_pll/pll.c.obj
 .text          0x00000000        0x0 CMakeFiles/main.dir/__/pico-sdk/src/rp2_common/hardware_vreg/vreg.c.obj
 .data          0x00000000        0x0 CMakeFiles/main.dir/__/pico-sdk/src/rp2_common/hardware_vreg/vreg.c.obj
 .bss           0x00000000        0x0 CMakeFiles/main.dir/__/pico-sdk/src/rp2_common/hardware_vreg/vreg.c.obj
 .text.vreg_set_voltage
                0x00000000       0x1c CMakeFiles/main.dir/__/pico-sdk/src/rp2_common/hardware_vreg/vreg.c.obj
 .comment       0x00000000       0x58 CMakeFiles/main.dir/__/pico-sdk/src/rp2_common/hardware_vreg/vreg.c.obj
 .ARM.attributes
                0x00000000       0x32 CMakeFiles/main.dir/__/pico-sdk/src/rp2_common/hardware_vreg/vreg.c.obj
 .text          0x00000000        0x0 CMakeFiles/main.dir/__/pico-sdk/src/rp2_common/hardware_watchdog/watchdog.c.obj
 .data          0x00000000        0x0 CMakeFiles/main.dir/__/pico-sdk/src/rp2_common/hardware_watchdog/watchdog.c.obj
 .bss           0x00000000        0x0 CMakeFiles/main.dir/__/pico-sdk/src/rp2_common/hardware_watchdog/watchdog.c.obj
 .text.watchdog_update
                0x00000000       0x14 CMakeFiles/main.dir/__/pico-sdk/src/rp2_common/hardware_watchdog/watchdog.c.obj
 .text.watchdog_get_count
                0x00000000       0x10 CMakeFiles/main.dir/__/pico-sdk/src/rp2_common/hardware_watchdog/watchdog.c.obj
 .text._watchdog_enable
                0x00000000       0x7c CMakeFiles/main.dir/__/pico-sdk/src/rp2_common/hardware_watchdog/watchdog.c.obj
 .text.watchdog_enable
                0x00000000       0x84 CMakeFiles/main.dir/__/pico-sdk/src/rp2_common/hardware_watchdog/watchdog.c.obj
 .text.watchdog_caused_reboot
                0x00000000       0x10 CMakeFiles/main.dir/__/pico-sdk/src/rp2_common/hardware_watchdog/watchdog.c.obj
 .text.watchdog_enable_caused_reboot
                0x00000000       0x24 CMakeFiles/main.dir/__/pico-sdk/src/rp2_common/hardware_watchdog/watchdog.c.obj
 .text          0x00000000        0x0 CMakeFiles/main.dir/__/pico-sdk/src/rp2_common/hardware_xosc/xosc.c.obj
 .data          0x00000000        0x0 CMakeFiles/main.dir/__/pico-sdk/src/rp2_common/hardware_xosc/xosc.c.obj
 .bss           0x00000000        0x0 CMakeFiles/main.dir/__/pico-sdk/src/rp2_common/hardware_xosc/xosc.c.obj
 .text.xosc_disable
                0x00000000       0x24 CMakeFiles/main.dir/__/pico-sdk/src/rp2_common/hardware_xosc/xosc.c.obj
 .text.xosc_dormant
                0x00000000       0x18 CMakeFiles/main.dir/__/pico-sdk/src/rp2_common/hardware_xosc/xosc.c.obj
 .text          0x00000000        0x0 CMakeFiles/main.dir/__/pico-sdk/src/rp2_common/pico_printf/printf.c.obj
 .data          0x00000000        0x0 CMakeFiles/main.dir/__/pico-sdk/src/rp2_common/pico_printf/printf.c.obj
 .bss           0x00000000        0x0 CMakeFiles/main.dir/__/pico-sdk/src/rp2_common/pico_printf/printf.c.obj
 .text.__wrap_snprintf
                0x00000000       0x28 CMakeFiles/main.dir/__/pico-sdk/src/rp2_common/pico_printf/printf.c.obj
 .text.weak_raw_printf
                0x00000000       0x40 CMakeFiles/main.dir/__/pico-sdk/src/rp2_common/pico_printf/printf.c.obj
 .data          0x00000000        0x0 CMakeFiles/main.dir/__/pico-sdk/src/rp2_common/pico_bit_ops/bit_ops_aeabi.S.obj
 .bss           0x00000000        0x0 CMakeFiles/main.dir/__/pico-sdk/src/rp2_common/pico_bit_ops/bit_ops_aeabi.S.obj
 .text.clzsi    0x00000000        0xc CMakeFiles/main.dir/__/pico-sdk/src/rp2_common/pico_bit_ops/bit_ops_aeabi.S.obj
 .text.ctzsi    0x00000000        0xc CMakeFiles/main.dir/__/pico-sdk/src/rp2_common/pico_bit_ops/bit_ops_aeabi.S.obj
 .text.popcountsi
                0x00000000        0xc CMakeFiles/main.dir/__/pico-sdk/src/rp2_common/pico_bit_ops/bit_ops_aeabi.S.obj
 .text.clzdi    0x00000000       0x18 CMakeFiles/main.dir/__/pico-sdk/src/rp2_common/pico_bit_ops/bit_ops_aeabi.S.obj
 .text.ctzdi    0x00000000       0x18 CMakeFiles/main.dir/__/pico-sdk/src/rp2_common/pico_bit_ops/bit_ops_aeabi.S.obj
 .text.popcountdi
                0x00000000       0x18 CMakeFiles/main.dir/__/pico-sdk/src/rp2_common/pico_bit_ops/bit_ops_aeabi.S.obj
 .text.reverse32
                0x00000000        0xc CMakeFiles/main.dir/__/pico-sdk/src/rp2_common/pico_bit_ops/bit_ops_aeabi.S.obj
 .text.__rev    0x00000000        0xc CMakeFiles/main.dir/__/pico-sdk/src/rp2_common/pico_bit_ops/bit_ops_aeabi.S.obj
 .text.__revll  0x00000000       0x18 CMakeFiles/main.dir/__/pico-sdk/src/rp2_common/pico_bit_ops/bit_ops_aeabi.S.obj
 .text          0x00000000        0x0 CMakeFiles/main.dir/__/pico-sdk/src/rp2_common/pico_bootrom/bootrom.c.obj
 .data          0x00000000        0x0 CMakeFiles/main.dir/__/pico-sdk/src/rp2_common/pico_bootrom/bootrom.c.obj
 .bss           0x00000000        0x0 CMakeFiles/main.dir/__/pico-sdk/src/rp2_common/pico_bootrom/bootrom.c.obj
 .text          0x00000000        0x0 CMakeFiles/main.dir/__/pico-sdk/src/rp2_common/pico_divider/divider.S.obj
 .data          0x00000000        0x0 CMakeFiles/main.dir/__/pico-sdk/src/rp2_common/pico_divider/divider.S.obj
 .bss           0x00000000        0x0 CMakeFiles/main.dir/__/pico-sdk/src/rp2_common/pico_divider/divider.S.obj
 .text.divmod_s64s64_rem
                0x00000000        0xc CMakeFiles/main.dir/__/pico-sdk/src/rp2_common/pico_divider/divider.S.obj
 .text.divmod_u64u64_rem
                0x00000000        0xc CMakeFiles/main.dir/__/pico-sdk/src/rp2_common/pico_divider/divider.S.obj
 .text          0x00000000        0x0 CMakeFiles/main.dir/__/pico-sdk/src/rp2_common/pico_double/double_aeabi.S.obj
 .data          0x00000000        0x0 CMakeFiles/main.dir/__/pico-sdk/src/rp2_common/pico_double/double_aeabi.S.obj
 .bss           0x00000000        0x0 CMakeFiles/main.dir/__/pico-sdk/src/rp2_common/pico_double/double_aeabi.S.obj
 .text.push_r8_r11
                0x00000000        0xc CMakeFiles/main.dir/__/pico-sdk/src/rp2_common/pico_double/double_aeabi.S.obj
 .text.pop_r8_r11
                0x00000000        0xc CMakeFiles/main.dir/__/pico-sdk/src/rp2_common/pico_double/double_aeabi.S.obj
 .text.__wrap___aeabi_dcmpeq
                0x00000000       0x10 CMakeFiles/main.dir/__/pico-sdk/src/rp2_common/pico_double/double_aeabi.S.obj
 .text.__wrap___aeabi_ui2d
                0x00000000       0x18 CMakeFiles/main.dir/__/pico-sdk/src/rp2_common/pico_double/double_aeabi.S.obj
 .text.double2int
                0x00000000       0x18 CMakeFiles/main.dir/__/pico-sdk/src/rp2_common/pico_double/double_aeabi.S.obj
 .text.fix2double
                0x00000000       0x18 CMakeFiles/main.dir/__/pico-sdk/src/rp2_common/pico_double/double_aeabi.S.obj
 .text.ufix2double
                0x00000000       0x28 CMakeFiles/main.dir/__/pico-sdk/src/rp2_common/pico_double/double_aeabi.S.obj
 .text.fix642double
                0x00000000       0x18 CMakeFiles/main.dir/__/pico-sdk/src/rp2_common/pico_double/double_aeabi.S.obj
 .text.__wrap___aeabi_l2d
                0x00000000       0x18 CMakeFiles/main.dir/__/pico-sdk/src/rp2_common/pico_double/double_aeabi.S.obj
 .text.__wrap___aeabi_ul2d
                0x00000000       0x18 CMakeFiles/main.dir/__/pico-sdk/src/rp2_common/pico_double/double_aeabi.S.obj
 .text.__wrap___aeabi_d2lz
                0x00000000       0x26 CMakeFiles/main.dir/__/pico-sdk/src/rp2_common/pico_double/double_aeabi.S.obj
 .text.double2int64
                0x00000000       0x18 CMakeFiles/main.dir/__/pico-sdk/src/rp2_common/pico_double/double_aeabi.S.obj
 .text.double2fix64
                0x00000000       0x18 CMakeFiles/main.dir/__/pico-sdk/src/rp2_common/pico_double/double_aeabi.S.obj
 .text.double2ufix64
                0x00000000       0x18 CMakeFiles/main.dir/__/pico-sdk/src/rp2_common/pico_double/double_aeabi.S.obj
 .text.double2fix
                0x00000000       0x18 CMakeFiles/main.dir/__/pico-sdk/src/rp2_common/pico_double/double_aeabi.S.obj
 .text.double2ufix
                0x00000000       0x18 CMakeFiles/main.dir/__/pico-sdk/src/rp2_common/pico_double/double_aeabi.S.obj
 .text.__wrap___aeabi_d2f
                0x00000000       0x18 CMakeFiles/main.dir/__/pico-sdk/src/rp2_common/pico_double/double_aeabi.S.obj
 .text.__wrap_srqt
                0x00000000       0x18 CMakeFiles/main.dir/__/pico-sdk/src/rp2_common/pico_double/double_aeabi.S.obj
 .text.__wrap_sincostan_remainder
                0x00000000       0x14 CMakeFiles/main.dir/__/pico-sdk/src/rp2_common/pico_double/double_aeabi.S.obj
 .text.__wrap_cos
                0x00000000       0x2c CMakeFiles/main.dir/__/pico-sdk/src/rp2_common/pico_double/double_aeabi.S.obj
 .text.__wrap_sin
                0x00000000       0x2c CMakeFiles/main.dir/__/pico-sdk/src/rp2_common/pico_double/double_aeabi.S.obj
 .text.__wrap_sincos
                0x00000000       0xa0 CMakeFiles/main.dir/__/pico-sdk/src/rp2_common/pico_double/double_aeabi.S.obj
 .text.__wrap_tan
                0x00000000       0x5c CMakeFiles/main.dir/__/pico-sdk/src/rp2_common/pico_double/double_aeabi.S.obj
 .text.__wrap_atan2
                0x00000000       0x18 CMakeFiles/main.dir/__/pico-sdk/src/rp2_common/pico_double/double_aeabi.S.obj
 .text.__wrap_exp
                0x00000000       0x18 CMakeFiles/main.dir/__/pico-sdk/src/rp2_common/pico_double/double_aeabi.S.obj
 .text.__wrap_log
                0x00000000       0x18 CMakeFiles/main.dir/__/pico-sdk/src/rp2_common/pico_double/double_aeabi.S.obj
 .text          0x00000000        0x0 CMakeFiles/main.dir/__/pico-sdk/src/rp2_common/pico_double/double_init_rom.c.obj
 .data          0x00000000        0x0 CMakeFiles/main.dir/__/pico-sdk/src/rp2_common/pico_double/double_init_rom.c.obj
 .bss           0x00000000        0x0 CMakeFiles/main.dir/__/pico-sdk/src/rp2_common/pico_double/double_init_rom.c.obj
 .text          0x00000000        0x0 CMakeFiles/main.dir/__/pico-sdk/src/rp2_common/pico_double/double_math.c.obj
 .data          0x00000000        0x0 CMakeFiles/main.dir/__/pico-sdk/src/rp2_common/pico_double/double_math.c.obj
 .bss           0x00000000        0x0 CMakeFiles/main.dir/__/pico-sdk/src/rp2_common/pico_double/double_math.c.obj
 .text.dpow_1   0x00000000      0x27c CMakeFiles/main.dir/__/pico-sdk/src/rp2_common/pico_double/double_math.c.obj
 .text.dpow_int2
                0x00000000       0x64 CMakeFiles/main.dir/__/pico-sdk/src/rp2_common/pico_double/double_math.c.obj
 .text.dpow_0   0x00000000      0x260 CMakeFiles/main.dir/__/pico-sdk/src/rp2_common/pico_double/double_math.c.obj
 .text.dpowint_0
                0x00000000      0x260 CMakeFiles/main.dir/__/pico-sdk/src/rp2_common/pico_double/double_math.c.obj
 .text.__wrap_ldexp
                0x00000000       0x4c CMakeFiles/main.dir/__/pico-sdk/src/rp2_common/pico_double/double_math.c.obj
 .text.__wrap_copysign
                0x00000000       0x10 CMakeFiles/main.dir/__/pico-sdk/src/rp2_common/pico_double/double_math.c.obj
 .text.__wrap_trunc
                0x00000000       0x50 CMakeFiles/main.dir/__/pico-sdk/src/rp2_common/pico_double/double_math.c.obj
 .text.__wrap_round
                0x00000000       0xa0 CMakeFiles/main.dir/__/pico-sdk/src/rp2_common/pico_double/double_math.c.obj
 .text.__wrap_floor
                0x00000000       0x90 CMakeFiles/main.dir/__/pico-sdk/src/rp2_common/pico_double/double_math.c.obj
 .text.__wrap_ceil
                0x00000000       0x94 CMakeFiles/main.dir/__/pico-sdk/src/rp2_common/pico_double/double_math.c.obj
 .text.__wrap_asin
                0x00000000       0x58 CMakeFiles/main.dir/__/pico-sdk/src/rp2_common/pico_double/double_math.c.obj
 .text.__wrap_acos
                0x00000000       0x54 CMakeFiles/main.dir/__/pico-sdk/src/rp2_common/pico_double/double_math.c.obj
 .text.__wrap_atan
                0x00000000       0x40 CMakeFiles/main.dir/__/pico-sdk/src/rp2_common/pico_double/double_math.c.obj
 .text.__wrap_sinh
                0x00000000       0x54 CMakeFiles/main.dir/__/pico-sdk/src/rp2_common/pico_double/double_math.c.obj
 .text.__wrap_cosh
                0x00000000       0x54 CMakeFiles/main.dir/__/pico-sdk/src/rp2_common/pico_double/double_math.c.obj
 .text.__wrap_tanh
                0x00000000       0x68 CMakeFiles/main.dir/__/pico-sdk/src/rp2_common/pico_double/double_math.c.obj
 .text.__wrap_asinh
                0x00000000       0xb0 CMakeFiles/main.dir/__/pico-sdk/src/rp2_common/pico_double/double_math.c.obj
 .text.__wrap_acosh
                0x00000000       0x7c CMakeFiles/main.dir/__/pico-sdk/src/rp2_common/pico_double/double_math.c.obj
 .text.__wrap_atanh
                0x00000000       0x60 CMakeFiles/main.dir/__/pico-sdk/src/rp2_common/pico_double/double_math.c.obj
 .text.__wrap_exp2
                0x00000000       0xbc CMakeFiles/main.dir/__/pico-sdk/src/rp2_common/pico_double/double_math.c.obj
 .text.__wrap_log2
                0x00000000       0x18 CMakeFiles/main.dir/__/pico-sdk/src/rp2_common/pico_double/double_math.c.obj
 .text.__wrap_exp10
                0x00000000       0x14 CMakeFiles/main.dir/__/pico-sdk/src/rp2_common/pico_double/double_math.c.obj
 .text.__wrap_log10
                0x00000000       0x18 CMakeFiles/main.dir/__/pico-sdk/src/rp2_common/pico_double/double_math.c.obj
 .text.__wrap_expm1
                0x00000000       0x14 CMakeFiles/main.dir/__/pico-sdk/src/rp2_common/pico_double/double_math.c.obj
 .text.__wrap_log1p
                0x00000000       0x14 CMakeFiles/main.dir/__/pico-sdk/src/rp2_common/pico_double/double_math.c.obj
 .text.__wrap_fma
                0x00000000       0x10 CMakeFiles/main.dir/__/pico-sdk/src/rp2_common/pico_double/double_math.c.obj
 .text.__wrap_powint
                0x00000000       0xac CMakeFiles/main.dir/__/pico-sdk/src/rp2_common/pico_double/double_math.c.obj
 .text.__wrap_pow
                0x00000000      0x2f0 CMakeFiles/main.dir/__/pico-sdk/src/rp2_common/pico_double/double_math.c.obj
 .text.__wrap_hypot
                0x00000000      0x1a0 CMakeFiles/main.dir/__/pico-sdk/src/rp2_common/pico_double/double_math.c.obj
 .text.__wrap_cbrt
                0x00000000       0xcc CMakeFiles/main.dir/__/pico-sdk/src/rp2_common/pico_double/double_math.c.obj
 .text.__wrap_fmod
                0x00000000      0x168 CMakeFiles/main.dir/__/pico-sdk/src/rp2_common/pico_double/double_math.c.obj
 .text.__wrap_remquo
                0x00000000      0x2d0 CMakeFiles/main.dir/__/pico-sdk/src/rp2_common/pico_double/double_math.c.obj
 .text.__wrap_drem
                0x00000000       0x10 CMakeFiles/main.dir/__/pico-sdk/src/rp2_common/pico_double/double_math.c.obj
 .text.__wrap_remainder
                0x00000000       0x10 CMakeFiles/main.dir/__/pico-sdk/src/rp2_common/pico_double/double_math.c.obj
 .comment       0x00000000       0x58 CMakeFiles/main.dir/__/pico-sdk/src/rp2_common/pico_double/double_math.c.obj
 .ARM.attributes
                0x00000000       0x32 CMakeFiles/main.dir/__/pico-sdk/src/rp2_common/pico_double/double_math.c.obj
 .text          0x00000000        0x0 CMakeFiles/main.dir/__/pico-sdk/src/rp2_common/pico_double/double_v1_rom_shim.S.obj
 .data          0x00000000        0x0 CMakeFiles/main.dir/__/pico-sdk/src/rp2_common/pico_double/double_v1_rom_shim.S.obj
 .bss           0x00000000        0x0 CMakeFiles/main.dir/__/pico-sdk/src/rp2_common/pico_double/double_v1_rom_shim.S.obj
 .text.dsqrt_shim
                0x00000000      0x1a8 CMakeFiles/main.dir/__/pico-sdk/src/rp2_common/pico_double/double_v1_rom_shim.S.obj
 .text.dcordic_vec_step
                0x00000000        0xe CMakeFiles/main.dir/__/pico-sdk/src/rp2_common/pico_double/double_v1_rom_shim.S.obj
 .text.dcordic_rot_step
                0x00000000       0x76 CMakeFiles/main.dir/__/pico-sdk/src/rp2_common/pico_double/double_v1_rom_shim.S.obj
 .text.double2int_shim
                0x00000000        0xe CMakeFiles/main.dir/__/pico-sdk/src/rp2_common/pico_double/double_v1_rom_shim.S.obj
 .text.double2int64_shim
                0x00000000       0x1a CMakeFiles/main.dir/__/pico-sdk/src/rp2_common/pico_double/double_v1_rom_shim.S.obj
 .text.double2float_shim
                0x00000000       0x5c CMakeFiles/main.dir/__/pico-sdk/src/rp2_common/pico_double/double_v1_rom_shim.S.obj
 .text.x2double_shims
                0x00000000       0x90 CMakeFiles/main.dir/__/pico-sdk/src/rp2_common/pico_double/double_v1_rom_shim.S.obj
 .text.dreduce  0x00000000       0x82 CMakeFiles/main.dir/__/pico-sdk/src/rp2_common/pico_double/double_v1_rom_shim.S.obj
 .text.dtan_shim
                0x00000000       0x20 CMakeFiles/main.dir/__/pico-sdk/src/rp2_common/pico_double/double_v1_rom_shim.S.obj
 .text.dcos_shim
                0x00000000       0x10 CMakeFiles/main.dir/__/pico-sdk/src/rp2_common/pico_double/double_v1_rom_shim.S.obj
 .text.dsin_shim
                0x00000000       0x14 CMakeFiles/main.dir/__/pico-sdk/src/rp2_common/pico_double/double_v1_rom_shim.S.obj
 .text.dsincos_shim
                0x00000000       0x20 CMakeFiles/main.dir/__/pico-sdk/src/rp2_common/pico_double/double_v1_rom_shim.S.obj
 .text.dtrig_guts
                0x00000000      0x2ec CMakeFiles/main.dir/__/pico-sdk/src/rp2_common/pico_double/double_v1_rom_shim.S.obj
 .text.dexp_guts
                0x00000000      0x268 CMakeFiles/main.dir/__/pico-sdk/src/rp2_common/pico_double/double_v1_rom_shim.S.obj
 .text          0x00000000        0x0 CMakeFiles/main.dir/__/pico-sdk/src/rp2_common/pico_int64_ops/pico_int64_ops_aeabi.S.obj
 .data          0x00000000        0x0 CMakeFiles/main.dir/__/pico-sdk/src/rp2_common/pico_int64_ops/pico_int64_ops_aeabi.S.obj
 .bss           0x00000000        0x0 CMakeFiles/main.dir/__/pico-sdk/src/rp2_common/pico_int64_ops/pico_int64_ops_aeabi.S.obj
 .text          0x00000000        0x0 CMakeFiles/main.dir/__/pico-sdk/src/rp2_common/pico_float/float_aeabi.S.obj
 .data          0x00000000        0x0 CMakeFiles/main.dir/__/pico-sdk/src/rp2_common/pico_float/float_aeabi.S.obj
 .bss           0x00000000        0x0 CMakeFiles/main.dir/__/pico-sdk/src/rp2_common/pico_float/float_aeabi.S.obj
 .text.__wrap___aeabi_cfcmple
                0x00000000       0x50 CMakeFiles/main.dir/__/pico-sdk/src/rp2_common/pico_float/float_aeabi.S.obj
 .text.__wrap___aeabi_fcmpeq
                0x00000000       0x10 CMakeFiles/main.dir/__/pico-sdk/src/rp2_common/pico_float/float_aeabi.S.obj
 .text.__wrap___aeabi_fcmplt
                0x00000000        0xc CMakeFiles/main.dir/__/pico-sdk/src/rp2_common/pico_float/float_aeabi.S.obj
 .text.__wrap___aeabi_fcmple
                0x00000000       0x10 CMakeFiles/main.dir/__/pico-sdk/src/rp2_common/pico_float/float_aeabi.S.obj
 .text.__wrap___aeabi_fcmpge
                0x00000000       0x10 CMakeFiles/main.dir/__/pico-sdk/src/rp2_common/pico_float/float_aeabi.S.obj
 .text.__wrap___aeabi_fcmpgt
                0x00000000        0xa CMakeFiles/main.dir/__/pico-sdk/src/rp2_common/pico_float/float_aeabi.S.obj
 .text.__wrap___aeabi_fcmpun
                0x00000000       0x18 CMakeFiles/main.dir/__/pico-sdk/src/rp2_common/pico_float/float_aeabi.S.obj
 .text.__wrap___aeabi_ui2f
                0x00000000        0xa CMakeFiles/main.dir/__/pico-sdk/src/rp2_common/pico_float/float_aeabi.S.obj
 .text.__wrap___aeabi_f2iz
                0x00000000       0x4e CMakeFiles/main.dir/__/pico-sdk/src/rp2_common/pico_float/float_aeabi.S.obj
 .text.float2int
                0x00000000       0x14 CMakeFiles/main.dir/__/pico-sdk/src/rp2_common/pico_float/float_aeabi.S.obj
 .text.float2fix
                0x00000000       0x14 CMakeFiles/main.dir/__/pico-sdk/src/rp2_common/pico_float/float_aeabi.S.obj
 .text.float2ufix
                0x00000000        0xc CMakeFiles/main.dir/__/pico-sdk/src/rp2_common/pico_float/float_aeabi.S.obj
 .text.__wrap___aeabi_f2uiz
                0x00000000        0xc CMakeFiles/main.dir/__/pico-sdk/src/rp2_common/pico_float/float_aeabi.S.obj
 .text.fix2float
                0x00000000        0xc CMakeFiles/main.dir/__/pico-sdk/src/rp2_common/pico_float/float_aeabi.S.obj
 .text.ufix2float
                0x00000000        0xc CMakeFiles/main.dir/__/pico-sdk/src/rp2_common/pico_float/float_aeabi.S.obj
 .text.fix642float
                0x00000000       0x14 CMakeFiles/main.dir/__/pico-sdk/src/rp2_common/pico_float/float_aeabi.S.obj
 .text.ufix642float
                0x00000000       0x14 CMakeFiles/main.dir/__/pico-sdk/src/rp2_common/pico_float/float_aeabi.S.obj
 .text.__wrap___aeabi_l2f
                0x00000000       0x20 CMakeFiles/main.dir/__/pico-sdk/src/rp2_common/pico_float/float_aeabi.S.obj
 .text.__wrap___aeabi_ul2f
                0x00000000       0x20 CMakeFiles/main.dir/__/pico-sdk/src/rp2_common/pico_float/float_aeabi.S.obj
 .text.__wrap___aeabi_f2lz
                0x00000000       0x26 CMakeFiles/main.dir/__/pico-sdk/src/rp2_common/pico_float/float_aeabi.S.obj
 .text.float2int64
                0x00000000       0x14 CMakeFiles/main.dir/__/pico-sdk/src/rp2_common/pico_float/float_aeabi.S.obj
 .text.float2fix64
                0x00000000       0x14 CMakeFiles/main.dir/__/pico-sdk/src/rp2_common/pico_float/float_aeabi.S.obj
 .text.__wrap___aeabi_f2ulz
                0x00000000       0x14 CMakeFiles/main.dir/__/pico-sdk/src/rp2_common/pico_float/float_aeabi.S.obj
 .text.float2ufix64
                0x00000000       0x14 CMakeFiles/main.dir/__/pico-sdk/src/rp2_common/pico_float/float_aeabi.S.obj
 .text.__wrap_srqtf
                0x00000000       0x20 CMakeFiles/main.dir/__/pico-sdk/src/rp2_common/pico_float/float_aeabi.S.obj
 .text.__wrap_cosf
                0x00000000       0x24 CMakeFiles/main.dir/__/pico-sdk/src/rp2_common/pico_float/float_aeabi.S.obj
 .text.__wrap_sinf
                0x00000000       0x24 CMakeFiles/main.dir/__/pico-sdk/src/rp2_common/pico_float/float_aeabi.S.obj
 .text.__wrap_sincosf
                0x00000000       0x30 CMakeFiles/main.dir/__/pico-sdk/src/rp2_common/pico_float/float_aeabi.S.obj
 .text.__wrap_tanf
                0x00000000       0x4c CMakeFiles/main.dir/__/pico-sdk/src/rp2_common/pico_float/float_aeabi.S.obj
 .text.__wrap_atan2f
                0x00000000       0x14 CMakeFiles/main.dir/__/pico-sdk/src/rp2_common/pico_float/float_aeabi.S.obj
 .text.__wrap_expf
                0x00000000        0xc CMakeFiles/main.dir/__/pico-sdk/src/rp2_common/pico_float/float_aeabi.S.obj
 .text.__wrap_logf
                0x00000000        0xc CMakeFiles/main.dir/__/pico-sdk/src/rp2_common/pico_float/float_aeabi.S.obj
 .text          0x00000000        0x0 CMakeFiles/main.dir/__/pico-sdk/src/rp2_common/pico_float/float_init_rom.c.obj
 .data          0x00000000        0x0 CMakeFiles/main.dir/__/pico-sdk/src/rp2_common/pico_float/float_init_rom.c.obj
 .bss           0x00000000        0x0 CMakeFiles/main.dir/__/pico-sdk/src/rp2_common/pico_float/float_init_rom.c.obj
 .bss.sf_clz_func
                0x00000000        0x4 CMakeFiles/main.dir/__/pico-sdk/src/rp2_common/pico_float/float_init_rom.c.obj
 .text          0x00000000        0x0 CMakeFiles/main.dir/__/pico-sdk/src/rp2_common/pico_float/float_math.c.obj
 .data          0x00000000        0x0 CMakeFiles/main.dir/__/pico-sdk/src/rp2_common/pico_float/float_math.c.obj
 .bss           0x00000000        0x0 CMakeFiles/main.dir/__/pico-sdk/src/rp2_common/pico_float/float_math.c.obj
 .text.fpow_int2
                0x00000000       0x54 CMakeFiles/main.dir/__/pico-sdk/src/rp2_common/pico_float/float_math.c.obj
 .text.fpow_0   0x00000000      0x17c CMakeFiles/main.dir/__/pico-sdk/src/rp2_common/pico_float/float_math.c.obj
 .text.fpowint_0
                0x00000000      0x16c CMakeFiles/main.dir/__/pico-sdk/src/rp2_common/pico_float/float_math.c.obj
 .text.__wrap_ldexpf
                0x00000000       0x30 CMakeFiles/main.dir/__/pico-sdk/src/rp2_common/pico_float/float_math.c.obj
 .text.__wrap_copysignf
                0x00000000        0xc CMakeFiles/main.dir/__/pico-sdk/src/rp2_common/pico_float/float_math.c.obj
 .text.__wrap_truncf
                0x00000000       0x20 CMakeFiles/main.dir/__/pico-sdk/src/rp2_common/pico_float/float_math.c.obj
 .text.__wrap_roundf
                0x00000000       0x3c CMakeFiles/main.dir/__/pico-sdk/src/rp2_common/pico_float/float_math.c.obj
 .text.__wrap_floorf
                0x00000000       0x40 CMakeFiles/main.dir/__/pico-sdk/src/rp2_common/pico_float/float_math.c.obj
 .text.__wrap_ceilf
                0x00000000       0x40 CMakeFiles/main.dir/__/pico-sdk/src/rp2_common/pico_float/float_math.c.obj
 .text.__wrap_asinf
                0x00000000       0x40 CMakeFiles/main.dir/__/pico-sdk/src/rp2_common/pico_float/float_math.c.obj
 .text.__wrap_acosf
                0x00000000       0x40 CMakeFiles/main.dir/__/pico-sdk/src/rp2_common/pico_float/float_math.c.obj
 .text.__wrap_atanf
                0x00000000       0x2c CMakeFiles/main.dir/__/pico-sdk/src/rp2_common/pico_float/float_math.c.obj
 .text.__wrap_sinhf
                0x00000000       0x3c CMakeFiles/main.dir/__/pico-sdk/src/rp2_common/pico_float/float_math.c.obj
 .text.__wrap_coshf
                0x00000000       0x3c CMakeFiles/main.dir/__/pico-sdk/src/rp2_common/pico_float/float_math.c.obj
 .text.__wrap_tanhf
                0x00000000       0x4c CMakeFiles/main.dir/__/pico-sdk/src/rp2_common/pico_float/float_math.c.obj
 .text.__wrap_asinhf
                0x00000000       0xa8 CMakeFiles/main.dir/__/pico-sdk/src/rp2_common/pico_float/float_math.c.obj
 .text.__wrap_acoshf
                0x00000000       0x70 CMakeFiles/main.dir/__/pico-sdk/src/rp2_common/pico_float/float_math.c.obj
 .text.__wrap_atanhf
                0x00000000       0x44 CMakeFiles/main.dir/__/pico-sdk/src/rp2_common/pico_float/float_math.c.obj
 .text.__wrap_exp2f
                0x00000000       0x20 CMakeFiles/main.dir/__/pico-sdk/src/rp2_common/pico_float/float_math.c.obj
 .text.__wrap_log2f
                0x00000000       0x14 CMakeFiles/main.dir/__/pico-sdk/src/rp2_common/pico_float/float_math.c.obj
 .text.__wrap_exp10f
                0x00000000       0x20 CMakeFiles/main.dir/__/pico-sdk/src/rp2_common/pico_float/float_math.c.obj
 .text.__wrap_log10f
                0x00000000       0x14 CMakeFiles/main.dir/__/pico-sdk/src/rp2_common/pico_float/float_math.c.obj
 .text.__wrap_expm1f
                0x00000000       0x1c CMakeFiles/main.dir/__/pico-sdk/src/rp2_common/pico_float/float_math.c.obj
 .text.__wrap_log1pf
                0x00000000       0x1c CMakeFiles/main.dir/__/pico-sdk/src/rp2_common/pico_float/float_math.c.obj
 .text.__wrap_fmaf
                0x00000000       0x3c CMakeFiles/main.dir/__/pico-sdk/src/rp2_common/pico_float/float_math.c.obj
 .text.__wrap_powintf
                0x00000000       0x8c CMakeFiles/main.dir/__/pico-sdk/src/rp2_common/pico_float/float_math.c.obj
 .text.__wrap_powf
                0x00000000      0x188 CMakeFiles/main.dir/__/pico-sdk/src/rp2_common/pico_float/float_math.c.obj
 .text.__wrap_hypotf
                0x00000000      0x100 CMakeFiles/main.dir/__/pico-sdk/src/rp2_common/pico_float/float_math.c.obj
 .text.__wrap_cbrtf
                0x00000000       0xa0 CMakeFiles/main.dir/__/pico-sdk/src/rp2_common/pico_float/float_math.c.obj
 .text.__wrap_fmodf
                0x00000000       0xb0 CMakeFiles/main.dir/__/pico-sdk/src/rp2_common/pico_float/float_math.c.obj
 .text.__wrap_remquof
                0x00000000      0x140 CMakeFiles/main.dir/__/pico-sdk/src/rp2_common/pico_float/float_math.c.obj
 .text.__wrap_dremf
                0x00000000        0xc CMakeFiles/main.dir/__/pico-sdk/src/rp2_common/pico_float/float_math.c.obj
 .text.__wrap_remainderf
                0x00000000        0xc CMakeFiles/main.dir/__/pico-sdk/src/rp2_common/pico_float/float_math.c.obj
 .comment       0x00000000       0x58 CMakeFiles/main.dir/__/pico-sdk/src/rp2_common/pico_float/float_math.c.obj
 .ARM.attributes
                0x00000000       0x32 CMakeFiles/main.dir/__/pico-sdk/src/rp2_common/pico_float/float_math.c.obj
 .text          0x00000000        0x0 CMakeFiles/main.dir/__/pico-sdk/src/rp2_common/pico_float/float_v1_rom_shim.S.obj
 .data          0x00000000        0x0 CMakeFiles/main.dir/__/pico-sdk/src/rp2_common/pico_float/float_v1_rom_shim.S.obj
 .bss           0x00000000        0x0 CMakeFiles/main.dir/__/pico-sdk/src/rp2_common/pico_float/float_v1_rom_shim.S.obj
 .text.642float_shims
                0x00000000       0x44 CMakeFiles/main.dir/__/pico-sdk/src/rp2_common/pico_float/float_v1_rom_shim.S.obj
 .text.fatan2_shim
                0x00000000       0x88 CMakeFiles/main.dir/__/pico-sdk/src/rp2_common/pico_float/float_v1_rom_shim.S.obj
 .text.float232_shims
                0x00000000       0x18 CMakeFiles/main.dir/__/pico-sdk/src/rp2_common/pico_float/float_v1_rom_shim.S.obj
 .text.float264_shims
                0x00000000       0x4c CMakeFiles/main.dir/__/pico-sdk/src/rp2_common/pico_float/float_v1_rom_shim.S.obj
 .text.d2fix_a_float
                0x00000000       0x5c CMakeFiles/main.dir/__/pico-sdk/src/rp2_common/pico_float/float_v1_rom_shim.S.obj
 .text          0x00000000        0x0 CMakeFiles/main.dir/__/pico-sdk/src/rp2_common/pico_malloc/pico_malloc.c.obj
 .data          0x00000000        0x0 CMakeFiles/main.dir/__/pico-sdk/src/rp2_common/pico_malloc/pico_malloc.c.obj
 .bss           0x00000000        0x0 CMakeFiles/main.dir/__/pico-sdk/src/rp2_common/pico_malloc/pico_malloc.c.obj
 .text.__wrap_malloc
                0x00000000       0x24 CMakeFiles/main.dir/__/pico-sdk/src/rp2_common/pico_malloc/pico_malloc.c.obj
 .text.__wrap_calloc
                0x00000000       0x24 CMakeFiles/main.dir/__/pico-sdk/src/rp2_common/pico_malloc/pico_malloc.c.obj
 .text.__wrap_free
                0x00000000        0x8 CMakeFiles/main.dir/__/pico-sdk/src/rp2_common/pico_malloc/pico_malloc.c.obj
 .rodata.__wrap_malloc.str1.4
                0x00000000        0xe CMakeFiles/main.dir/__/pico-sdk/src/rp2_common/pico_malloc/pico_malloc.c.obj
 .comment       0x00000000       0x58 CMakeFiles/main.dir/__/pico-sdk/src/rp2_common/pico_malloc/pico_malloc.c.obj
 .ARM.attributes
                0x00000000       0x32 CMakeFiles/main.dir/__/pico-sdk/src/rp2_common/pico_malloc/pico_malloc.c.obj
 .data          0x00000000        0x0 CMakeFiles/main.dir/__/pico-sdk/src/rp2_common/pico_mem_ops/mem_ops_aeabi.S.obj
 .bss           0x00000000        0x0 CMakeFiles/main.dir/__/pico-sdk/src/rp2_common/pico_mem_ops/mem_ops_aeabi.S.obj
 .text.aeabi_memset_memcpy
                0x00000000       0x24 CMakeFiles/main.dir/__/pico-sdk/src/rp2_common/pico_mem_ops/mem_ops_aeabi.S.obj
 .text          0x00000000        0x0 CMakeFiles/main.dir/__/pico-sdk/src/rp2_common/pico_standard_link/crt0.S.obj
 .data          0x00000000        0x0 CMakeFiles/main.dir/__/pico-sdk/src/rp2_common/pico_standard_link/crt0.S.obj
 .bss           0x00000000        0x0 CMakeFiles/main.dir/__/pico-sdk/src/rp2_common/pico_standard_link/crt0.S.obj
 .text          0x00000000        0x0 CMakeFiles/main.dir/__/pico-sdk/src/rp2_common/pico_standard_link/new_delete.cpp.obj
 .data          0x00000000        0x0 CMakeFiles/main.dir/__/pico-sdk/src/rp2_common/pico_standard_link/new_delete.cpp.obj
 .bss           0x00000000        0x0 CMakeFiles/main.dir/__/pico-sdk/src/rp2_common/pico_standard_link/new_delete.cpp.obj
 .comment       0x00000000       0x58 CMakeFiles/main.dir/__/pico-sdk/src/rp2_common/pico_standard_link/new_delete.cpp.obj
 .ARM.attributes
                0x00000000       0x32 CMakeFiles/main.dir/__/pico-sdk/src/rp2_common/pico_standard_link/new_delete.cpp.obj
 .text          0x00000000        0x0 CMakeFiles/main.dir/__/pico-sdk/src/rp2_common/pico_standard_link/binary_info.c.obj
 .data          0x00000000        0x0 CMakeFiles/main.dir/__/pico-sdk/src/rp2_common/pico_standard_link/binary_info.c.obj
 .bss           0x00000000        0x0 CMakeFiles/main.dir/__/pico-sdk/src/rp2_common/pico_standard_link/binary_info.c.obj
 .text          0x00000000        0x0 CMakeFiles/main.dir/__/pico-sdk/src/rp2_common/pico_stdio/stdio.c.obj
 .data          0x00000000        0x0 CMakeFiles/main.dir/__/pico-sdk/src/rp2_common/pico_stdio/stdio.c.obj
 .bss           0x00000000        0x0 CMakeFiles/main.dir/__/pico-sdk/src/rp2_common/pico_stdio/stdio.c.obj
 .text.stdio_out_chars_no_crlf
                0x00000000       0x10 CMakeFiles/main.dir/__/pico-sdk/src/rp2_common/pico_stdio/stdio.c.obj
 .text.stdout_serialize_begin
                0x00000000       0x30 CMakeFiles/main.dir/__/pico-sdk/src/rp2_common/pico_stdio/stdio.c.obj
 .text.stdout_serialize_end
                0x00000000       0x10 CMakeFiles/main.dir/__/pico-sdk/src/rp2_common/pico_stdio/stdio.c.obj
 .text.putchar_raw
                0x00000000       0xa0 CMakeFiles/main.dir/__/pico-sdk/src/rp2_common/pico_stdio/stdio.c.obj
 .text.puts_raw
                0x00000000       0xe8 CMakeFiles/main.dir/__/pico-sdk/src/rp2_common/pico_stdio/stdio.c.obj
 .text._read    0x00000000       0x98 CMakeFiles/main.dir/__/pico-sdk/src/rp2_common/pico_stdio/stdio.c.obj
 .text._write   0x00000000       0xb0 CMakeFiles/main.dir/__/pico-sdk/src/rp2_common/pico_stdio/stdio.c.obj
 .text.stdio_flush
                0x00000000       0x28 CMakeFiles/main.dir/__/pico-sdk/src/rp2_common/pico_stdio/stdio.c.obj
 .text.__wrap_getchar
                0x00000000       0x78 CMakeFiles/main.dir/__/pico-sdk/src/rp2_common/pico_stdio/stdio.c.obj
 .text.stdio_filter_driver
                0x00000000        0xc CMakeFiles/main.dir/__/pico-sdk/src/rp2_common/pico_stdio/stdio.c.obj
 .text          0x00000000        0x0 CMakeFiles/main.dir/__/pico-sdk/src/rp2_common/pico_stdio_usb/reset_interface.c.obj
 .data          0x00000000        0x0 CMakeFiles/main.dir/__/pico-sdk/src/rp2_common/pico_stdio_usb/reset_interface.c.obj
 .bss           0x00000000        0x0 CMakeFiles/main.dir/__/pico-sdk/src/rp2_common/pico_stdio_usb/reset_interface.c.obj
 .text          0x00000000        0x0 CMakeFiles/main.dir/__/pico-sdk/src/rp2_common/pico_stdio_usb/stdio_usb.c.obj
 .data          0x00000000        0x0 CMakeFiles/main.dir/__/pico-sdk/src/rp2_common/pico_stdio_usb/stdio_usb.c.obj
 .bss           0x00000000        0x0 CMakeFiles/main.dir/__/pico-sdk/src/rp2_common/pico_stdio_usb/stdio_usb.c.obj
 .text.stdio_usb_connected
                0x00000000        0xc CMakeFiles/main.dir/__/pico-sdk/src/rp2_common/pico_stdio_usb/stdio_usb.c.obj
 .text          0x00000000        0x0 CMakeFiles/main.dir/__/pico-sdk/src/rp2_common/pico_stdio_usb/stdio_usb_descriptors.c.obj
 .data          0x00000000        0x0 CMakeFiles/main.dir/__/pico-sdk/src/rp2_common/pico_stdio_usb/stdio_usb_descriptors.c.obj
 .bss           0x00000000        0x0 CMakeFiles/main.dir/__/pico-sdk/src/rp2_common/pico_stdio_usb/stdio_usb_descriptors.c.obj
 .text          0x00000000        0x0 CMakeFiles/main.dir/__/pico-sdk/lib/tinyusb/src/portable/raspberrypi/rp2040/dcd_rp2040.c.obj
 .data          0x00000000        0x0 CMakeFiles/main.dir/__/pico-sdk/lib/tinyusb/src/portable/raspberrypi/rp2040/dcd_rp2040.c.obj
 .bss           0x00000000        0x0 CMakeFiles/main.dir/__/pico-sdk/lib/tinyusb/src/portable/raspberrypi/rp2040/dcd_rp2040.c.obj
 .text.dcd_int_disable
                0x00000000        0xc CMakeFiles/main.dir/__/pico-sdk/lib/tinyusb/src/portable/raspberrypi/rp2040/dcd_rp2040.c.obj
 .text.dcd_remote_wakeup
                0x00000000       0x10 CMakeFiles/main.dir/__/pico-sdk/lib/tinyusb/src/portable/raspberrypi/rp2040/dcd_rp2040.c.obj
 .text.dcd_disconnect
                0x00000000       0x10 CMakeFiles/main.dir/__/pico-sdk/lib/tinyusb/src/portable/raspberrypi/rp2040/dcd_rp2040.c.obj
 .text.dcd_edpt_close
                0x00000000        0x4 CMakeFiles/main.dir/__/pico-sdk/lib/tinyusb/src/portable/raspberrypi/rp2040/dcd_rp2040.c.obj
 .text.dcd_int_handler
                0x00000000      0x21c CMakeFiles/main.dir/__/pico-sdk/lib/tinyusb/src/portable/raspberrypi/rp2040/dcd_rp2040.c.obj
 .text          0x00000000        0x0 CMakeFiles/main.dir/__/pico-sdk/lib/tinyusb/src/portable/raspberrypi/rp2040/rp2040_usb.c.obj
 .data          0x00000000        0x0 CMakeFiles/main.dir/__/pico-sdk/lib/tinyusb/src/portable/raspberrypi/rp2040/rp2040_usb.c.obj
 .bss           0x00000000        0x0 CMakeFiles/main.dir/__/pico-sdk/lib/tinyusb/src/portable/raspberrypi/rp2040/rp2040_usb.c.obj
 .text          0x00000000        0x0 CMakeFiles/main.dir/__/pico-sdk/lib/tinyusb/src/device/usbd.c.obj
 .data          0x00000000        0x0 CMakeFiles/main.dir/__/pico-sdk/lib/tinyusb/src/device/usbd.c.obj
 .bss           0x00000000        0x0 CMakeFiles/main.dir/__/pico-sdk/lib/tinyusb/src/device/usbd.c.obj
 .text.tud_speed_get
                0x00000000        0xc CMakeFiles/main.dir/__/pico-sdk/lib/tinyusb/src/device/usbd.c.obj
 .text.tud_connected
                0x00000000       0x10 CMakeFiles/main.dir/__/pico-sdk/lib/tinyusb/src/device/usbd.c.obj
 .text.tud_remote_wakeup
                0x00000000       0x24 CMakeFiles/main.dir/__/pico-sdk/lib/tinyusb/src/device/usbd.c.obj
 .text.tud_disconnect
                0x00000000       0x18 CMakeFiles/main.dir/__/pico-sdk/lib/tinyusb/src/device/usbd.c.obj
 .text.tud_connect
                0x00000000       0x18 CMakeFiles/main.dir/__/pico-sdk/lib/tinyusb/src/device/usbd.c.obj
 .text.tud_task_event_ready
                0x00000000       0x20 CMakeFiles/main.dir/__/pico-sdk/lib/tinyusb/src/device/usbd.c.obj
 .text.dcd_event_handler
                0x00000000      0x12c CMakeFiles/main.dir/__/pico-sdk/lib/tinyusb/src/device/usbd.c.obj
 .text.usbd_defer_func
                0x00000000       0x4c CMakeFiles/main.dir/__/pico-sdk/lib/tinyusb/src/device/usbd.c.obj
 .text.usbd_edpt_xfer_fifo
                0x00000000       0x48 CMakeFiles/main.dir/__/pico-sdk/lib/tinyusb/src/device/usbd.c.obj
 .text.usbd_edpt_busy
                0x00000000       0x1c CMakeFiles/main.dir/__/pico-sdk/lib/tinyusb/src/device/usbd.c.obj
 .text.usbd_edpt_stall
                0x00000000       0x34 CMakeFiles/main.dir/__/pico-sdk/lib/tinyusb/src/device/usbd.c.obj
 .text.usbd_edpt_clear_stall
                0x00000000       0x34 CMakeFiles/main.dir/__/pico-sdk/lib/tinyusb/src/device/usbd.c.obj
 .text.usbd_edpt_stalled
                0x00000000       0x1c CMakeFiles/main.dir/__/pico-sdk/lib/tinyusb/src/device/usbd.c.obj
 .text.usbd_edpt_close
                0x00000000       0x40 CMakeFiles/main.dir/__/pico-sdk/lib/tinyusb/src/device/usbd.c.obj
 .text          0x00000000        0x0 CMakeFiles/main.dir/__/pico-sdk/lib/tinyusb/src/device/usbd_control.c.obj
 .data          0x00000000        0x0 CMakeFiles/main.dir/__/pico-sdk/lib/tinyusb/src/device/usbd_control.c.obj
 .bss           0x00000000        0x0 CMakeFiles/main.dir/__/pico-sdk/lib/tinyusb/src/device/usbd_control.c.obj
 .text          0x00000000        0x0 CMakeFiles/main.dir/__/pico-sdk/lib/tinyusb/src/class/audio/audio_device.c.obj
 .data          0x00000000        0x0 CMakeFiles/main.dir/__/pico-sdk/lib/tinyusb/src/class/audio/audio_device.c.obj
 .bss           0x00000000        0x0 CMakeFiles/main.dir/__/pico-sdk/lib/tinyusb/src/class/audio/audio_device.c.obj
 .comment       0x00000000       0x58 CMakeFiles/main.dir/__/pico-sdk/lib/tinyusb/src/class/audio/audio_device.c.obj
 .ARM.attributes
                0x00000000       0x32 CMakeFiles/main.dir/__/pico-sdk/lib/tinyusb/src/class/audio/audio_device.c.obj
 .text          0x00000000        0x0 CMakeFiles/main.dir/__/pico-sdk/lib/tinyusb/src/class/cdc/cdc_device.c.obj
 .data          0x00000000        0x0 CMakeFiles/main.dir/__/pico-sdk/lib/tinyusb/src/class/cdc/cdc_device.c.obj
 .bss           0x00000000        0x0 CMakeFiles/main.dir/__/pico-sdk/lib/tinyusb/src/class/cdc/cdc_device.c.obj
 .text.tud_cdc_n_get_line_state
                0x00000000       0x14 CMakeFiles/main.dir/__/pico-sdk/lib/tinyusb/src/class/cdc/cdc_device.c.obj
 .text.tud_cdc_n_get_line_coding
                0x00000000       0x20 CMakeFiles/main.dir/__/pico-sdk/lib/tinyusb/src/class/cdc/cdc_device.c.obj
 .text.tud_cdc_n_set_wanted_char
                0x00000000       0x14 CMakeFiles/main.dir/__/pico-sdk/lib/tinyusb/src/class/cdc/cdc_device.c.obj
 .text.tud_cdc_n_peek
                0x00000000       0x1c CMakeFiles/main.dir/__/pico-sdk/lib/tinyusb/src/class/cdc/cdc_device.c.obj
 .text.tud_cdc_n_read_flush
                0x00000000       0x5c CMakeFiles/main.dir/__/pico-sdk/lib/tinyusb/src/class/cdc/cdc_device.c.obj
 .text.tud_cdc_n_write_clear
                0x00000000       0x1c CMakeFiles/main.dir/__/pico-sdk/lib/tinyusb/src/class/cdc/cdc_device.c.obj
 .text          0x00000000        0x0 CMakeFiles/main.dir/__/pico-sdk/lib/tinyusb/src/class/dfu/dfu_device.c.obj
 .data          0x00000000        0x0 CMakeFiles/main.dir/__/pico-sdk/lib/tinyusb/src/class/dfu/dfu_device.c.obj
 .bss           0x00000000        0x0 CMakeFiles/main.dir/__/pico-sdk/lib/tinyusb/src/class/dfu/dfu_device.c.obj
 .comment       0x00000000       0x58 CMakeFiles/main.dir/__/pico-sdk/lib/tinyusb/src/class/dfu/dfu_device.c.obj
 .ARM.attributes
                0x00000000       0x32 CMakeFiles/main.dir/__/pico-sdk/lib/tinyusb/src/class/dfu/dfu_device.c.obj
 .text          0x00000000        0x0 CMakeFiles/main.dir/__/pico-sdk/lib/tinyusb/src/class/dfu/dfu_rt_device.c.obj
 .data          0x00000000        0x0 CMakeFiles/main.dir/__/pico-sdk/lib/tinyusb/src/class/dfu/dfu_rt_device.c.obj
 .bss           0x00000000        0x0 CMakeFiles/main.dir/__/pico-sdk/lib/tinyusb/src/class/dfu/dfu_rt_device.c.obj
 .comment       0x00000000       0x58 CMakeFiles/main.dir/__/pico-sdk/lib/tinyusb/src/class/dfu/dfu_rt_device.c.obj
 .ARM.attributes
                0x00000000       0x32 CMakeFiles/main.dir/__/pico-sdk/lib/tinyusb/src/class/dfu/dfu_rt_device.c.obj
 .text          0x00000000        0x0 CMakeFiles/main.dir/__/pico-sdk/lib/tinyusb/src/class/hid/hid_device.c.obj
 .data          0x00000000        0x0 CMakeFiles/main.dir/__/pico-sdk/lib/tinyusb/src/class/hid/hid_device.c.obj
 .bss           0x00000000        0x0 CMakeFiles/main.dir/__/pico-sdk/lib/tinyusb/src/class/hid/hid_device.c.obj
 .comment       0x00000000       0x58 CMakeFiles/main.dir/__/pico-sdk/lib/tinyusb/src/class/hid/hid_device.c.obj
 .ARM.attributes
                0x00000000       0x32 CMakeFiles/main.dir/__/pico-sdk/lib/tinyusb/src/class/hid/hid_device.c.obj
 .text          0x00000000        0x0 CMakeFiles/main.dir/__/pico-sdk/lib/tinyusb/src/class/midi/midi_device.c.obj
 .data          0x00000000        0x0 CMakeFiles/main.dir/__/pico-sdk/lib/tinyusb/src/class/midi/midi_device.c.obj
 .bss           0x00000000        0x0 CMakeFiles/main.dir/__/pico-sdk/lib/tinyusb/src/class/midi/midi_device.c.obj
 .comment       0x00000000       0x58 CMakeFiles/main.dir/__/pico-sdk/lib/tinyusb/src/class/midi/midi_device.c.obj
 .ARM.attributes
                0x00000000       0x32 CMakeFiles/main.dir/__/pico-sdk/lib/tinyusb/src/class/midi/midi_device.c.obj
 .text          0x00000000        0x0 CMakeFiles/main.dir/__/pico-sdk/lib/tinyusb/src/class/msc/msc_device.c.obj
 .data          0x00000000        0x0 CMakeFiles/main.dir/__/pico-sdk/lib/tinyusb/src/class/msc/msc_device.c.obj
 .bss           0x00000000        0x0 CMakeFiles/main.dir/__/pico-sdk/lib/tinyusb/src/class/msc/msc_device.c.obj
 .comment       0x00000000       0x58 CMakeFiles/main.dir/__/pico-sdk/lib/tinyusb/src/class/msc/msc_device.c.obj
 .ARM.attributes
                0x00000000       0x32 CMakeFiles/main.dir/__/pico-sdk/lib/tinyusb/src/class/msc/msc_device.c.obj
 .text          0x00000000        0x0 CMakeFiles/main.dir/__/pico-sdk/lib/tinyusb/src/class/net/ecm_rndis_device.c.obj
 .data          0x00000000        0x0 CMakeFiles/main.dir/__/pico-sdk/lib/tinyusb/src/class/net/ecm_rndis_device.c.obj
 .bss           0x00000000        0x0 CMakeFiles/main.dir/__/pico-sdk/lib/tinyusb/src/class/net/ecm_rndis_device.c.obj
 .comment       0x00000000       0x58 CMakeFiles/main.dir/__/pico-sdk/lib/tinyusb/src/class/net/ecm_rndis_device.c.obj
 .ARM.attributes
                0x00000000       0x32 CMakeFiles/main.dir/__/pico-sdk/lib/tinyusb/src/class/net/ecm_rndis_device.c.obj
 .text          0x00000000        0x0 CMakeFiles/main.dir/__/pico-sdk/lib/tinyusb/src/class/net/ncm_device.c.obj
 .data          0x00000000        0x0 CMakeFiles/main.dir/__/pico-sdk/lib/tinyusb/src/class/net/ncm_device.c.obj
 .bss           0x00000000        0x0 CMakeFiles/main.dir/__/pico-sdk/lib/tinyusb/src/class/net/ncm_device.c.obj
 .comment       0x00000000       0x58 CMakeFiles/main.dir/__/pico-sdk/lib/tinyusb/src/class/net/ncm_device.c.obj
 .ARM.attributes
                0x00000000       0x32 CMakeFiles/main.dir/__/pico-sdk/lib/tinyusb/src/class/net/ncm_device.c.obj
 .text          0x00000000        0x0 CMakeFiles/main.dir/__/pico-sdk/lib/tinyusb/src/class/usbtmc/usbtmc_device.c.obj
 .data          0x00000000        0x0 CMakeFiles/main.dir/__/pico-sdk/lib/tinyusb/src/class/usbtmc/usbtmc_device.c.obj
 .bss           0x00000000        0x0 CMakeFiles/main.dir/__/pico-sdk/lib/tinyusb/src/class/usbtmc/usbtmc_device.c.obj
 .comment       0x00000000       0x58 CMakeFiles/main.dir/__/pico-sdk/lib/tinyusb/src/class/usbtmc/usbtmc_device.c.obj
 .ARM.attributes
                0x00000000       0x32 CMakeFiles/main.dir/__/pico-sdk/lib/tinyusb/src/class/usbtmc/usbtmc_device.c.obj
 .text          0x00000000        0x0 CMakeFiles/main.dir/__/pico-sdk/lib/tinyusb/src/class/vendor/vendor_device.c.obj
 .data          0x00000000        0x0 CMakeFiles/main.dir/__/pico-sdk/lib/tinyusb/src/class/vendor/vendor_device.c.obj
 .bss           0x00000000        0x0 CMakeFiles/main.dir/__/pico-sdk/lib/tinyusb/src/class/vendor/vendor_device.c.obj
 .comment       0x00000000       0x58 CMakeFiles/main.dir/__/pico-sdk/lib/tinyusb/src/class/vendor/vendor_device.c.obj
 .ARM.attributes
                0x00000000       0x32 CMakeFiles/main.dir/__/pico-sdk/lib/tinyusb/src/class/vendor/vendor_device.c.obj
 .text          0x00000000        0x0 CMakeFiles/main.dir/__/pico-sdk/lib/tinyusb/src/class/video/video_device.c.obj
 .data          0x00000000        0x0 CMakeFiles/main.dir/__/pico-sdk/lib/tinyusb/src/class/video/video_device.c.obj
 .bss           0x00000000        0x0 CMakeFiles/main.dir/__/pico-sdk/lib/tinyusb/src/class/video/video_device.c.obj
 .comment       0x00000000       0x58 CMakeFiles/main.dir/__/pico-sdk/lib/tinyusb/src/class/video/video_device.c.obj
 .ARM.attributes
                0x00000000       0x32 CMakeFiles/main.dir/__/pico-sdk/lib/tinyusb/src/class/video/video_device.c.obj
 .text          0x00000000        0x0 CMakeFiles/main.dir/__/pico-sdk/lib/tinyusb/src/tusb.c.obj
 .data          0x00000000        0x0 CMakeFiles/main.dir/__/pico-sdk/lib/tinyusb/src/tusb.c.obj
 .bss           0x00000000        0x0 CMakeFiles/main.dir/__/pico-sdk/lib/tinyusb/src/tusb.c.obj
 .text.tu_desc_get_interface_total_len
                0x00000000       0x44 CMakeFiles/main.dir/__/pico-sdk/lib/tinyusb/src/tusb.c.obj
 .text          0x00000000        0x0 CMakeFiles/main.dir/__/pico-sdk/lib/tinyusb/src/common/tusb_fifo.c.obj
 .data          0x00000000        0x0 CMakeFiles/main.dir/__/pico-sdk/lib/tinyusb/src/common/tusb_fifo.c.obj
 .bss           0x00000000        0x0 CMakeFiles/main.dir/__/pico-sdk/lib/tinyusb/src/common/tusb_fifo.c.obj
 .text.tu_fifo_full
                0x00000000       0x24 CMakeFiles/main.dir/__/pico-sdk/lib/tinyusb/src/common/tusb_fifo.c.obj
 .text.tu_fifo_overflowed
                0x00000000       0x20 CMakeFiles/main.dir/__/pico-sdk/lib/tinyusb/src/common/tusb_fifo.c.obj
 .text.tu_fifo_correct_read_pointer
                0x00000000       0x40 CMakeFiles/main.dir/__/pico-sdk/lib/tinyusb/src/common/tusb_fifo.c.obj
 .text.tu_fifo_read_n_const_addr_full_words
                0x00000000      0x22c CMakeFiles/main.dir/__/pico-sdk/lib/tinyusb/src/common/tusb_fifo.c.obj
 .text.tu_fifo_peek
                0x00000000       0x7c CMakeFiles/main.dir/__/pico-sdk/lib/tinyusb/src/common/tusb_fifo.c.obj
 .text.tu_fifo_peek_n
                0x00000000       0xdc CMakeFiles/main.dir/__/pico-sdk/lib/tinyusb/src/common/tusb_fifo.c.obj
 .text.tu_fifo_write_n_const_addr_full_words
                0x00000000      0x1ec CMakeFiles/main.dir/__/pico-sdk/lib/tinyusb/src/common/tusb_fifo.c.obj
 .text.tu_fifo_advance_write_pointer
                0x00000000       0x1c CMakeFiles/main.dir/__/pico-sdk/lib/tinyusb/src/common/tusb_fifo.c.obj
 .text.tu_fifo_advance_read_pointer
                0x00000000       0x1c CMakeFiles/main.dir/__/pico-sdk/lib/tinyusb/src/common/tusb_fifo.c.obj
 .text.tu_fifo_get_read_info
                0x00000000       0xa4 CMakeFiles/main.dir/__/pico-sdk/lib/tinyusb/src/common/tusb_fifo.c.obj
 .text.tu_fifo_get_write_info
                0x00000000       0x64 CMakeFiles/main.dir/__/pico-sdk/lib/tinyusb/src/common/tusb_fifo.c.obj
 .text          0x00000000        0x0 CMakeFiles/main.dir/__/pico-sdk/src/rp2_common/pico_fix/rp2040_usb_device_enumeration/rp2040_usb_device_enumeration.c.obj
 .data          0x00000000        0x0 CMakeFiles/main.dir/__/pico-sdk/src/rp2_common/pico_fix/rp2040_usb_device_enumeration/rp2040_usb_device_enumeration.c.obj
 .bss           0x00000000        0x0 CMakeFiles/main.dir/__/pico-sdk/src/rp2_common/pico_fix/rp2040_usb_device_enumeration/rp2040_usb_device_enumeration.c.obj
 .text.hw_enumeration_fix_force_ls_j_done
                0x00000000       0x48 CMakeFiles/main.dir/__/pico-sdk/src/rp2_common/pico_fix/rp2040_usb_device_enumeration/rp2040_usb_device_enumeration.c.obj
 .text.hw_enumeration_fix_force_ls_j
                0x00000000      0x10c CMakeFiles/main.dir/__/pico-sdk/src/rp2_common/pico_fix/rp2040_usb_device_enumeration/rp2040_usb_device_enumeration.c.obj
 .text.hw_enumeration_fix_wait_se0_callback
                0x00000000       0x24 CMakeFiles/main.dir/__/pico-sdk/src/rp2_common/pico_fix/rp2040_usb_device_enumeration/rp2040_usb_device_enumeration.c.obj
 .text.rp2040_usb_device_enumeration_fix
                0x00000000       0x68 CMakeFiles/main.dir/__/pico-sdk/src/rp2_common/pico_fix/rp2040_usb_device_enumeration/rp2040_usb_device_enumeration.c.obj
 .bss.gpio_ctrl_prev
                0x00000000        0x4 CMakeFiles/main.dir/__/pico-sdk/src/rp2_common/pico_fix/rp2040_usb_device_enumeration/rp2040_usb_device_enumeration.c.obj
 .bss.pad_ctrl_prev
                0x00000000        0x4 CMakeFiles/main.dir/__/pico-sdk/src/rp2_common/pico_fix/rp2040_usb_device_enumeration/rp2040_usb_device_enumeration.c.obj
 .rodata.hw_enumeration_fix_force_ls_j.str1.4
                0x00000000       0x22 CMakeFiles/main.dir/__/pico-sdk/src/rp2_common/pico_fix/rp2040_usb_device_enumeration/rp2040_usb_device_enumeration.c.obj
 .comment       0x00000000       0x58 CMakeFiles/main.dir/__/pico-sdk/src/rp2_common/pico_fix/rp2040_usb_device_enumeration/rp2040_usb_device_enumeration.c.obj
 .ARM.attributes
                0x00000000       0x32 CMakeFiles/main.dir/__/pico-sdk/src/rp2_common/pico_fix/rp2040_usb_device_enumeration/rp2040_usb_device_enumeration.c.obj
 .text          0x00000000        0x0 CMakeFiles/main.dir/__/pico-sdk/src/rp2_common/pico_unique_id/unique_id.c.obj
 .data          0x00000000        0x0 CMakeFiles/main.dir/__/pico-sdk/src/rp2_common/pico_unique_id/unique_id.c.obj
 .bss           0x00000000        0x0 CMakeFiles/main.dir/__/pico-sdk/src/rp2_common/pico_unique_id/unique_id.c.obj
 .text.pico_get_unique_board_id
                0x00000000       0x10 CMakeFiles/main.dir/__/pico-sdk/src/rp2_common/pico_unique_id/unique_id.c.obj
 .text          0x00000000        0x0 CMakeFiles/main.dir/__/pico-sdk/src/rp2_common/hardware_flash/flash.c.obj
 .data          0x00000000        0x0 CMakeFiles/main.dir/__/pico-sdk/src/rp2_common/hardware_flash/flash.c.obj
 .bss           0x00000000        0x0 CMakeFiles/main.dir/__/pico-sdk/src/rp2_common/hardware_flash/flash.c.obj
 .text          0x00000000        0x0 CMakeFiles/main.dir/__/pico-sdk/src/rp2_common/hardware_spi/spi.c.obj
 .data          0x00000000        0x0 CMakeFiles/main.dir/__/pico-sdk/src/rp2_common/hardware_spi/spi.c.obj
 .bss           0x00000000        0x0 CMakeFiles/main.dir/__/pico-sdk/src/rp2_common/hardware_spi/spi.c.obj
 .text.spi_deinit
                0x00000000       0x3c CMakeFiles/main.dir/__/pico-sdk/src/rp2_common/hardware_spi/spi.c.obj
 .text.spi_set_baudrate
                0x00000000       0x94 CMakeFiles/main.dir/__/pico-sdk/src/rp2_common/hardware_spi/spi.c.obj
 .text.spi_get_baudrate
                0x00000000       0x1c CMakeFiles/main.dir/__/pico-sdk/src/rp2_common/hardware_spi/spi.c.obj
 .time_critical.spi_read_blocking
                0x00000000       0x48 CMakeFiles/main.dir/__/pico-sdk/src/rp2_common/hardware_spi/spi.c.obj
 .time_critical.spi_write16_read16_blocking
                0x00000000       0x58 CMakeFiles/main.dir/__/pico-sdk/src/rp2_common/hardware_spi/spi.c.obj
 .time_critical.spi_write16_blocking
                0x00000000       0x50 CMakeFiles/main.dir/__/pico-sdk/src/rp2_common/hardware_spi/spi.c.obj
 .time_critical.spi_read16_blocking
                0x00000000       0x48 CMakeFiles/main.dir/__/pico-sdk/src/rp2_common/hardware_spi/spi.c.obj
 .text          0x00000000        0x0 CMakeFiles/main.dir/__/pico-sdk/src/rp2_common/hardware_interp/interp.c.obj
 .data          0x00000000        0x0 CMakeFiles/main.dir/__/pico-sdk/src/rp2_common/hardware_interp/interp.c.obj
 .bss           0x00000000        0x0 CMakeFiles/main.dir/__/pico-sdk/src/rp2_common/hardware_interp/interp.c.obj
 .text.interp_claim_lane
                0x00000000       0x28 CMakeFiles/main.dir/__/pico-sdk/src/rp2_common/hardware_interp/interp.c.obj
 .text.interp_claim_lane_mask
                0x00000000       0x48 CMakeFiles/main.dir/__/pico-sdk/src/rp2_common/hardware_interp/interp.c.obj
 .text.interp_unclaim_lane
                0x00000000       0x20 CMakeFiles/main.dir/__/pico-sdk/src/rp2_common/hardware_interp/interp.c.obj
 .text.interp_lane_is_claimed
                0x00000000       0x20 CMakeFiles/main.dir/__/pico-sdk/src/rp2_common/hardware_interp/interp.c.obj
 .text.interp_unclaim_lane_mask
                0x00000000       0x40 CMakeFiles/main.dir/__/pico-sdk/src/rp2_common/hardware_interp/interp.c.obj
 .text.interp_save
                0x00000000       0x20 CMakeFiles/main.dir/__/pico-sdk/src/rp2_common/hardware_interp/interp.c.obj
 .text.interp_restore
                0x00000000       0x20 CMakeFiles/main.dir/__/pico-sdk/src/rp2_common/hardware_interp/interp.c.obj
 .bss._claimed  0x00000000        0x1 CMakeFiles/main.dir/__/pico-sdk/src/rp2_common/hardware_interp/interp.c.obj
 .rodata.interp_claim_lane.str1.4
                0x00000000       0x18 CMakeFiles/main.dir/__/pico-sdk/src/rp2_common/hardware_interp/interp.c.obj
 .comment       0x00000000       0x58 CMakeFiles/main.dir/__/pico-sdk/src/rp2_common/hardware_interp/interp.c.obj
 .ARM.attributes
                0x00000000       0x32 CMakeFiles/main.dir/__/pico-sdk/src/rp2_common/hardware_interp/interp.c.obj
 .text          0x00000000        0x0 CMakeFiles/main.dir/__/pico-sdk/src/rp2_common/hardware_i2c/i2c.c.obj
 .data          0x00000000        0x0 CMakeFiles/main.dir/__/pico-sdk/src/rp2_common/hardware_i2c/i2c.c.obj
 .bss           0x00000000        0x0 CMakeFiles/main.dir/__/pico-sdk/src/rp2_common/hardware_i2c/i2c.c.obj
 .text.i2c_deinit
                0x00000000       0x20 CMakeFiles/main.dir/__/pico-sdk/src/rp2_common/hardware_i2c/i2c.c.obj
 .text.i2c_set_baudrate
                0x00000000       0xc0 CMakeFiles/main.dir/__/pico-sdk/src/rp2_common/hardware_i2c/i2c.c.obj
 .text.i2c_set_slave_mode
                0x00000000       0x3c CMakeFiles/main.dir/__/pico-sdk/src/rp2_common/hardware_i2c/i2c.c.obj
 .text.i2c_write_blocking
                0x00000000       0xdc CMakeFiles/main.dir/__/pico-sdk/src/rp2_common/hardware_i2c/i2c.c.obj
 .text.i2c_write_timeout_per_char_us
                0x00000000       0x44 CMakeFiles/main.dir/__/pico-sdk/src/rp2_common/hardware_i2c/i2c.c.obj
 .text.i2c_read_blocking
                0x00000000       0x98 CMakeFiles/main.dir/__/pico-sdk/src/rp2_common/hardware_i2c/i2c.c.obj
 .text.i2c_read_timeout_per_char_us
                0x00000000       0x44 CMakeFiles/main.dir/__/pico-sdk/src/rp2_common/hardware_i2c/i2c.c.obj
 .group         0x00000000       0x14 libLoRa_pico_lib.a(LoRa-RP2040.cpp.obj)
 .text          0x00000000        0x0 libLoRa_pico_lib.a(LoRa-RP2040.cpp.obj)
 .data          0x00000000        0x0 libLoRa_pico_lib.a(LoRa-RP2040.cpp.obj)
 .bss           0x00000000        0x0 libLoRa_pico_lib.a(LoRa-RP2040.cpp.obj)
 .ARM.extab.text._ZN9LoRaClass5flushEv
                0x00000000        0x0 libLoRa_pico_lib.a(LoRa-RP2040.cpp.obj)
 .text._ZN9LoRaClass10onDio0RiseEjm
                0x00000000      0x190 libLoRa_pico_lib.a(LoRa-RP2040.cpp.obj)
 .ARM.extab.text._ZN9LoRaClass10onDio0RiseEjm
                0x00000000        0xc libLoRa_pico_lib.a(LoRa-RP2040.cpp.obj)
 .ARM.exidx.text._ZN9LoRaClass10onDio0RiseEjm
                0x00000000        0x8 libLoRa_pico_lib.a(LoRa-RP2040.cpp.obj)
 .text._ZN9LoRaClassC2Ev
                0x00000000       0x30 libLoRa_pico_lib.a(LoRa-RP2040.cpp.obj)
 .ARM.extab.text._ZN9LoRaClassC2Ev
                0x00000000        0x0 libLoRa_pico_lib.a(LoRa-RP2040.cpp.obj)
 .ARM.exidx.text._ZN9LoRaClassC2Ev
                0x00000000        0x8 libLoRa_pico_lib.a(LoRa-RP2040.cpp.obj)
 .text._ZN9LoRaClass3endEv
                0x00000000       0x5c libLoRa_pico_lib.a(LoRa-RP2040.cpp.obj)
 .ARM.extab.text._ZN9LoRaClass3endEv
                0x00000000        0xc libLoRa_pico_lib.a(LoRa-RP2040.cpp.obj)
 .ARM.exidx.text._ZN9LoRaClass3endEv
                0x00000000        0x8 libLoRa_pico_lib.a(LoRa-RP2040.cpp.obj)
 .text._ZN9LoRaClass14isTransmittingEv
                0x00000000       0xd0 libLoRa_pico_lib.a(LoRa-RP2040.cpp.obj)
 .ARM.extab.text._ZN9LoRaClass14isTransmittingEv
                0x00000000        0xc libLoRa_pico_lib.a(LoRa-RP2040.cpp.obj)
 .ARM.exidx.text._ZN9LoRaClass14isTransmittingEv
                0x00000000        0x8 libLoRa_pico_lib.a(LoRa-RP2040.cpp.obj)
 .text._ZN9LoRaClass9packetSnrEv
                0x00000000       0x78 libLoRa_pico_lib.a(LoRa-RP2040.cpp.obj)
 .ARM.extab.text._ZN9LoRaClass9packetSnrEv
                0x00000000        0xc libLoRa_pico_lib.a(LoRa-RP2040.cpp.obj)
 .ARM.exidx.text._ZN9LoRaClass9packetSnrEv
                0x00000000        0x8 libLoRa_pico_lib.a(LoRa-RP2040.cpp.obj)
 .text._ZN9LoRaClass20packetFrequencyErrorEv
                0x00000000      0x190 libLoRa_pico_lib.a(LoRa-RP2040.cpp.obj)
 .ARM.extab.text._ZN9LoRaClass20packetFrequencyErrorEv
                0x00000000        0xc libLoRa_pico_lib.a(LoRa-RP2040.cpp.obj)
 .ARM.exidx.text._ZN9LoRaClass20packetFrequencyErrorEv
                0x00000000        0x8 libLoRa_pico_lib.a(LoRa-RP2040.cpp.obj)
 .text._ZN9LoRaClass4rssiEv
                0x00000000       0x7c libLoRa_pico_lib.a(LoRa-RP2040.cpp.obj)
 .ARM.extab.text._ZN9LoRaClass4rssiEv
                0x00000000        0xc libLoRa_pico_lib.a(LoRa-RP2040.cpp.obj)
 .ARM.exidx.text._ZN9LoRaClass4rssiEv
                0x00000000        0x8 libLoRa_pico_lib.a(LoRa-RP2040.cpp.obj)
 .text._ZN9LoRaClass9onReceiveEPFviE
                0x00000000       0x24 libLoRa_pico_lib.a(LoRa-RP2040.cpp.obj)
 .ARM.extab.text._ZN9LoRaClass9onReceiveEPFviE
                0x00000000        0x0 libLoRa_pico_lib.a(LoRa-RP2040.cpp.obj)
 .ARM.exidx.text._ZN9LoRaClass9onReceiveEPFviE
                0x00000000        0x8 libLoRa_pico_lib.a(LoRa-RP2040.cpp.obj)
 .text._ZN9LoRaClass8onTxDoneEPFvvE
                0x00000000       0x24 libLoRa_pico_lib.a(LoRa-RP2040.cpp.obj)
 .ARM.extab.text._ZN9LoRaClass8onTxDoneEPFvvE
                0x00000000        0x0 libLoRa_pico_lib.a(LoRa-RP2040.cpp.obj)
 .ARM.exidx.text._ZN9LoRaClass8onTxDoneEPFvvE
                0x00000000        0x8 libLoRa_pico_lib.a(LoRa-RP2040.cpp.obj)
 .text._ZN9LoRaClass4idleEv
                0x00000000       0x54 libLoRa_pico_lib.a(LoRa-RP2040.cpp.obj)
 .ARM.extab.text._ZN9LoRaClass4idleEv
                0x00000000        0xc libLoRa_pico_lib.a(LoRa-RP2040.cpp.obj)
 .ARM.exidx.text._ZN9LoRaClass4idleEv
                0x00000000        0x8 libLoRa_pico_lib.a(LoRa-RP2040.cpp.obj)
 .text._ZN9LoRaClass5sleepEv
                0x00000000       0x58 libLoRa_pico_lib.a(LoRa-RP2040.cpp.obj)
 .ARM.extab.text._ZN9LoRaClass5sleepEv
                0x00000000        0xc libLoRa_pico_lib.a(LoRa-RP2040.cpp.obj)
 .ARM.exidx.text._ZN9LoRaClass5sleepEv
                0x00000000        0x8 libLoRa_pico_lib.a(LoRa-RP2040.cpp.obj)
 .text._ZN9LoRaClass12setFrequencyEl
                0x00000000       0xe0 libLoRa_pico_lib.a(LoRa-RP2040.cpp.obj)
 .ARM.extab.text._ZN9LoRaClass12setFrequencyEl
                0x00000000        0xc libLoRa_pico_lib.a(LoRa-RP2040.cpp.obj)
 .ARM.exidx.text._ZN9LoRaClass12setFrequencyEl
                0x00000000        0x8 libLoRa_pico_lib.a(LoRa-RP2040.cpp.obj)
 .text._ZN9LoRaClass18getSpreadingFactorEv
                0x00000000       0x64 libLoRa_pico_lib.a(LoRa-RP2040.cpp.obj)
 .ARM.extab.text._ZN9LoRaClass18getSpreadingFactorEv
                0x00000000        0xc libLoRa_pico_lib.a(LoRa-RP2040.cpp.obj)
 .ARM.exidx.text._ZN9LoRaClass18getSpreadingFactorEv
                0x00000000        0x8 libLoRa_pico_lib.a(LoRa-RP2040.cpp.obj)
 .text._ZN9LoRaClass18getSignalBandwidthEv
                0x00000000       0x70 libLoRa_pico_lib.a(LoRa-RP2040.cpp.obj)
 .ARM.extab.text._ZN9LoRaClass18getSignalBandwidthEv
                0x00000000        0xc libLoRa_pico_lib.a(LoRa-RP2040.cpp.obj)
 .ARM.exidx.text._ZN9LoRaClass18getSignalBandwidthEv
                0x00000000        0x8 libLoRa_pico_lib.a(LoRa-RP2040.cpp.obj)
 .text._ZN9LoRaClass10setLdoFlagEv
                0x00000000      0x144 libLoRa_pico_lib.a(LoRa-RP2040.cpp.obj)
 .ARM.extab.text._ZN9LoRaClass10setLdoFlagEv
                0x00000000        0xc libLoRa_pico_lib.a(LoRa-RP2040.cpp.obj)
 .ARM.exidx.text._ZN9LoRaClass10setLdoFlagEv
                0x00000000        0x8 libLoRa_pico_lib.a(LoRa-RP2040.cpp.obj)
 .text._ZN9LoRaClass11setSyncWordEi
                0x00000000       0x54 libLoRa_pico_lib.a(LoRa-RP2040.cpp.obj)
 .ARM.extab.text._ZN9LoRaClass11setSyncWordEi
                0x00000000        0xc libLoRa_pico_lib.a(LoRa-RP2040.cpp.obj)
 .ARM.exidx.text._ZN9LoRaClass11setSyncWordEi
                0x00000000        0x8 libLoRa_pico_lib.a(LoRa-RP2040.cpp.obj)
 .text._ZN9LoRaClass10disableCrcEv
                0x00000000       0x94 libLoRa_pico_lib.a(LoRa-RP2040.cpp.obj)
 .ARM.extab.text._ZN9LoRaClass10disableCrcEv
                0x00000000        0xc libLoRa_pico_lib.a(LoRa-RP2040.cpp.obj)
 .ARM.exidx.text._ZN9LoRaClass10disableCrcEv
                0x00000000        0x8 libLoRa_pico_lib.a(LoRa-RP2040.cpp.obj)
 .text._ZN9LoRaClass14enableInvertIQEv
                0x00000000       0x88 libLoRa_pico_lib.a(LoRa-RP2040.cpp.obj)
 .ARM.extab.text._ZN9LoRaClass14enableInvertIQEv
                0x00000000        0xc libLoRa_pico_lib.a(LoRa-RP2040.cpp.obj)
 .ARM.exidx.text._ZN9LoRaClass14enableInvertIQEv
                0x00000000        0x8 libLoRa_pico_lib.a(LoRa-RP2040.cpp.obj)
 .text._ZN9LoRaClass15disableInvertIQEv
                0x00000000       0x88 libLoRa_pico_lib.a(LoRa-RP2040.cpp.obj)
 .ARM.extab.text._ZN9LoRaClass15disableInvertIQEv
                0x00000000        0xc libLoRa_pico_lib.a(LoRa-RP2040.cpp.obj)
 .ARM.exidx.text._ZN9LoRaClass15disableInvertIQEv
                0x00000000        0x8 libLoRa_pico_lib.a(LoRa-RP2040.cpp.obj)
 .text._ZN9LoRaClass6setOCPEh
                0x00000000       0x74 libLoRa_pico_lib.a(LoRa-RP2040.cpp.obj)
 .ARM.extab.text._ZN9LoRaClass6setOCPEh
                0x00000000        0x0 libLoRa_pico_lib.a(LoRa-RP2040.cpp.obj)
 .ARM.exidx.text._ZN9LoRaClass6setOCPEh
                0x00000000        0x8 libLoRa_pico_lib.a(LoRa-RP2040.cpp.obj)
 .text._ZN9LoRaClass7setGainEh
                0x00000000      0x170 libLoRa_pico_lib.a(LoRa-RP2040.cpp.obj)
 .ARM.extab.text._ZN9LoRaClass7setGainEh
                0x00000000        0xc libLoRa_pico_lib.a(LoRa-RP2040.cpp.obj)
 .ARM.exidx.text._ZN9LoRaClass7setGainEh
                0x00000000        0x8 libLoRa_pico_lib.a(LoRa-RP2040.cpp.obj)
 .text._ZN9LoRaClass6randomEv
                0x00000000       0x60 libLoRa_pico_lib.a(LoRa-RP2040.cpp.obj)
 .ARM.extab.text._ZN9LoRaClass6randomEv
                0x00000000        0xc libLoRa_pico_lib.a(LoRa-RP2040.cpp.obj)
 .ARM.exidx.text._ZN9LoRaClass6randomEv
                0x00000000        0x8 libLoRa_pico_lib.a(LoRa-RP2040.cpp.obj)
 .text._ZN9LoRaClass7setPinsEiii
                0x00000000        0x8 libLoRa_pico_lib.a(LoRa-RP2040.cpp.obj)
 .ARM.extab.text._ZN9LoRaClass7setPinsEiii
                0x00000000        0x0 libLoRa_pico_lib.a(LoRa-RP2040.cpp.obj)
 .ARM.exidx.text._ZN9LoRaClass7setPinsEiii
                0x00000000        0x8 libLoRa_pico_lib.a(LoRa-RP2040.cpp.obj)
 .text._ZN9LoRaClass6setSPIER8spi_inst
                0x00000000        0x4 libLoRa_pico_lib.a(LoRa-RP2040.cpp.obj)
 .ARM.extab.text._ZN9LoRaClass6setSPIER8spi_inst
                0x00000000        0x0 libLoRa_pico_lib.a(LoRa-RP2040.cpp.obj)
 .ARM.exidx.text._ZN9LoRaClass6setSPIER8spi_inst
                0x00000000        0x8 libLoRa_pico_lib.a(LoRa-RP2040.cpp.obj)
 .text._ZN9LoRaClass15setSPIFrequencyEm
                0x00000000       0x10 libLoRa_pico_lib.a(LoRa-RP2040.cpp.obj)
 .ARM.extab.text._ZN9LoRaClass15setSPIFrequencyEm
                0x00000000        0x0 libLoRa_pico_lib.a(LoRa-RP2040.cpp.obj)
 .ARM.exidx.text._ZN9LoRaClass15setSPIFrequencyEm
                0x00000000        0x8 libLoRa_pico_lib.a(LoRa-RP2040.cpp.obj)
 .text._ZN9LoRaClass13dumpRegistersEv
                0x00000000       0x80 libLoRa_pico_lib.a(LoRa-RP2040.cpp.obj)
 .ARM.extab.text._ZN9LoRaClass13dumpRegistersEv
                0x00000000        0xc libLoRa_pico_lib.a(LoRa-RP2040.cpp.obj)
 .ARM.exidx.text._ZN9LoRaClass13dumpRegistersEv
                0x00000000        0x8 libLoRa_pico_lib.a(LoRa-RP2040.cpp.obj)
 .text._ZN9LoRaClass18explicitHeaderModeEv
                0x00000000       0x90 libLoRa_pico_lib.a(LoRa-RP2040.cpp.obj)
 .ARM.extab.text._ZN9LoRaClass18explicitHeaderModeEv
                0x00000000        0xc libLoRa_pico_lib.a(LoRa-RP2040.cpp.obj)
 .ARM.exidx.text._ZN9LoRaClass18explicitHeaderModeEv
                0x00000000        0x8 libLoRa_pico_lib.a(LoRa-RP2040.cpp.obj)
 .text._ZN9LoRaClass18implicitHeaderModeEv
                0x00000000       0x98 libLoRa_pico_lib.a(LoRa-RP2040.cpp.obj)
 .ARM.extab.text._ZN9LoRaClass18implicitHeaderModeEv
                0x00000000        0xc libLoRa_pico_lib.a(LoRa-RP2040.cpp.obj)
 .ARM.exidx.text._ZN9LoRaClass18implicitHeaderModeEv
                0x00000000        0x8 libLoRa_pico_lib.a(LoRa-RP2040.cpp.obj)
 .text._ZN9LoRaClass14handleDio0RiseEv
                0x00000000      0x188 libLoRa_pico_lib.a(LoRa-RP2040.cpp.obj)
 .ARM.extab.text._ZN9LoRaClass14handleDio0RiseEv
                0x00000000        0xc libLoRa_pico_lib.a(LoRa-RP2040.cpp.obj)
 .ARM.exidx.text._ZN9LoRaClass14handleDio0RiseEv
                0x00000000        0x8 libLoRa_pico_lib.a(LoRa-RP2040.cpp.obj)
 .text._ZN9LoRaClass12readRegisterEh
                0x00000000       0x64 libLoRa_pico_lib.a(LoRa-RP2040.cpp.obj)
 .ARM.extab.text._ZN9LoRaClass12readRegisterEh
                0x00000000        0xc libLoRa_pico_lib.a(LoRa-RP2040.cpp.obj)
 .ARM.exidx.text._ZN9LoRaClass12readRegisterEh
                0x00000000        0x8 libLoRa_pico_lib.a(LoRa-RP2040.cpp.obj)
 .text._ZN9LoRaClass13writeRegisterEhh
                0x00000000       0x58 libLoRa_pico_lib.a(LoRa-RP2040.cpp.obj)
 .ARM.extab.text._ZN9LoRaClass13writeRegisterEhh
                0x00000000        0xc libLoRa_pico_lib.a(LoRa-RP2040.cpp.obj)
 .ARM.exidx.text._ZN9LoRaClass13writeRegisterEhh
                0x00000000        0x8 libLoRa_pico_lib.a(LoRa-RP2040.cpp.obj)
 .text._ZN9LoRaClass14singleTransferEhh
                0x00000000       0x5c libLoRa_pico_lib.a(LoRa-RP2040.cpp.obj)
 .ARM.extab.text._ZN9LoRaClass14singleTransferEhh
                0x00000000        0xc libLoRa_pico_lib.a(LoRa-RP2040.cpp.obj)
 .ARM.exidx.text._ZN9LoRaClass14singleTransferEhh
                0x00000000        0x8 libLoRa_pico_lib.a(LoRa-RP2040.cpp.obj)
 .ARM.extab.text.startup._GLOBAL__sub_I__ZN9LoRaClassC2Ev
                0x00000000        0x0 libLoRa_pico_lib.a(LoRa-RP2040.cpp.obj)
 .rodata._ZN9LoRaClass13dumpRegistersEv.str1.4
                0x00000000        0xb libLoRa_pico_lib.a(LoRa-RP2040.cpp.obj)
 .data          0x00000000        0x0 libKISS.a(kiss.cpp.obj)
 .text          0x00000000        0x0 libi2c_sensor.a(i2c_sensor.cpp.obj)
 .data          0x00000000        0x0 libi2c_sensor.a(i2c_sensor.cpp.obj)
 .bss           0x00000000        0x0 libi2c_sensor.a(i2c_sensor.cpp.obj)
 .text._Z9reg_writeP8i2c_instjhPhh
                0x00000000       0x78 libi2c_sensor.a(i2c_sensor.cpp.obj)
 .ARM.extab.text._Z9reg_writeP8i2c_instjhPhh
                0x00000000        0xc libi2c_sensor.a(i2c_sensor.cpp.obj)
 .ARM.exidx.text._Z9reg_writeP8i2c_instjhPhh
                0x00000000        0x8 libi2c_sensor.a(i2c_sensor.cpp.obj)
 .text._Z8reg_readP8i2c_instjhPhh
                0x00000000       0x94 libi2c_sensor.a(i2c_sensor.cpp.obj)
 .ARM.extab.text._Z8reg_readP8i2c_instjhPhh
                0x00000000        0xc libi2c_sensor.a(i2c_sensor.cpp.obj)
 .ARM.exidx.text._Z8reg_readP8i2c_instjhPhh
                0x00000000        0x8 libi2c_sensor.a(i2c_sensor.cpp.obj)
 .text          0x00000000        0x0 /tmp/ccWYemgR.o
 .data          0x00000000        0x0 /tmp/ccWYemgR.o
 .bss           0x00000000        0x0 /tmp/ccWYemgR.o
 .data          0x00000000        0x0 /usr/lib/gcc/arm-none-eabi/7.3.1/thumb/v6-m/libgcc.a(_dvmd_tls.o)
 .bss           0x00000000        0x0 /usr/lib/gcc/arm-none-eabi/7.3.1/thumb/v6-m/libgcc.a(_dvmd_tls.o)
 .data          0x00000000        0x0 /usr/lib/gcc/arm-none-eabi/7.3.1/thumb/v6-m/libgcc.a(unwind-arm.o)
 .bss           0x00000000        0x0 /usr/lib/gcc/arm-none-eabi/7.3.1/thumb/v6-m/libgcc.a(unwind-arm.o)
 .debug_info    0x00000000     0x1c24 /usr/lib/gcc/arm-none-eabi/7.3.1/thumb/v6-m/libgcc.a(unwind-arm.o)
 .debug_abbrev  0x00000000      0x3d4 /usr/lib/gcc/arm-none-eabi/7.3.1/thumb/v6-m/libgcc.a(unwind-arm.o)
 .debug_loc     0x00000000     0x1cf2 /usr/lib/gcc/arm-none-eabi/7.3.1/thumb/v6-m/libgcc.a(unwind-arm.o)
 .debug_aranges
                0x00000000       0x20 /usr/lib/gcc/arm-none-eabi/7.3.1/thumb/v6-m/libgcc.a(unwind-arm.o)
 .debug_ranges  0x00000000      0x120 /usr/lib/gcc/arm-none-eabi/7.3.1/thumb/v6-m/libgcc.a(unwind-arm.o)
 .debug_line    0x00000000      0x4de /usr/lib/gcc/arm-none-eabi/7.3.1/thumb/v6-m/libgcc.a(unwind-arm.o)
 .debug_str     0x00000000      0xca0 /usr/lib/gcc/arm-none-eabi/7.3.1/thumb/v6-m/libgcc.a(unwind-arm.o)
 .comment       0x00000000       0x58 /usr/lib/gcc/arm-none-eabi/7.3.1/thumb/v6-m/libgcc.a(unwind-arm.o)
 .debug_frame   0x00000000      0x2b4 /usr/lib/gcc/arm-none-eabi/7.3.1/thumb/v6-m/libgcc.a(unwind-arm.o)
 .ARM.attributes
                0x00000000       0x2c /usr/lib/gcc/arm-none-eabi/7.3.1/thumb/v6-m/libgcc.a(unwind-arm.o)
 .data          0x00000000        0x0 /usr/lib/gcc/arm-none-eabi/7.3.1/thumb/v6-m/libgcc.a(libunwind.o)
 .bss           0x00000000        0x0 /usr/lib/gcc/arm-none-eabi/7.3.1/thumb/v6-m/libgcc.a(libunwind.o)
 .debug_line    0x00000000       0x87 /usr/lib/gcc/arm-none-eabi/7.3.1/thumb/v6-m/libgcc.a(libunwind.o)
 .debug_info    0x00000000       0x26 /usr/lib/gcc/arm-none-eabi/7.3.1/thumb/v6-m/libgcc.a(libunwind.o)
 .debug_abbrev  0x00000000       0x14 /usr/lib/gcc/arm-none-eabi/7.3.1/thumb/v6-m/libgcc.a(libunwind.o)
 .debug_aranges
                0x00000000       0x20 /usr/lib/gcc/arm-none-eabi/7.3.1/thumb/v6-m/libgcc.a(libunwind.o)
 .debug_str     0x00000000       0x9d /usr/lib/gcc/arm-none-eabi/7.3.1/thumb/v6-m/libgcc.a(libunwind.o)
 .ARM.attributes
                0x00000000       0x1e /usr/lib/gcc/arm-none-eabi/7.3.1/thumb/v6-m/libgcc.a(libunwind.o)
 .data          0x00000000        0x0 /usr/lib/gcc/arm-none-eabi/7.3.1/thumb/v6-m/libgcc.a(pr-support.o)
 .bss           0x00000000        0x0 /usr/lib/gcc/arm-none-eabi/7.3.1/thumb/v6-m/libgcc.a(pr-support.o)
 .debug_info    0x00000000      0x90c /usr/lib/gcc/arm-none-eabi/7.3.1/thumb/v6-m/libgcc.a(pr-support.o)
 .debug_abbrev  0x00000000      0x278 /usr/lib/gcc/arm-none-eabi/7.3.1/thumb/v6-m/libgcc.a(pr-support.o)
 .debug_loc     0x00000000      0x525 /usr/lib/gcc/arm-none-eabi/7.3.1/thumb/v6-m/libgcc.a(pr-support.o)
 .debug_aranges
                0x00000000       0x20 /usr/lib/gcc/arm-none-eabi/7.3.1/thumb/v6-m/libgcc.a(pr-support.o)
 .debug_ranges  0x00000000       0x38 /usr/lib/gcc/arm-none-eabi/7.3.1/thumb/v6-m/libgcc.a(pr-support.o)
 .debug_line    0x00000000      0x1d7 /usr/lib/gcc/arm-none-eabi/7.3.1/thumb/v6-m/libgcc.a(pr-support.o)
 .debug_str     0x00000000      0x56a /usr/lib/gcc/arm-none-eabi/7.3.1/thumb/v6-m/libgcc.a(pr-support.o)
 .comment       0x00000000       0x58 /usr/lib/gcc/arm-none-eabi/7.3.1/thumb/v6-m/libgcc.a(pr-support.o)
 .debug_frame   0x00000000       0xf4 /usr/lib/gcc/arm-none-eabi/7.3.1/thumb/v6-m/libgcc.a(pr-support.o)
 .ARM.attributes
                0x00000000       0x2c /usr/lib/gcc/arm-none-eabi/7.3.1/thumb/v6-m/libgcc.a(pr-support.o)
 .data          0x00000000        0x0 /usr/lib/gcc/arm-none-eabi/7.3.1/../../../arm-none-eabi/lib/thumb/v6-m/libc.a(lib_a-abort.o)
 .bss           0x00000000        0x0 /usr/lib/gcc/arm-none-eabi/7.3.1/../../../arm-none-eabi/lib/thumb/v6-m/libc.a(lib_a-abort.o)
 .debug_info    0x00000000      0x92b /usr/lib/gcc/arm-none-eabi/7.3.1/../../../arm-none-eabi/lib/thumb/v6-m/libc.a(lib_a-abort.o)
 .debug_abbrev  0x00000000      0x1e1 /usr/lib/gcc/arm-none-eabi/7.3.1/../../../arm-none-eabi/lib/thumb/v6-m/libc.a(lib_a-abort.o)
 .debug_aranges
                0x00000000       0x20 /usr/lib/gcc/arm-none-eabi/7.3.1/../../../arm-none-eabi/lib/thumb/v6-m/libc.a(lib_a-abort.o)
 .debug_line    0x00000000      0x133 /usr/lib/gcc/arm-none-eabi/7.3.1/../../../arm-none-eabi/lib/thumb/v6-m/libc.a(lib_a-abort.o)
 .debug_str     0x00000000      0x5c2 /usr/lib/gcc/arm-none-eabi/7.3.1/../../../arm-none-eabi/lib/thumb/v6-m/libc.a(lib_a-abort.o)
 .comment       0x00000000       0x58 /usr/lib/gcc/arm-none-eabi/7.3.1/../../../arm-none-eabi/lib/thumb/v6-m/libc.a(lib_a-abort.o)
 .debug_frame   0x00000000       0x28 /usr/lib/gcc/arm-none-eabi/7.3.1/../../../arm-none-eabi/lib/thumb/v6-m/libc.a(lib_a-abort.o)
 .ARM.attributes
                0x00000000       0x2c /usr/lib/gcc/arm-none-eabi/7.3.1/../../../arm-none-eabi/lib/thumb/v6-m/libc.a(lib_a-abort.o)
 .text          0x00000000       0x10 /usr/lib/gcc/arm-none-eabi/7.3.1/../../../arm-none-eabi/lib/thumb/v6-m/libc.a(lib_a-atexit.o)
 .data          0x00000000        0x0 /usr/lib/gcc/arm-none-eabi/7.3.1/../../../arm-none-eabi/lib/thumb/v6-m/libc.a(lib_a-atexit.o)
 .bss           0x00000000        0x0 /usr/lib/gcc/arm-none-eabi/7.3.1/../../../arm-none-eabi/lib/thumb/v6-m/libc.a(lib_a-atexit.o)
 .debug_info    0x00000000      0x90c /usr/lib/gcc/arm-none-eabi/7.3.1/../../../arm-none-eabi/lib/thumb/v6-m/libc.a(lib_a-atexit.o)
 .debug_abbrev  0x00000000      0x1fe /usr/lib/gcc/arm-none-eabi/7.3.1/../../../arm-none-eabi/lib/thumb/v6-m/libc.a(lib_a-atexit.o)
 .debug_loc     0x00000000       0x2c /usr/lib/gcc/arm-none-eabi/7.3.1/../../../arm-none-eabi/lib/thumb/v6-m/libc.a(lib_a-atexit.o)
 .debug_aranges
                0x00000000       0x20 /usr/lib/gcc/arm-none-eabi/7.3.1/../../../arm-none-eabi/lib/thumb/v6-m/libc.a(lib_a-atexit.o)
 .debug_line    0x00000000      0x129 /usr/lib/gcc/arm-none-eabi/7.3.1/../../../arm-none-eabi/lib/thumb/v6-m/libc.a(lib_a-atexit.o)
 .debug_str     0x00000000      0x5cf /usr/lib/gcc/arm-none-eabi/7.3.1/../../../arm-none-eabi/lib/thumb/v6-m/libc.a(lib_a-atexit.o)
 .comment       0x00000000       0x58 /usr/lib/gcc/arm-none-eabi/7.3.1/../../../arm-none-eabi/lib/thumb/v6-m/libc.a(lib_a-atexit.o)
 .debug_frame   0x00000000       0x28 /usr/lib/gcc/arm-none-eabi/7.3.1/../../../arm-none-eabi/lib/thumb/v6-m/libc.a(lib_a-atexit.o)
 .ARM.attributes
                0x00000000       0x2c /usr/lib/gcc/arm-none-eabi/7.3.1/../../../arm-none-eabi/lib/thumb/v6-m/libc.a(lib_a-atexit.o)
 .text          0x00000000       0x18 /usr/lib/gcc/arm-none-eabi/7.3.1/../../../arm-none-eabi/lib/thumb/v6-m/libc.a(lib_a-calloc.o)
 .data          0x00000000        0x0 /usr/lib/gcc/arm-none-eabi/7.3.1/../../../arm-none-eabi/lib/thumb/v6-m/libc.a(lib_a-calloc.o)
 .bss           0x00000000        0x0 /usr/lib/gcc/arm-none-eabi/7.3.1/../../../arm-none-eabi/lib/thumb/v6-m/libc.a(lib_a-calloc.o)
 .debug_info    0x00000000      0x8fa /usr/lib/gcc/arm-none-eabi/7.3.1/../../../arm-none-eabi/lib/thumb/v6-m/libc.a(lib_a-calloc.o)
 .debug_abbrev  0x00000000      0x1f1 /usr/lib/gcc/arm-none-eabi/7.3.1/../../../arm-none-eabi/lib/thumb/v6-m/libc.a(lib_a-calloc.o)
 .debug_loc     0x00000000       0x58 /usr/lib/gcc/arm-none-eabi/7.3.1/../../../arm-none-eabi/lib/thumb/v6-m/libc.a(lib_a-calloc.o)
 .debug_aranges
                0x00000000       0x20 /usr/lib/gcc/arm-none-eabi/7.3.1/../../../arm-none-eabi/lib/thumb/v6-m/libc.a(lib_a-calloc.o)
 .debug_line    0x00000000      0x11e /usr/lib/gcc/arm-none-eabi/7.3.1/../../../arm-none-eabi/lib/thumb/v6-m/libc.a(lib_a-calloc.o)
 .debug_str     0x00000000      0x5a1 /usr/lib/gcc/arm-none-eabi/7.3.1/../../../arm-none-eabi/lib/thumb/v6-m/libc.a(lib_a-calloc.o)
 .comment       0x00000000       0x58 /usr/lib/gcc/arm-none-eabi/7.3.1/../../../arm-none-eabi/lib/thumb/v6-m/libc.a(lib_a-calloc.o)
 .debug_frame   0x00000000       0x28 /usr/lib/gcc/arm-none-eabi/7.3.1/../../../arm-none-eabi/lib/thumb/v6-m/libc.a(lib_a-calloc.o)
 .ARM.attributes
                0x00000000       0x2c /usr/lib/gcc/arm-none-eabi/7.3.1/../../../arm-none-eabi/lib/thumb/v6-m/libc.a(lib_a-calloc.o)
 .text          0x00000000       0x58 /usr/lib/gcc/arm-none-eabi/7.3.1/../../../arm-none-eabi/lib/thumb/v6-m/libc.a(lib_a-callocr.o)
 .data          0x00000000        0x0 /usr/lib/gcc/arm-none-eabi/7.3.1/../../../arm-none-eabi/lib/thumb/v6-m/libc.a(lib_a-callocr.o)
 .bss           0x00000000        0x0 /usr/lib/gcc/arm-none-eabi/7.3.1/../../../arm-none-eabi/lib/thumb/v6-m/libc.a(lib_a-callocr.o)
 .debug_info    0x00000000      0xb5d /usr/lib/gcc/arm-none-eabi/7.3.1/../../../arm-none-eabi/lib/thumb/v6-m/libc.a(lib_a-callocr.o)
 .debug_abbrev  0x00000000      0x235 /usr/lib/gcc/arm-none-eabi/7.3.1/../../../arm-none-eabi/lib/thumb/v6-m/libc.a(lib_a-callocr.o)
 .debug_loc     0x00000000      0x226 /usr/lib/gcc/arm-none-eabi/7.3.1/../../../arm-none-eabi/lib/thumb/v6-m/libc.a(lib_a-callocr.o)
 .debug_aranges
                0x00000000       0x20 /usr/lib/gcc/arm-none-eabi/7.3.1/../../../arm-none-eabi/lib/thumb/v6-m/libc.a(lib_a-callocr.o)
 .debug_ranges  0x00000000       0x30 /usr/lib/gcc/arm-none-eabi/7.3.1/../../../arm-none-eabi/lib/thumb/v6-m/libc.a(lib_a-callocr.o)
 .debug_line    0x00000000      0x12b /usr/lib/gcc/arm-none-eabi/7.3.1/../../../arm-none-eabi/lib/thumb/v6-m/libc.a(lib_a-callocr.o)
 .debug_str     0x00000000      0x710 /usr/lib/gcc/arm-none-eabi/7.3.1/../../../arm-none-eabi/lib/thumb/v6-m/libc.a(lib_a-callocr.o)
 .comment       0x00000000       0x58 /usr/lib/gcc/arm-none-eabi/7.3.1/../../../arm-none-eabi/lib/thumb/v6-m/libc.a(lib_a-callocr.o)
 .debug_frame   0x00000000       0x28 /usr/lib/gcc/arm-none-eabi/7.3.1/../../../arm-none-eabi/lib/thumb/v6-m/libc.a(lib_a-callocr.o)
 .ARM.attributes
                0x00000000       0x2c /usr/lib/gcc/arm-none-eabi/7.3.1/../../../arm-none-eabi/lib/thumb/v6-m/libc.a(lib_a-callocr.o)
 .text          0x00000000       0x34 /usr/lib/gcc/arm-none-eabi/7.3.1/../../../arm-none-eabi/lib/thumb/v6-m/libc.a(lib_a-fini.o)
 .data          0x00000000        0x0 /usr/lib/gcc/arm-none-eabi/7.3.1/../../../arm-none-eabi/lib/thumb/v6-m/libc.a(lib_a-fini.o)
 .bss           0x00000000        0x0 /usr/lib/gcc/arm-none-eabi/7.3.1/../../../arm-none-eabi/lib/thumb/v6-m/libc.a(lib_a-fini.o)
 .debug_info    0x00000000       0xf3 /usr/lib/gcc/arm-none-eabi/7.3.1/../../../arm-none-eabi/lib/thumb/v6-m/libc.a(lib_a-fini.o)
 .debug_abbrev  0x00000000       0xba /usr/lib/gcc/arm-none-eabi/7.3.1/../../../arm-none-eabi/lib/thumb/v6-m/libc.a(lib_a-fini.o)
 .debug_loc     0x00000000       0x3e /usr/lib/gcc/arm-none-eabi/7.3.1/../../../arm-none-eabi/lib/thumb/v6-m/libc.a(lib_a-fini.o)
 .debug_aranges
                0x00000000       0x20 /usr/lib/gcc/arm-none-eabi/7.3.1/../../../arm-none-eabi/lib/thumb/v6-m/libc.a(lib_a-fini.o)
 .debug_line    0x00000000       0x9f /usr/lib/gcc/arm-none-eabi/7.3.1/../../../arm-none-eabi/lib/thumb/v6-m/libc.a(lib_a-fini.o)
 .debug_str     0x00000000      0x1de /usr/lib/gcc/arm-none-eabi/7.3.1/../../../arm-none-eabi/lib/thumb/v6-m/libc.a(lib_a-fini.o)
 .comment       0x00000000       0x58 /usr/lib/gcc/arm-none-eabi/7.3.1/../../../arm-none-eabi/lib/thumb/v6-m/libc.a(lib_a-fini.o)
 .debug_frame   0x00000000       0x2c /usr/lib/gcc/arm-none-eabi/7.3.1/../../../arm-none-eabi/lib/thumb/v6-m/libc.a(lib_a-fini.o)
 .ARM.attributes
                0x00000000       0x2c /usr/lib/gcc/arm-none-eabi/7.3.1/../../../arm-none-eabi/lib/thumb/v6-m/libc.a(lib_a-fini.o)
 .text          0x00000000        0x0 /usr/lib/gcc/arm-none-eabi/7.3.1/../../../arm-none-eabi/lib/thumb/v6-m/libc.a(lib_a-impure.o)
 .bss           0x00000000        0x0 /usr/lib/gcc/arm-none-eabi/7.3.1/../../../arm-none-eabi/lib/thumb/v6-m/libc.a(lib_a-impure.o)
 .rodata        0x00000000        0x4 /usr/lib/gcc/arm-none-eabi/7.3.1/../../../arm-none-eabi/lib/thumb/v6-m/libc.a(lib_a-impure.o)
 .debug_info    0x00000000      0x8a9 /usr/lib/gcc/arm-none-eabi/7.3.1/../../../arm-none-eabi/lib/thumb/v6-m/libc.a(lib_a-impure.o)
 .debug_abbrev  0x00000000      0x192 /usr/lib/gcc/arm-none-eabi/7.3.1/../../../arm-none-eabi/lib/thumb/v6-m/libc.a(lib_a-impure.o)
 .debug_aranges
                0x00000000       0x18 /usr/lib/gcc/arm-none-eabi/7.3.1/../../../arm-none-eabi/lib/thumb/v6-m/libc.a(lib_a-impure.o)
 .debug_line    0x00000000       0xd4 /usr/lib/gcc/arm-none-eabi/7.3.1/../../../arm-none-eabi/lib/thumb/v6-m/libc.a(lib_a-impure.o)
 .debug_str     0x00000000      0x584 /usr/lib/gcc/arm-none-eabi/7.3.1/../../../arm-none-eabi/lib/thumb/v6-m/libc.a(lib_a-impure.o)
 .comment       0x00000000       0x58 /usr/lib/gcc/arm-none-eabi/7.3.1/../../../arm-none-eabi/lib/thumb/v6-m/libc.a(lib_a-impure.o)
 .ARM.attributes
                0x00000000       0x2c /usr/lib/gcc/arm-none-eabi/7.3.1/../../../arm-none-eabi/lib/thumb/v6-m/libc.a(lib_a-impure.o)
 .text          0x00000000       0x48 /usr/lib/gcc/arm-none-eabi/7.3.1/../../../arm-none-eabi/lib/thumb/v6-m/libc.a(lib_a-init.o)
 .data          0x00000000        0x0 /usr/lib/gcc/arm-none-eabi/7.3.1/../../../arm-none-eabi/lib/thumb/v6-m/libc.a(lib_a-init.o)
 .bss           0x00000000        0x0 /usr/lib/gcc/arm-none-eabi/7.3.1/../../../arm-none-eabi/lib/thumb/v6-m/libc.a(lib_a-init.o)
 .debug_info    0x00000000      0x109 /usr/lib/gcc/arm-none-eabi/7.3.1/../../../arm-none-eabi/lib/thumb/v6-m/libc.a(lib_a-init.o)
 .debug_abbrev  0x00000000       0xba /usr/lib/gcc/arm-none-eabi/7.3.1/../../../arm-none-eabi/lib/thumb/v6-m/libc.a(lib_a-init.o)
 .debug_loc     0x00000000       0x84 /usr/lib/gcc/arm-none-eabi/7.3.1/../../../arm-none-eabi/lib/thumb/v6-m/libc.a(lib_a-init.o)
 .debug_aranges
                0x00000000       0x20 /usr/lib/gcc/arm-none-eabi/7.3.1/../../../arm-none-eabi/lib/thumb/v6-m/libc.a(lib_a-init.o)
 .debug_line    0x00000000       0xbf /usr/lib/gcc/arm-none-eabi/7.3.1/../../../arm-none-eabi/lib/thumb/v6-m/libc.a(lib_a-init.o)
 .debug_str     0x00000000      0x208 /usr/lib/gcc/arm-none-eabi/7.3.1/../../../arm-none-eabi/lib/thumb/v6-m/libc.a(lib_a-init.o)
 .comment       0x00000000       0x58 /usr/lib/gcc/arm-none-eabi/7.3.1/../../../arm-none-eabi/lib/thumb/v6-m/libc.a(lib_a-init.o)
 .debug_frame   0x00000000       0x2c /usr/lib/gcc/arm-none-eabi/7.3.1/../../../arm-none-eabi/lib/thumb/v6-m/libc.a(lib_a-init.o)
 .ARM.attributes
                0x00000000       0x2c /usr/lib/gcc/arm-none-eabi/7.3.1/../../../arm-none-eabi/lib/thumb/v6-m/libc.a(lib_a-init.o)
 .text          0x00000000       0x28 /usr/lib/gcc/arm-none-eabi/7.3.1/../../../arm-none-eabi/lib/thumb/v6-m/libc.a(lib_a-malloc.o)
 .data          0x00000000        0x0 /usr/lib/gcc/arm-none-eabi/7.3.1/../../../arm-none-eabi/lib/thumb/v6-m/libc.a(lib_a-malloc.o)
 .bss           0x00000000        0x0 /usr/lib/gcc/arm-none-eabi/7.3.1/../../../arm-none-eabi/lib/thumb/v6-m/libc.a(lib_a-malloc.o)
 .debug_info    0x00000000      0x926 /usr/lib/gcc/arm-none-eabi/7.3.1/../../../arm-none-eabi/lib/thumb/v6-m/libc.a(lib_a-malloc.o)
 .debug_abbrev  0x00000000      0x1fc /usr/lib/gcc/arm-none-eabi/7.3.1/../../../arm-none-eabi/lib/thumb/v6-m/libc.a(lib_a-malloc.o)
 .debug_loc     0x00000000       0x58 /usr/lib/gcc/arm-none-eabi/7.3.1/../../../arm-none-eabi/lib/thumb/v6-m/libc.a(lib_a-malloc.o)
 .debug_aranges
                0x00000000       0x20 /usr/lib/gcc/arm-none-eabi/7.3.1/../../../arm-none-eabi/lib/thumb/v6-m/libc.a(lib_a-malloc.o)
 .debug_line    0x00000000      0x130 /usr/lib/gcc/arm-none-eabi/7.3.1/../../../arm-none-eabi/lib/thumb/v6-m/libc.a(lib_a-malloc.o)
 .debug_str     0x00000000      0x5b5 /usr/lib/gcc/arm-none-eabi/7.3.1/../../../arm-none-eabi/lib/thumb/v6-m/libc.a(lib_a-malloc.o)
 .comment       0x00000000       0x58 /usr/lib/gcc/arm-none-eabi/7.3.1/../../../arm-none-eabi/lib/thumb/v6-m/libc.a(lib_a-malloc.o)
 .debug_frame   0x00000000       0x40 /usr/lib/gcc/arm-none-eabi/7.3.1/../../../arm-none-eabi/lib/thumb/v6-m/libc.a(lib_a-malloc.o)
 .ARM.attributes
                0x00000000       0x2c /usr/lib/gcc/arm-none-eabi/7.3.1/../../../arm-none-eabi/lib/thumb/v6-m/libc.a(lib_a-malloc.o)
 .debug_info    0x00000000      0xde7 /usr/lib/gcc/arm-none-eabi/7.3.1/../../../arm-none-eabi/lib/thumb/v6-m/libc.a(lib_a-mallocr.o)
 .debug_abbrev  0x00000000      0x2cd /usr/lib/gcc/arm-none-eabi/7.3.1/../../../arm-none-eabi/lib/thumb/v6-m/libc.a(lib_a-mallocr.o)
 .debug_loc     0x00000000      0xdce /usr/lib/gcc/arm-none-eabi/7.3.1/../../../arm-none-eabi/lib/thumb/v6-m/libc.a(lib_a-mallocr.o)
 .debug_aranges
                0x00000000       0x20 /usr/lib/gcc/arm-none-eabi/7.3.1/../../../arm-none-eabi/lib/thumb/v6-m/libc.a(lib_a-mallocr.o)
 .debug_ranges  0x00000000       0x40 /usr/lib/gcc/arm-none-eabi/7.3.1/../../../arm-none-eabi/lib/thumb/v6-m/libc.a(lib_a-mallocr.o)
 .debug_line    0x00000000      0x36d /usr/lib/gcc/arm-none-eabi/7.3.1/../../../arm-none-eabi/lib/thumb/v6-m/libc.a(lib_a-mallocr.o)
 .debug_str     0x00000000      0x7ec /usr/lib/gcc/arm-none-eabi/7.3.1/../../../arm-none-eabi/lib/thumb/v6-m/libc.a(lib_a-mallocr.o)
 .comment       0x00000000       0x58 /usr/lib/gcc/arm-none-eabi/7.3.1/../../../arm-none-eabi/lib/thumb/v6-m/libc.a(lib_a-mallocr.o)
 .debug_frame   0x00000000       0x3c /usr/lib/gcc/arm-none-eabi/7.3.1/../../../arm-none-eabi/lib/thumb/v6-m/libc.a(lib_a-mallocr.o)
 .ARM.attributes
                0x00000000       0x2c /usr/lib/gcc/arm-none-eabi/7.3.1/../../../arm-none-eabi/lib/thumb/v6-m/libc.a(lib_a-mallocr.o)
 .data          0x00000000        0x0 /usr/lib/gcc/arm-none-eabi/7.3.1/../../../arm-none-eabi/lib/thumb/v6-m/libc.a(lib_a-memmove.o)
 .bss           0x00000000        0x0 /usr/lib/gcc/arm-none-eabi/7.3.1/../../../arm-none-eabi/lib/thumb/v6-m/libc.a(lib_a-memmove.o)
 .data          0x00000000        0x0 /usr/lib/gcc/arm-none-eabi/7.3.1/../../../arm-none-eabi/lib/thumb/v6-m/libc.a(lib_a-mlock.o)
 .bss           0x00000000        0x0 /usr/lib/gcc/arm-none-eabi/7.3.1/../../../arm-none-eabi/lib/thumb/v6-m/libc.a(lib_a-mlock.o)
 .debug_info    0x00000000      0x8dc /usr/lib/gcc/arm-none-eabi/7.3.1/../../../arm-none-eabi/lib/thumb/v6-m/libc.a(lib_a-mlock.o)
 .debug_abbrev  0x00000000      0x1d7 /usr/lib/gcc/arm-none-eabi/7.3.1/../../../arm-none-eabi/lib/thumb/v6-m/libc.a(lib_a-mlock.o)
 .debug_aranges
                0x00000000       0x20 /usr/lib/gcc/arm-none-eabi/7.3.1/../../../arm-none-eabi/lib/thumb/v6-m/libc.a(lib_a-mlock.o)
 .debug_line    0x00000000      0x11a /usr/lib/gcc/arm-none-eabi/7.3.1/../../../arm-none-eabi/lib/thumb/v6-m/libc.a(lib_a-mlock.o)
 .debug_str     0x00000000      0x5b0 /usr/lib/gcc/arm-none-eabi/7.3.1/../../../arm-none-eabi/lib/thumb/v6-m/libc.a(lib_a-mlock.o)
 .comment       0x00000000       0x58 /usr/lib/gcc/arm-none-eabi/7.3.1/../../../arm-none-eabi/lib/thumb/v6-m/libc.a(lib_a-mlock.o)
 .debug_frame   0x00000000       0x30 /usr/lib/gcc/arm-none-eabi/7.3.1/../../../arm-none-eabi/lib/thumb/v6-m/libc.a(lib_a-mlock.o)
 .ARM.attributes
                0x00000000       0x2c /usr/lib/gcc/arm-none-eabi/7.3.1/../../../arm-none-eabi/lib/thumb/v6-m/libc.a(lib_a-mlock.o)
 .data          0x00000000        0x0 /usr/lib/gcc/arm-none-eabi/7.3.1/../../../arm-none-eabi/lib/thumb/v6-m/libc.a(lib_a-sbrkr.o)
 .bss           0x00000000        0x0 /usr/lib/gcc/arm-none-eabi/7.3.1/../../../arm-none-eabi/lib/thumb/v6-m/libc.a(lib_a-sbrkr.o)
 .debug_info    0x00000000      0x95f /usr/lib/gcc/arm-none-eabi/7.3.1/../../../arm-none-eabi/lib/thumb/v6-m/libc.a(lib_a-sbrkr.o)
 .debug_abbrev  0x00000000      0x215 /usr/lib/gcc/arm-none-eabi/7.3.1/../../../arm-none-eabi/lib/thumb/v6-m/libc.a(lib_a-sbrkr.o)
 .debug_loc     0x00000000       0x58 /usr/lib/gcc/arm-none-eabi/7.3.1/../../../arm-none-eabi/lib/thumb/v6-m/libc.a(lib_a-sbrkr.o)
 .debug_aranges
                0x00000000       0x20 /usr/lib/gcc/arm-none-eabi/7.3.1/../../../arm-none-eabi/lib/thumb/v6-m/libc.a(lib_a-sbrkr.o)
 .debug_line    0x00000000      0x132 /usr/lib/gcc/arm-none-eabi/7.3.1/../../../arm-none-eabi/lib/thumb/v6-m/libc.a(lib_a-sbrkr.o)
 .debug_str     0x00000000      0x5c7 /usr/lib/gcc/arm-none-eabi/7.3.1/../../../arm-none-eabi/lib/thumb/v6-m/libc.a(lib_a-sbrkr.o)
 .comment       0x00000000       0x58 /usr/lib/gcc/arm-none-eabi/7.3.1/../../../arm-none-eabi/lib/thumb/v6-m/libc.a(lib_a-sbrkr.o)
 .debug_frame   0x00000000       0x2c /usr/lib/gcc/arm-none-eabi/7.3.1/../../../arm-none-eabi/lib/thumb/v6-m/libc.a(lib_a-sbrkr.o)
 .ARM.attributes
                0x00000000       0x2c /usr/lib/gcc/arm-none-eabi/7.3.1/../../../arm-none-eabi/lib/thumb/v6-m/libc.a(lib_a-sbrkr.o)
 .data          0x00000000        0x0 /usr/lib/gcc/arm-none-eabi/7.3.1/../../../arm-none-eabi/lib/thumb/v6-m/libc.a(lib_a-signal.o)
 .bss           0x00000000        0x0 /usr/lib/gcc/arm-none-eabi/7.3.1/../../../arm-none-eabi/lib/thumb/v6-m/libc.a(lib_a-signal.o)
 .debug_info    0x00000000      0xc59 /usr/lib/gcc/arm-none-eabi/7.3.1/../../../arm-none-eabi/lib/thumb/v6-m/libc.a(lib_a-signal.o)
 .debug_abbrev  0x00000000      0x2ea /usr/lib/gcc/arm-none-eabi/7.3.1/../../../arm-none-eabi/lib/thumb/v6-m/libc.a(lib_a-signal.o)
 .debug_loc     0x00000000      0x479 /usr/lib/gcc/arm-none-eabi/7.3.1/../../../arm-none-eabi/lib/thumb/v6-m/libc.a(lib_a-signal.o)
 .debug_aranges
                0x00000000       0x20 /usr/lib/gcc/arm-none-eabi/7.3.1/../../../arm-none-eabi/lib/thumb/v6-m/libc.a(lib_a-signal.o)
 .debug_ranges  0x00000000       0x28 /usr/lib/gcc/arm-none-eabi/7.3.1/../../../arm-none-eabi/lib/thumb/v6-m/libc.a(lib_a-signal.o)
 .debug_line    0x00000000      0x1d7 /usr/lib/gcc/arm-none-eabi/7.3.1/../../../arm-none-eabi/lib/thumb/v6-m/libc.a(lib_a-signal.o)
 .debug_str     0x00000000      0x627 /usr/lib/gcc/arm-none-eabi/7.3.1/../../../arm-none-eabi/lib/thumb/v6-m/libc.a(lib_a-signal.o)
 .comment       0x00000000       0x58 /usr/lib/gcc/arm-none-eabi/7.3.1/../../../arm-none-eabi/lib/thumb/v6-m/libc.a(lib_a-signal.o)
 .debug_frame   0x00000000       0xf8 /usr/lib/gcc/arm-none-eabi/7.3.1/../../../arm-none-eabi/lib/thumb/v6-m/libc.a(lib_a-signal.o)
 .ARM.attributes
                0x00000000       0x2c /usr/lib/gcc/arm-none-eabi/7.3.1/../../../arm-none-eabi/lib/thumb/v6-m/libc.a(lib_a-signal.o)
 .data          0x00000000        0x0 /usr/lib/gcc/arm-none-eabi/7.3.1/../../../arm-none-eabi/lib/thumb/v6-m/libc.a(lib_a-signalr.o)
 .bss           0x00000000        0x0 /usr/lib/gcc/arm-none-eabi/7.3.1/../../../arm-none-eabi/lib/thumb/v6-m/libc.a(lib_a-signalr.o)
 .debug_info    0x00000000      0x99f /usr/lib/gcc/arm-none-eabi/7.3.1/../../../arm-none-eabi/lib/thumb/v6-m/libc.a(lib_a-signalr.o)
 .debug_abbrev  0x00000000      0x20d /usr/lib/gcc/arm-none-eabi/7.3.1/../../../arm-none-eabi/lib/thumb/v6-m/libc.a(lib_a-signalr.o)
 .debug_loc     0x00000000       0xa5 /usr/lib/gcc/arm-none-eabi/7.3.1/../../../arm-none-eabi/lib/thumb/v6-m/libc.a(lib_a-signalr.o)
 .debug_aranges
                0x00000000       0x20 /usr/lib/gcc/arm-none-eabi/7.3.1/../../../arm-none-eabi/lib/thumb/v6-m/libc.a(lib_a-signalr.o)
 .debug_line    0x00000000      0x145 /usr/lib/gcc/arm-none-eabi/7.3.1/../../../arm-none-eabi/lib/thumb/v6-m/libc.a(lib_a-signalr.o)
 .debug_str     0x00000000      0x5cc /usr/lib/gcc/arm-none-eabi/7.3.1/../../../arm-none-eabi/lib/thumb/v6-m/libc.a(lib_a-signalr.o)
 .comment       0x00000000       0x58 /usr/lib/gcc/arm-none-eabi/7.3.1/../../../arm-none-eabi/lib/thumb/v6-m/libc.a(lib_a-signalr.o)
 .debug_frame   0x00000000       0x44 /usr/lib/gcc/arm-none-eabi/7.3.1/../../../arm-none-eabi/lib/thumb/v6-m/libc.a(lib_a-signalr.o)
 .ARM.attributes
                0x00000000       0x2c /usr/lib/gcc/arm-none-eabi/7.3.1/../../../arm-none-eabi/lib/thumb/v6-m/libc.a(lib_a-signalr.o)
 .data          0x00000000        0x0 /usr/lib/gcc/arm-none-eabi/7.3.1/../../../arm-none-eabi/lib/thumb/v6-m/libc.a(lib_a-strcmp.o)
 .bss           0x00000000        0x0 /usr/lib/gcc/arm-none-eabi/7.3.1/../../../arm-none-eabi/lib/thumb/v6-m/libc.a(lib_a-strcmp.o)
 .data          0x00000000        0x0 /usr/lib/gcc/arm-none-eabi/7.3.1/../../../arm-none-eabi/lib/thumb/v6-m/libc.a(lib_a-strlen-stub.o)
 .bss           0x00000000        0x0 /usr/lib/gcc/arm-none-eabi/7.3.1/../../../arm-none-eabi/lib/thumb/v6-m/libc.a(lib_a-strlen-stub.o)
 .text          0x00000000       0x88 /usr/lib/gcc/arm-none-eabi/7.3.1/../../../arm-none-eabi/lib/thumb/v6-m/libc.a(lib_a-__atexit.o)
 .data          0x00000000        0x0 /usr/lib/gcc/arm-none-eabi/7.3.1/../../../arm-none-eabi/lib/thumb/v6-m/libc.a(lib_a-__atexit.o)
 .bss           0x00000000        0x0 /usr/lib/gcc/arm-none-eabi/7.3.1/../../../arm-none-eabi/lib/thumb/v6-m/libc.a(lib_a-__atexit.o)
 .debug_info    0x00000000      0x937 /usr/lib/gcc/arm-none-eabi/7.3.1/../../../arm-none-eabi/lib/thumb/v6-m/libc.a(lib_a-__atexit.o)
 .debug_abbrev  0x00000000      0x212 /usr/lib/gcc/arm-none-eabi/7.3.1/../../../arm-none-eabi/lib/thumb/v6-m/libc.a(lib_a-__atexit.o)
 .debug_loc     0x00000000      0x138 /usr/lib/gcc/arm-none-eabi/7.3.1/../../../arm-none-eabi/lib/thumb/v6-m/libc.a(lib_a-__atexit.o)
 .debug_aranges
                0x00000000       0x20 /usr/lib/gcc/arm-none-eabi/7.3.1/../../../arm-none-eabi/lib/thumb/v6-m/libc.a(lib_a-__atexit.o)
 .debug_line    0x00000000      0x148 /usr/lib/gcc/arm-none-eabi/7.3.1/../../../arm-none-eabi/lib/thumb/v6-m/libc.a(lib_a-__atexit.o)
 .debug_str     0x00000000      0x5ed /usr/lib/gcc/arm-none-eabi/7.3.1/../../../arm-none-eabi/lib/thumb/v6-m/libc.a(lib_a-__atexit.o)
 .comment       0x00000000       0x58 /usr/lib/gcc/arm-none-eabi/7.3.1/../../../arm-none-eabi/lib/thumb/v6-m/libc.a(lib_a-__atexit.o)
 .debug_frame   0x00000000       0x38 /usr/lib/gcc/arm-none-eabi/7.3.1/../../../arm-none-eabi/lib/thumb/v6-m/libc.a(lib_a-__atexit.o)
 .ARM.attributes
                0x00000000       0x2c /usr/lib/gcc/arm-none-eabi/7.3.1/../../../arm-none-eabi/lib/thumb/v6-m/libc.a(lib_a-__atexit.o)
 .data          0x00000000        0x0 /usr/lib/gcc/arm-none-eabi/7.3.1/../../../arm-none-eabi/lib/thumb/v6-m/libc.a(lib_a-freer.o)
 .bss           0x00000000        0x0 /usr/lib/gcc/arm-none-eabi/7.3.1/../../../arm-none-eabi/lib/thumb/v6-m/libc.a(lib_a-freer.o)
 .debug_info    0x00000000      0xc97 /usr/lib/gcc/arm-none-eabi/7.3.1/../../../arm-none-eabi/lib/thumb/v6-m/libc.a(lib_a-freer.o)
 .debug_abbrev  0x00000000      0x273 /usr/lib/gcc/arm-none-eabi/7.3.1/../../../arm-none-eabi/lib/thumb/v6-m/libc.a(lib_a-freer.o)
 .debug_loc     0x00000000      0x46c /usr/lib/gcc/arm-none-eabi/7.3.1/../../../arm-none-eabi/lib/thumb/v6-m/libc.a(lib_a-freer.o)
 .debug_aranges
                0x00000000       0x20 /usr/lib/gcc/arm-none-eabi/7.3.1/../../../arm-none-eabi/lib/thumb/v6-m/libc.a(lib_a-freer.o)
 .debug_line    0x00000000      0x200 /usr/lib/gcc/arm-none-eabi/7.3.1/../../../arm-none-eabi/lib/thumb/v6-m/libc.a(lib_a-freer.o)
 .debug_str     0x00000000      0x765 /usr/lib/gcc/arm-none-eabi/7.3.1/../../../arm-none-eabi/lib/thumb/v6-m/libc.a(lib_a-freer.o)
 .comment       0x00000000       0x58 /usr/lib/gcc/arm-none-eabi/7.3.1/../../../arm-none-eabi/lib/thumb/v6-m/libc.a(lib_a-freer.o)
 .debug_frame   0x00000000       0x58 /usr/lib/gcc/arm-none-eabi/7.3.1/../../../arm-none-eabi/lib/thumb/v6-m/libc.a(lib_a-freer.o)
 .ARM.attributes
                0x00000000       0x2c /usr/lib/gcc/arm-none-eabi/7.3.1/../../../arm-none-eabi/lib/thumb/v6-m/libc.a(lib_a-freer.o)
 .text          0x00000000       0xb0 /usr/lib/gcc/arm-none-eabi/7.3.1/../../../arm-none-eabi/lib/thumb/v6-m/libc.a(lib_a-reent.o)
 .data          0x00000000        0x0 /usr/lib/gcc/arm-none-eabi/7.3.1/../../../arm-none-eabi/lib/thumb/v6-m/libc.a(lib_a-reent.o)
 .bss           0x00000000        0x0 /usr/lib/gcc/arm-none-eabi/7.3.1/../../../arm-none-eabi/lib/thumb/v6-m/libc.a(lib_a-reent.o)
 .debug_info    0x00000000      0xa12 /usr/lib/gcc/arm-none-eabi/7.3.1/../../../arm-none-eabi/lib/thumb/v6-m/libc.a(lib_a-reent.o)
 .debug_abbrev  0x00000000      0x273 /usr/lib/gcc/arm-none-eabi/7.3.1/../../../arm-none-eabi/lib/thumb/v6-m/libc.a(lib_a-reent.o)
 .debug_loc     0x00000000      0x112 /usr/lib/gcc/arm-none-eabi/7.3.1/../../../arm-none-eabi/lib/thumb/v6-m/libc.a(lib_a-reent.o)
 .debug_aranges
                0x00000000       0x20 /usr/lib/gcc/arm-none-eabi/7.3.1/../../../arm-none-eabi/lib/thumb/v6-m/libc.a(lib_a-reent.o)
 .debug_line    0x00000000      0x14b /usr/lib/gcc/arm-none-eabi/7.3.1/../../../arm-none-eabi/lib/thumb/v6-m/libc.a(lib_a-reent.o)
 .debug_str     0x00000000      0x5c0 /usr/lib/gcc/arm-none-eabi/7.3.1/../../../arm-none-eabi/lib/thumb/v6-m/libc.a(lib_a-reent.o)
 .comment       0x00000000       0x58 /usr/lib/gcc/arm-none-eabi/7.3.1/../../../arm-none-eabi/lib/thumb/v6-m/libc.a(lib_a-reent.o)
 .debug_frame   0x00000000       0x48 /usr/lib/gcc/arm-none-eabi/7.3.1/../../../arm-none-eabi/lib/thumb/v6-m/libc.a(lib_a-reent.o)
 .ARM.attributes
                0x00000000       0x2c /usr/lib/gcc/arm-none-eabi/7.3.1/../../../arm-none-eabi/lib/thumb/v6-m/libc.a(lib_a-reent.o)
 .data          0x00000000        0x0 /usr/lib/gcc/arm-none-eabi/7.3.1/../../../arm-none-eabi/lib/thumb/v6-m/libnosys.a(getpid.o)
 .bss           0x00000000        0x0 /usr/lib/gcc/arm-none-eabi/7.3.1/../../../arm-none-eabi/lib/thumb/v6-m/libnosys.a(getpid.o)
 .stab          0x00000000       0x24 /usr/lib/gcc/arm-none-eabi/7.3.1/../../../arm-none-eabi/lib/thumb/v6-m/libnosys.a(getpid.o)
 .debug_info    0x00000000      0x8d5 /usr/lib/gcc/arm-none-eabi/7.3.1/../../../arm-none-eabi/lib/thumb/v6-m/libnosys.a(getpid.o)
 .debug_abbrev  0x00000000      0x1ae /usr/lib/gcc/arm-none-eabi/7.3.1/../../../arm-none-eabi/lib/thumb/v6-m/libnosys.a(getpid.o)
 .debug_aranges
                0x00000000       0x20 /usr/lib/gcc/arm-none-eabi/7.3.1/../../../arm-none-eabi/lib/thumb/v6-m/libnosys.a(getpid.o)
 .debug_line    0x00000000       0xf1 /usr/lib/gcc/arm-none-eabi/7.3.1/../../../arm-none-eabi/lib/thumb/v6-m/libnosys.a(getpid.o)
 .debug_str     0x00000000      0x580 /usr/lib/gcc/arm-none-eabi/7.3.1/../../../arm-none-eabi/lib/thumb/v6-m/libnosys.a(getpid.o)
 .comment       0x00000000       0x58 /usr/lib/gcc/arm-none-eabi/7.3.1/../../../arm-none-eabi/lib/thumb/v6-m/libnosys.a(getpid.o)
 .debug_frame   0x00000000       0x20 /usr/lib/gcc/arm-none-eabi/7.3.1/../../../arm-none-eabi/lib/thumb/v6-m/libnosys.a(getpid.o)
 .ARM.attributes
                0x00000000       0x2c /usr/lib/gcc/arm-none-eabi/7.3.1/../../../arm-none-eabi/lib/thumb/v6-m/libnosys.a(getpid.o)
 .data          0x00000000        0x0 /usr/lib/gcc/arm-none-eabi/7.3.1/../../../arm-none-eabi/lib/thumb/v6-m/libnosys.a(kill.o)
 .bss           0x00000000        0x0 /usr/lib/gcc/arm-none-eabi/7.3.1/../../../arm-none-eabi/lib/thumb/v6-m/libnosys.a(kill.o)
 .stab          0x00000000       0x18 /usr/lib/gcc/arm-none-eabi/7.3.1/../../../arm-none-eabi/lib/thumb/v6-m/libnosys.a(kill.o)
                                 0x24 (size before relaxing)
 .debug_info    0x00000000      0x8f2 /usr/lib/gcc/arm-none-eabi/7.3.1/../../../arm-none-eabi/lib/thumb/v6-m/libnosys.a(kill.o)
 .debug_abbrev  0x00000000      0x1cc /usr/lib/gcc/arm-none-eabi/7.3.1/../../../arm-none-eabi/lib/thumb/v6-m/libnosys.a(kill.o)
 .debug_loc     0x00000000       0x21 /usr/lib/gcc/arm-none-eabi/7.3.1/../../../arm-none-eabi/lib/thumb/v6-m/libnosys.a(kill.o)
 .debug_aranges
                0x00000000       0x20 /usr/lib/gcc/arm-none-eabi/7.3.1/../../../arm-none-eabi/lib/thumb/v6-m/libnosys.a(kill.o)
 .debug_line    0x00000000       0xef /usr/lib/gcc/arm-none-eabi/7.3.1/../../../arm-none-eabi/lib/thumb/v6-m/libnosys.a(kill.o)
 .debug_str     0x00000000      0x57c /usr/lib/gcc/arm-none-eabi/7.3.1/../../../arm-none-eabi/lib/thumb/v6-m/libnosys.a(kill.o)
 .comment       0x00000000       0x58 /usr/lib/gcc/arm-none-eabi/7.3.1/../../../arm-none-eabi/lib/thumb/v6-m/libnosys.a(kill.o)
 .debug_frame   0x00000000       0x20 /usr/lib/gcc/arm-none-eabi/7.3.1/../../../arm-none-eabi/lib/thumb/v6-m/libnosys.a(kill.o)
 .ARM.attributes
                0x00000000       0x2c /usr/lib/gcc/arm-none-eabi/7.3.1/../../../arm-none-eabi/lib/thumb/v6-m/libnosys.a(kill.o)
 .text          0x00000000        0x0 /usr/lib/gcc/arm-none-eabi/7.3.1/thumb/v6-m/crtend.o
 .data          0x00000000        0x0 /usr/lib/gcc/arm-none-eabi/7.3.1/thumb/v6-m/crtend.o
 .bss           0x00000000        0x0 /usr/lib/gcc/arm-none-eabi/7.3.1/thumb/v6-m/crtend.o
 .eh_frame      0x00000000        0x4 /usr/lib/gcc/arm-none-eabi/7.3.1/thumb/v6-m/crtend.o
 .text          0x00000000        0x0 /usr/lib/gcc/arm-none-eabi/7.3.1/thumb/v6-m/crtn.o
 .data          0x00000000        0x0 /usr/lib/gcc/arm-none-eabi/7.3.1/thumb/v6-m/crtn.o
 .bss           0x00000000        0x0 /usr/lib/gcc/arm-none-eabi/7.3.1/thumb/v6-m/crtn.o
 .init          0x00000000        0x8 /usr/lib/gcc/arm-none-eabi/7.3.1/thumb/v6-m/crtn.o
 .fini          0x00000000        0x8 /usr/lib/gcc/arm-none-eabi/7.3.1/thumb/v6-m/crtn.o
 .ARM.attributes
                0x00000000       0x1e /usr/lib/gcc/arm-none-eabi/7.3.1/thumb/v6-m/crtn.o

Memory Configuration

Name             Origin             Length             Attributes
FLASH            0x10000000         0x00200000         xr
RAM              0x20000000         0x00040000         xrw
SCRATCH_X        0x20040000         0x00001000         xrw
SCRATCH_Y        0x20041000         0x00001000         xrw
*default*        0x00000000         0xffffffff

Linker script and memory map

LOAD /usr/lib/gcc/arm-none-eabi/7.3.1/thumb/v6-m/crti.o
LOAD /usr/lib/gcc/arm-none-eabi/7.3.1/thumb/v6-m/crtbegin.o
LOAD /usr/lib/gcc/arm-none-eabi/7.3.1/../../../arm-none-eabi/lib/thumb/v6-m/crt0.o

.flash_begin    0x10000000        0x0
                0x10000000                __flash_binary_start = .

.boot2          0x10000000      0x100
                0x10000000                __boot2_start__ = .
 *(.boot2)
 .boot2         0x10000000      0x100 /tmp/ccWYemgR.o
                0x10000100                __boot2_end__ = .
                0x00000001                ASSERT (((__boot2_end__ - __boot2_start__) == 0x100), ERROR: Pico second stage bootloader must be 256 bytes in size)

.text           0x10000100    0x10db0
                0x10000100                __logical_binary_start = .
 *(.vectors)
 .vectors       0x10000100       0xd4 CMakeFiles/main.dir/__/pico-sdk/src/rp2_common/pico_standard_link/crt0.S.obj
                0x10000100                __vectors
                0x10000100                __VECTOR_TABLE
                0x100001c0                isr_invalid
                0x100001c0                __default_isrs_start
                0x100001c2                isr_nmi
                0x100001c4                isr_hardfault
                0x100001c6                isr_svcall
                0x100001c8                isr_pendsv
                0x100001ca                isr_systick
                0x100001cc                isr_irq30
                0x100001cc                __unhandled_user_irq
                0x100001cc                isr_irq13
                0x100001cc                isr_irq27
                0x100001cc                isr_irq31
                0x100001cc                isr_irq5
                0x100001cc                isr_irq11
                0x100001cc                isr_irq23
                0x100001cc                isr_irq18
                0x100001cc                isr_irq28
                0x100001cc                isr_irq19
                0x100001cc                isr_irq0
                0x100001cc                isr_irq6
                0x100001cc                isr_irq22
                0x100001cc                isr_irq17
                0x100001cc                isr_irq14
                0x100001cc                isr_irq2
                0x100001cc                isr_irq10
                0x100001cc                isr_irq8
                0x100001cc                isr_irq24
                0x100001cc                isr_irq1
                0x100001cc                isr_irq7
                0x100001cc                isr_irq21
                0x100001cc                isr_irq20
                0x100001cc                isr_irq15
                0x100001cc                isr_irq25
                0x100001cc                isr_irq4
                0x100001cc                isr_irq16
                0x100001cc                isr_irq29
                0x100001cc                isr_irq26
                0x100001cc                __default_isrs_end
                0x100001cc                isr_irq3
                0x100001cc                isr_irq12
                0x100001cc                isr_irq9
                0x100001d2                unhandled_user_irq_num_in_r0
 *(.binary_info_header)
 .binary_info_header
                0x100001d4       0x14 CMakeFiles/main.dir/__/pico-sdk/src/rp2_common/pico_standard_link/crt0.S.obj
                0x100001e8                __binary_info_header_end = .
 *(.reset)
 .reset         0x100001e8       0xa8 CMakeFiles/main.dir/__/pico-sdk/src/rp2_common/pico_standard_link/crt0.S.obj
                0x100001e8                _entry_point
                0x10000266                __get_current_exception
 .reset         0x10000290       0x30 CMakeFiles/main.dir/__/pico-sdk/src/rp2_common/pico_standard_link/binary_info.c.obj
 *(.init)
 .init          0x100002c0        0x4 /usr/lib/gcc/arm-none-eabi/7.3.1/thumb/v6-m/crti.o
                0x100002c0                _init
 *(EXCLUDE_FILE(*libm.a: *libc.a:*lib_a-mem*.o *libgcc.a:) .text*)
 .text          0x100002c4       0x98 /usr/lib/gcc/arm-none-eabi/7.3.1/thumb/v6-m/crtbegin.o
 .text._ZN12aprssettingsC2Ev
                0x1000035c       0x94 CMakeFiles/main.dir/main.cpp.obj
                0x1000035c                aprssettings::aprssettings()
                0x1000035c                aprssettings::aprssettings()
 .text._ZN6statusC2Ev
                0x100003f0       0x4c CMakeFiles/main.dir/main.cpp.obj
                0x100003f0                status::status()
                0x100003f0                status::status()
 .text._Z7log_outPKcz
                0x1000043c       0x38 CMakeFiles/main.dir/main.cpp.obj
                0x1000043c                log_out(char const*, ...)
 .text._Z12ShowSettingsv
                0x10000474      0x11c CMakeFiles/main.dir/main.cpp.obj
                0x10000474                ShowSettings()
 .text._Z5setupv
                0x10000590      0x1d8 CMakeFiles/main.dir/main.cpp.obj
                0x10000590                setup()
 .text._Z10print_helpv
                0x10000768       0x88 CMakeFiles/main.dir/main.cpp.obj
                0x10000768                print_help()
 .text._Z10startRadiov
                0x100007f0       0x78 CMakeFiles/main.dir/main.cpp.obj
                0x100007f0                startRadio()
 .text._Z18ProcessSerialInputPc.part.0
                0x10000868      0x684 CMakeFiles/main.dir/main.cpp.obj
 .text._Z16ComposeAprsFramePh
                0x10000eec      0x3d4 CMakeFiles/main.dir/main.cpp.obj
                0x10000eec                ComposeAprsFrame(unsigned char*)
 .text._Z13decode_packetv
                0x100012c0      0x4e4 CMakeFiles/main.dir/main.cpp.obj
                0x100012c0                decode_packet()
 .text._Z24ComposeAprsFrameFromKissv
                0x100017a4      0x2bc CMakeFiles/main.dir/main.cpp.obj
                0x100017a4                ComposeAprsFrameFromKiss()
 .text._Z13ReadUSBSerialv
                0x10001a60      0x190 CMakeFiles/main.dir/main.cpp.obj
                0x10001a60                ReadUSBSerial()
 .text.startup._GLOBAL__sub_I_lastRssi
                0x10001bf0       0x5c CMakeFiles/main.dir/main.cpp.obj
 .text.startup.main
                0x10001c4c     0x397c CMakeFiles/main.dir/main.cpp.obj
                0x10001c4c                main
 .text.gpio_set_function
                0x100055c8       0x30 CMakeFiles/main.dir/__/pico-sdk/src/rp2_common/hardware_gpio/gpio.c.obj
                0x100055c8                gpio_set_function
 .text.gpio_set_pulls
                0x100055f8       0x34 CMakeFiles/main.dir/__/pico-sdk/src/rp2_common/hardware_gpio/gpio.c.obj
                0x100055f8                gpio_set_pulls
 .text.gpio_init
                0x1000562c       0x3c CMakeFiles/main.dir/__/pico-sdk/src/rp2_common/hardware_gpio/gpio.c.obj
                0x1000562c                gpio_init
 .text.hw_claim_or_assert
                0x10005668       0x44 CMakeFiles/main.dir/__/pico-sdk/src/rp2_common/hardware_claim/claim.c.obj
                0x10005668                hw_claim_or_assert
 .text.hw_claim_unused_from_range
                0x100056ac       0x9c CMakeFiles/main.dir/__/pico-sdk/src/rp2_common/hardware_claim/claim.c.obj
                0x100056ac                hw_claim_unused_from_range
 .text.running_on_fpga
                0x10005748       0x10 CMakeFiles/main.dir/__/pico-sdk/src/rp2_common/pico_platform/platform.c.obj
                0x10005748                running_on_fpga
 .text.spin_locks_reset
                0x10005758       0x1c CMakeFiles/main.dir/__/pico-sdk/src/rp2_common/hardware_sync/sync.c.obj
                0x10005758                spin_locks_reset
 .text.next_striped_spin_lock_num
                0x10005774       0x18 CMakeFiles/main.dir/__/pico-sdk/src/rp2_common/hardware_sync/sync.c.obj
                0x10005774                next_striped_spin_lock_num
 .text.spin_lock_claim_unused
                0x1000578c       0x20 CMakeFiles/main.dir/__/pico-sdk/src/rp2_common/hardware_sync/sync.c.obj
                0x1000578c                spin_lock_claim_unused
 .text.timer_pool_entry_comparator
                0x100057ac       0x34 CMakeFiles/main.dir/__/pico-sdk/src/common/pico_time/time.c.obj
                0x100057ac                timer_pool_entry_comparator
 .text.sleep_until_callback
                0x100057e0       0x30 CMakeFiles/main.dir/__/pico-sdk/src/common/pico_time/time.c.obj
 .text.add_alarm_under_lock
                0x10005810      0x120 CMakeFiles/main.dir/__/pico-sdk/src/common/pico_time/time.c.obj
 .text.alarm_pool_alarm_callback
                0x10005930      0x1dc CMakeFiles/main.dir/__/pico-sdk/src/common/pico_time/time.c.obj
 .text.alarm_pool_init_default
                0x10005b0c       0x64 CMakeFiles/main.dir/__/pico-sdk/src/common/pico_time/time.c.obj
                0x10005b0c                alarm_pool_init_default
 .text.alarm_pool_get_default
                0x10005b70        0x8 CMakeFiles/main.dir/__/pico-sdk/src/common/pico_time/time.c.obj
                0x10005b70                alarm_pool_get_default
 .text.alarm_pool_add_alarm_at
                0x10005b78      0x1ac CMakeFiles/main.dir/__/pico-sdk/src/common/pico_time/time.c.obj
                0x10005b78                alarm_pool_add_alarm_at
 .text.sleep_until
                0x10005d24      0x1ec CMakeFiles/main.dir/__/pico-sdk/src/common/pico_time/time.c.obj
                0x10005d24                sleep_until
 .text.sleep_ms
                0x10005f10       0x38 CMakeFiles/main.dir/__/pico-sdk/src/common/pico_time/time.c.obj
                0x10005f10                sleep_ms
 .text.best_effort_wfe_or_timeout
                0x10005f48      0x1b4 CMakeFiles/main.dir/__/pico-sdk/src/common/pico_time/time.c.obj
                0x10005f48                best_effort_wfe_or_timeout
 .text.check_single_timeout_us
                0x100060fc       0x28 CMakeFiles/main.dir/__/pico-sdk/src/common/pico_time/timeout_helper.c.obj
 .text.init_single_timeout_until
                0x10006124        0xc CMakeFiles/main.dir/__/pico-sdk/src/common/pico_time/timeout_helper.c.obj
                0x10006124                init_single_timeout_until
 .text.hardware_alarm_irq_handler
                0x10006130       0xb0 CMakeFiles/main.dir/__/pico-sdk/src/rp2_common/hardware_timer/timer.c.obj
 .text.hardware_alarm_claim
                0x100061e0       0x18 CMakeFiles/main.dir/__/pico-sdk/src/rp2_common/hardware_timer/timer.c.obj
                0x100061e0                hardware_alarm_claim
 .text.time_us_64
                0x100061f8       0x18 CMakeFiles/main.dir/__/pico-sdk/src/rp2_common/hardware_timer/timer.c.obj
                0x100061f8                time_us_64
 .text.busy_wait_us
                0x10006210       0x60 CMakeFiles/main.dir/__/pico-sdk/src/rp2_common/hardware_timer/timer.c.obj
                0x10006210                busy_wait_us
 .text.busy_wait_until
                0x10006270       0x20 CMakeFiles/main.dir/__/pico-sdk/src/rp2_common/hardware_timer/timer.c.obj
                0x10006270                busy_wait_until
 .text.hardware_alarm_set_callback
                0x10006290       0x8c CMakeFiles/main.dir/__/pico-sdk/src/rp2_common/hardware_timer/timer.c.obj
                0x10006290                hardware_alarm_set_callback
 .text.hardware_alarm_set_target
                0x1000631c       0xd8 CMakeFiles/main.dir/__/pico-sdk/src/rp2_common/hardware_timer/timer.c.obj
                0x1000631c                hardware_alarm_set_target
 .text.hardware_alarm_cancel
                0x100063f4       0x40 CMakeFiles/main.dir/__/pico-sdk/src/rp2_common/hardware_timer/timer.c.obj
                0x100063f4                hardware_alarm_cancel
 .text.lock_init
                0x10006434       0x10 CMakeFiles/main.dir/__/pico-sdk/src/common/pico_sync/lock_core.c.obj
                0x10006434                lock_init
 .text.mutex_init
                0x10006444       0x1c CMakeFiles/main.dir/__/pico-sdk/src/common/pico_sync/mutex.c.obj
                0x10006444                mutex_init
 .text.recursive_mutex_init
                0x10006460       0x1c CMakeFiles/main.dir/__/pico-sdk/src/common/pico_sync/mutex.c.obj
                0x10006460                recursive_mutex_init
 .text.critical_section_init
                0x1000647c       0x20 CMakeFiles/main.dir/__/pico-sdk/src/common/pico_sync/critical_section.c.obj
                0x1000647c                critical_section_init
 .text.ph_merge_two_pass.part.3
                0x1000649c       0xcc CMakeFiles/main.dir/__/pico-sdk/src/common/pico_util/pheap.c.obj
 .text.ph_post_alloc_init
                0x10006568       0x3c CMakeFiles/main.dir/__/pico-sdk/src/common/pico_util/pheap.c.obj
                0x10006568                ph_post_alloc_init
 .text.ph_remove_head
                0x100065a4      0x158 CMakeFiles/main.dir/__/pico-sdk/src/common/pico_util/pheap.c.obj
                0x100065a4                ph_remove_head
 .text.ph_remove_and_free_node
                0x100066fc      0x340 CMakeFiles/main.dir/__/pico-sdk/src/common/pico_util/pheap.c.obj
                0x100066fc                ph_remove_and_free_node
 .text.runtime_init
                0x10006a3c       0xf4 CMakeFiles/main.dir/__/pico-sdk/src/rp2_common/pico_runtime/runtime.c.obj
                0x10006a3c                runtime_init
 .text._exit    0x10006b30        0x4 CMakeFiles/main.dir/__/pico-sdk/src/rp2_common/pico_runtime/runtime.c.obj
                0x10006b30                _exit
 .text._sbrk    0x10006b34       0x34 CMakeFiles/main.dir/__/pico-sdk/src/rp2_common/pico_runtime/runtime.c.obj
                0x10006b34                _sbrk
 .text.exit     0x10006b68        0x4 CMakeFiles/main.dir/__/pico-sdk/src/rp2_common/pico_runtime/runtime.c.obj
                0x10006b68                exit
 .text.panic    0x10006b6c       0x30 CMakeFiles/main.dir/__/pico-sdk/src/rp2_common/pico_runtime/runtime.c.obj
                0x10006b6c                panic
 .text.hard_assertion_failure
                0x10006b9c        0xc CMakeFiles/main.dir/__/pico-sdk/src/rp2_common/pico_runtime/runtime.c.obj
                0x10006b9c                hard_assertion_failure
 .text.clocks_init
                0x10006ba8      0x2c8 CMakeFiles/main.dir/__/pico-sdk/src/rp2_common/hardware_clocks/clocks.c.obj
                0x10006ba8                clocks_init
 .text.clock_get_hz
                0x10006e70        0xc CMakeFiles/main.dir/__/pico-sdk/src/rp2_common/hardware_clocks/clocks.c.obj
                0x10006e70                clock_get_hz
 .text.irq_set_enabled
                0x10006e7c       0x24 CMakeFiles/main.dir/__/pico-sdk/src/rp2_common/hardware_irq/irq.c.obj
                0x10006e7c                irq_set_enabled
 .text.irq_set_pending
                0x10006ea0       0x10 CMakeFiles/main.dir/__/pico-sdk/src/rp2_common/hardware_irq/irq.c.obj
                0x10006ea0                irq_set_pending
 .text.irq_get_vtable_handler
                0x10006eb0       0x10 CMakeFiles/main.dir/__/pico-sdk/src/rp2_common/hardware_irq/irq.c.obj
                0x10006eb0                irq_get_vtable_handler
 .text.irq_set_exclusive_handler
                0x10006ec0       0x54 CMakeFiles/main.dir/__/pico-sdk/src/rp2_common/hardware_irq/irq.c.obj
                0x10006ec0                irq_set_exclusive_handler
 .text.irq_remove_handler
                0x10006f14      0x1c0 CMakeFiles/main.dir/__/pico-sdk/src/rp2_common/hardware_irq/irq.c.obj
                0x10006f14                irq_remove_handler
 .text.irq_add_tail_to_free_list
                0x100070d4       0xb4 CMakeFiles/main.dir/__/pico-sdk/src/rp2_common/hardware_irq/irq.c.obj
                0x100070d4                irq_add_tail_to_free_list
 .text.irq_init_priorities
                0x10007188       0x24 CMakeFiles/main.dir/__/pico-sdk/src/rp2_common/hardware_irq/irq.c.obj
                0x10007188                irq_init_priorities
 .text.pll_init
                0x100071ac       0xa4 CMakeFiles/main.dir/__/pico-sdk/src/rp2_common/hardware_pll/pll.c.obj
                0x100071ac                pll_init
 .text.watchdog_start_tick
                0x10007250       0x10 CMakeFiles/main.dir/__/pico-sdk/src/rp2_common/hardware_watchdog/watchdog.c.obj
                0x10007250                watchdog_start_tick
 .text.watchdog_reboot
                0x10007260       0x98 CMakeFiles/main.dir/__/pico-sdk/src/rp2_common/hardware_watchdog/watchdog.c.obj
                0x10007260                watchdog_reboot
 .text.xosc_init
                0x100072f8       0x28 CMakeFiles/main.dir/__/pico-sdk/src/rp2_common/hardware_xosc/xosc.c.obj
                0x100072f8                xosc_init
 .text._out_buffer
                0x10007320        0x8 CMakeFiles/main.dir/__/pico-sdk/src/rp2_common/pico_printf/printf.c.obj
 .text._out_null
                0x10007328        0x4 CMakeFiles/main.dir/__/pico-sdk/src/rp2_common/pico_printf/printf.c.obj
 .text._out_fct
                0x1000732c       0x10 CMakeFiles/main.dir/__/pico-sdk/src/rp2_common/pico_printf/printf.c.obj
 .text._out_char
                0x1000733c        0xc CMakeFiles/main.dir/__/pico-sdk/src/rp2_common/pico_printf/printf.c.obj
 .text._ntoa_format
                0x10007348      0x270 CMakeFiles/main.dir/__/pico-sdk/src/rp2_common/pico_printf/printf.c.obj
 .text._etoa.part.0
                0x100075b8      0x56c CMakeFiles/main.dir/__/pico-sdk/src/rp2_common/pico_printf/printf.c.obj
 .text._ftoa    0x10007b24      0x6f8 CMakeFiles/main.dir/__/pico-sdk/src/rp2_common/pico_printf/printf.c.obj
 .text._ftoa.part.1
                0x1000821c      0x54c CMakeFiles/main.dir/__/pico-sdk/src/rp2_common/pico_printf/printf.c.obj
 .text._vsnprintf
                0x10008768     0x11e0 CMakeFiles/main.dir/__/pico-sdk/src/rp2_common/pico_printf/printf.c.obj
 .text.__wrap_sprintf
                0x10009948       0x28 CMakeFiles/main.dir/__/pico-sdk/src/rp2_common/pico_printf/printf.c.obj
                0x10009948                __wrap_sprintf
 .text.__wrap_vsnprintf
                0x10009970       0x1c CMakeFiles/main.dir/__/pico-sdk/src/rp2_common/pico_printf/printf.c.obj
                0x10009970                __wrap_vsnprintf
 .text.vfctprintf
                0x1000998c       0x20 CMakeFiles/main.dir/__/pico-sdk/src/rp2_common/pico_printf/printf.c.obj
                0x1000998c                vfctprintf
 .text.weak_raw_vprintf
                0x100099ac       0x30 CMakeFiles/main.dir/__/pico-sdk/src/rp2_common/pico_printf/printf.c.obj
                0x100099ac                weak_raw_vprintf
 .text          0x100099dc       0x10 CMakeFiles/main.dir/__/pico-sdk/src/rp2_common/pico_bit_ops/bit_ops_aeabi.S.obj
 .text.rom_func_lookup
                0x100099ec       0x10 CMakeFiles/main.dir/__/pico-sdk/src/rp2_common/pico_bootrom/bootrom.c.obj
                0x100099ec                rom_func_lookup
 .text.rom_data_lookup
                0x100099fc       0x10 CMakeFiles/main.dir/__/pico-sdk/src/rp2_common/pico_bootrom/bootrom.c.obj
                0x100099fc                rom_data_lookup
 .text.rom_funcs_lookup
                0x10009a0c       0x3c CMakeFiles/main.dir/__/pico-sdk/src/rp2_common/pico_bootrom/bootrom.c.obj
                0x10009a0c                rom_funcs_lookup
 .text.__wrap___aeabi_idiv
                0x10009a48       0x50 CMakeFiles/main.dir/__/pico-sdk/src/rp2_common/pico_divider/divider.S.obj
                0x10009a48                __wrap___aeabi_idivmod
                0x10009a48                divmod_s32s32
                0x10009a48                div_s32s32
                0x10009a48                __wrap___aeabi_idiv
                0x10009a50                divmod_s32s32_unsafe
                0x10009a7c                divmod_s32s32_savestate
 .text.__wrap___aeabi_uidiv
                0x10009a98       0x4c CMakeFiles/main.dir/__/pico-sdk/src/rp2_common/pico_divider/divider.S.obj
                0x10009a98                __wrap___aeabi_uidiv
                0x10009a98                __wrap___aeabi_uidivmod
                0x10009a98                div_u32u32
                0x10009a98                divmod_u32u32
                0x10009aa0                divmod_u32u32_unsafe
                0x10009ac8                divmod_u32u32_savestate
 .text.__wrap___aeabi_ldiv
                0x10009ae4      0x434 CMakeFiles/main.dir/__/pico-sdk/src/rp2_common/pico_divider/divider.S.obj
                0x10009ae4                div_s64s64
                0x10009ae4                divmod_s64s64
                0x10009ae4                __wrap___aeabi_ldivmod
                0x10009b1c                div_u64u64
                0x10009b1c                divmod_u64u64
                0x10009b1c                __wrap___aeabi_uldivmod
                0x10009b2c                divmod_u64u64_savestate
                0x10009b54                divmod_s64s64_unsafe
                0x10009bdc                divmod_u64u64_unsafe
 .text.__wrap___aeabi_darithmetic
                0x10009f18       0x80 CMakeFiles/main.dir/__/pico-sdk/src/rp2_common/pico_double/double_aeabi.S.obj
                0x10009f18                __wrap___aeabi_drsub
                0x10009f1e                __wrap___aeabi_dsub
                0x10009f30                __wrap___aeabi_dadd
                0x10009f42                __wrap___aeabi_ddiv
                0x10009f7e                __wrap___aeabi_dmul
 .text.__wrap___aeabi_cdcmple
                0x10009f98       0x6c CMakeFiles/main.dir/__/pico-sdk/src/rp2_common/pico_double/double_aeabi.S.obj
                0x10009f98                __wrap___aeabi_cdrcmple
                0x10009fa8                __wrap___aeabi_cdcmple
                0x10009fa8                __wrap___aeabi_cdcmpeq
 .text.__wrap___aeabi_dcmplt
                0x1000a004        0xc CMakeFiles/main.dir/__/pico-sdk/src/rp2_common/pico_double/double_aeabi.S.obj
                0x1000a004                __wrap___aeabi_dcmplt
 .text.__wrap___aeabi_dcmple
                0x1000a010       0x10 CMakeFiles/main.dir/__/pico-sdk/src/rp2_common/pico_double/double_aeabi.S.obj
                0x1000a010                __wrap___aeabi_dcmple
 .text.__wrap___aeabi_dcmpge
                0x1000a020       0x10 CMakeFiles/main.dir/__/pico-sdk/src/rp2_common/pico_double/double_aeabi.S.obj
                0x1000a020                __wrap___aeabi_dcmpge
 .text.__wrap___aeabi_dcmpgt
                0x1000a030        0xa CMakeFiles/main.dir/__/pico-sdk/src/rp2_common/pico_double/double_aeabi.S.obj
                0x1000a030                __wrap___aeabi_dcmpgt
 .text.__wrap___aeabi_dcmpun
                0x1000a03a       0x1c CMakeFiles/main.dir/__/pico-sdk/src/rp2_common/pico_double/double_aeabi.S.obj
                0x1000a03a                __wrap___aeabi_dcmpun
 *fill*         0x1000a056        0x2 
 .text.__wrap___aeabi_i2d
                0x1000a058       0x38 CMakeFiles/main.dir/__/pico-sdk/src/rp2_common/pico_double/double_aeabi.S.obj
                0x1000a058                __wrap___aeabi_ui2d
                0x1000a060                __wrap___aeabi_i2d
 .text.__wrap___aeabi_d2iz
                0x1000a090       0x48 CMakeFiles/main.dir/__/pico-sdk/src/rp2_common/pico_double/double_aeabi.S.obj
                0x1000a090                __wrap___aeabi_d2iz
                0x1000a090                double2int_z
 .text.__wrap___aeabi_d2uiz
                0x1000a0d8       0x18 CMakeFiles/main.dir/__/pico-sdk/src/rp2_common/pico_double/double_aeabi.S.obj
                0x1000a0d8                double2uint
                0x1000a0d8                __wrap___aeabi_d2uiz
 .text.__wrap___aeabi_d2ulz
                0x1000a0f0       0x18 CMakeFiles/main.dir/__/pico-sdk/src/rp2_common/pico_double/double_aeabi.S.obj
                0x1000a0f0                __wrap___aeabi_d2ulz
 .text.__aeabi_double_init
                0x1000a108       0x60 CMakeFiles/main.dir/__/pico-sdk/src/rp2_common/pico_double/double_init_rom.c.obj
                0x1000a108                __aeabi_double_init
 .text.double_table_shim_on_use_helper
                0x1000a168       0x2c CMakeFiles/main.dir/__/pico-sdk/src/rp2_common/pico_double/double_v1_rom_shim.S.obj
                0x1000a168                double_table_shim_on_use_helper
 .text.__wrap___aeabi_dsub
                0x1000a194       0x10 CMakeFiles/main.dir/__/pico-sdk/src/rp2_common/pico_double/double_v1_rom_shim.S.obj
                0x1000a194                drsub_shim
                0x1000a19a                dsub_shim
 .text.dadd_shim
                0x1000a1a4      0x15c CMakeFiles/main.dir/__/pico-sdk/src/rp2_common/pico_double/double_v1_rom_shim.S.obj
                0x1000a1a4                dadd_shim
 .text.dmul_shim
                0x1000a300      0x15c CMakeFiles/main.dir/__/pico-sdk/src/rp2_common/pico_double/double_v1_rom_shim.S.obj
                0x1000a300                dmul_shim
 .text.ddiv_shim
                0x1000a45c      0x1b0 CMakeFiles/main.dir/__/pico-sdk/src/rp2_common/pico_double/double_v1_rom_shim.S.obj
                0x1000a45c                ddiv_shim
 .text.double2uint_shim
                0x1000a60c        0xe CMakeFiles/main.dir/__/pico-sdk/src/rp2_common/pico_double/double_v1_rom_shim.S.obj
                0x1000a60c                double2uint_shim
                0x1000a60e                double2ufix_shim
 *fill*         0x1000a61a        0x2 
 .text.double2uint64_shim
                0x1000a61c       0x70 CMakeFiles/main.dir/__/pico-sdk/src/rp2_common/pico_double/double_v1_rom_shim.S.obj
                0x1000a61c                double2uint64_shim
                0x1000a61e                double2ufix64_shim
                0x1000a63e                d2fix_a
 .text.dunpacks
                0x1000a68c       0x3c CMakeFiles/main.dir/__/pico-sdk/src/rp2_common/pico_double/double_v1_rom_shim.S.obj
                0x1000a68c                dunpacks
 .text.__aeabi_lmul
                0x1000a6c8       0x32 CMakeFiles/main.dir/__/pico-sdk/src/rp2_common/pico_int64_ops/pico_int64_ops_aeabi.S.obj
                0x1000a6c8                __wrap___aeabi_lmul
 *fill*         0x1000a6fa        0x2 
 .text.__wrap___aeabi_farithmetic
                0x1000a6fc       0x48 CMakeFiles/main.dir/__/pico-sdk/src/rp2_common/pico_float/float_aeabi.S.obj
                0x1000a6fc                __wrap___aeabi_frsub
                0x1000a702                __wrap___aeabi_fsub
                0x1000a708                __wrap___aeabi_fadd
                0x1000a70e                __wrap___aeabi_fdiv
                0x1000a736                __wrap___aeabi_fmul
 .text.__wrap___aeabi_i2f
                0x1000a744       0x44 CMakeFiles/main.dir/__/pico-sdk/src/rp2_common/pico_float/float_aeabi.S.obj
                0x1000a744                __wrap___aeabi_i2f
 .text.__wrap___aeabi_f2d
                0x1000a788       0x14 CMakeFiles/main.dir/__/pico-sdk/src/rp2_common/pico_float/float_aeabi.S.obj
                0x1000a788                __wrap___aeabi_f2d
 .text.__aeabi_float_init
                0x1000a79c       0x68 CMakeFiles/main.dir/__/pico-sdk/src/rp2_common/pico_float/float_init_rom.c.obj
                0x1000a79c                __aeabi_float_init
 .text.float_table_shim_on_use_helper
                0x1000a804       0x2c CMakeFiles/main.dir/__/pico-sdk/src/rp2_common/pico_float/float_v1_rom_shim.S.obj
                0x1000a804                float_table_shim_on_use_helper
 .text.float2double_shim
                0x1000a830       0x30 CMakeFiles/main.dir/__/pico-sdk/src/rp2_common/pico_float/float_v1_rom_shim.S.obj
                0x1000a830                float2double_shim
 .text          0x1000a860       0x10 CMakeFiles/main.dir/__/pico-sdk/src/rp2_common/pico_mem_ops/mem_ops_aeabi.S.obj
                0x1000a860                __aeabi_mem_init
 .text.memset   0x1000a870        0xc CMakeFiles/main.dir/__/pico-sdk/src/rp2_common/pico_mem_ops/mem_ops_aeabi.S.obj
                0x1000a870                __wrap_memset
 .text.memcpy   0x1000a87c        0xc CMakeFiles/main.dir/__/pico-sdk/src/rp2_common/pico_mem_ops/mem_ops_aeabi.S.obj
                0x1000a87c                __wrap___aeabi_memcpy
                0x1000a87c                __wrap_memcpy
 .text.stdio_out_chars_crlf
                0x1000a888       0x9c CMakeFiles/main.dir/__/pico-sdk/src/rp2_common/pico_stdio/stdio.c.obj
 .text.stdio_stack_buffer_flush.part.1
                0x1000a924       0xdc CMakeFiles/main.dir/__/pico-sdk/src/rp2_common/pico_stdio/stdio.c.obj
 .text.stdio_buffered_printer
                0x1000aa00       0x20 CMakeFiles/main.dir/__/pico-sdk/src/rp2_common/pico_stdio/stdio.c.obj
 .text.__wrap_putchar
                0x1000aa20       0xa0 CMakeFiles/main.dir/__/pico-sdk/src/rp2_common/pico_stdio/stdio.c.obj
                0x1000aa20                __wrap_putchar
 .text.__wrap_puts
                0x1000aac0       0xe8 CMakeFiles/main.dir/__/pico-sdk/src/rp2_common/pico_stdio/stdio.c.obj
                0x1000aac0                __wrap_puts
 .text.stdio_set_driver_enabled
                0x1000aba8       0x3c CMakeFiles/main.dir/__/pico-sdk/src/rp2_common/pico_stdio/stdio.c.obj
                0x1000aba8                stdio_set_driver_enabled
 .text.__wrap_vprintf
                0x1000abe4       0x94 CMakeFiles/main.dir/__/pico-sdk/src/rp2_common/pico_stdio/stdio.c.obj
                0x1000abe4                __wrap_vprintf
 .text.__wrap_printf
                0x1000ac78       0x18 CMakeFiles/main.dir/__/pico-sdk/src/rp2_common/pico_stdio/stdio.c.obj
                0x1000ac78                __wrap_printf
 .text.stdio_init_all
                0x1000ac90        0x8 CMakeFiles/main.dir/__/pico-sdk/src/rp2_common/pico_stdio/stdio.c.obj
                0x1000ac90                stdio_init_all
 .text.getchar_timeout_us
                0x1000ac98       0xa4 CMakeFiles/main.dir/__/pico-sdk/src/rp2_common/pico_stdio/stdio.c.obj
                0x1000ac98                getchar_timeout_us
 .text.stdio_set_translate_crlf
                0x1000ad3c       0x10 CMakeFiles/main.dir/__/pico-sdk/src/rp2_common/pico_stdio/stdio.c.obj
                0x1000ad3c                stdio_set_translate_crlf
 .text.resetd_init
                0x1000ad4c        0x4 CMakeFiles/main.dir/__/pico-sdk/src/rp2_common/pico_stdio_usb/reset_interface.c.obj
 .text.resetd_reset
                0x1000ad50        0xc CMakeFiles/main.dir/__/pico-sdk/src/rp2_common/pico_stdio_usb/reset_interface.c.obj
 .text.resetd_xfer_cb
                0x1000ad5c        0x4 CMakeFiles/main.dir/__/pico-sdk/src/rp2_common/pico_stdio_usb/reset_interface.c.obj
 .text.resetd_open
                0x1000ad60       0x28 CMakeFiles/main.dir/__/pico-sdk/src/rp2_common/pico_stdio_usb/reset_interface.c.obj
 .text.resetd_control_xfer_cb
                0x1000ad88       0x64 CMakeFiles/main.dir/__/pico-sdk/src/rp2_common/pico_stdio_usb/reset_interface.c.obj
 .text.usbd_app_driver_get_cb
                0x1000adec        0xc CMakeFiles/main.dir/__/pico-sdk/src/rp2_common/pico_stdio_usb/reset_interface.c.obj
                0x1000adec                usbd_app_driver_get_cb
 .text.tud_cdc_line_coding_cb
                0x1000adf8       0x34 CMakeFiles/main.dir/__/pico-sdk/src/rp2_common/pico_stdio_usb/reset_interface.c.obj
                0x1000adf8                tud_cdc_line_coding_cb
 .text.stdio_usb_in_chars
                0x1000ae2c       0x68 CMakeFiles/main.dir/__/pico-sdk/src/rp2_common/pico_stdio_usb/stdio_usb.c.obj
                0x1000ae2c                stdio_usb_in_chars
 .text.timer_task
                0x1000ae94       0x10 CMakeFiles/main.dir/__/pico-sdk/src/rp2_common/pico_stdio_usb/stdio_usb.c.obj
 .text.low_priority_worker_irq
                0x1000aea4       0x20 CMakeFiles/main.dir/__/pico-sdk/src/rp2_common/pico_stdio_usb/stdio_usb.c.obj
 .text.stdio_usb_out_chars
                0x1000aec4       0xf0 CMakeFiles/main.dir/__/pico-sdk/src/rp2_common/pico_stdio_usb/stdio_usb.c.obj
 .text.stdio_usb_init
                0x1000afb4       0x8c CMakeFiles/main.dir/__/pico-sdk/src/rp2_common/pico_stdio_usb/stdio_usb.c.obj
                0x1000afb4                stdio_usb_init
 .text.tud_descriptor_device_cb
                0x1000b040        0x8 CMakeFiles/main.dir/__/pico-sdk/src/rp2_common/pico_stdio_usb/stdio_usb_descriptors.c.obj
                0x1000b040                tud_descriptor_device_cb
 .text.tud_descriptor_configuration_cb
                0x1000b048        0x8 CMakeFiles/main.dir/__/pico-sdk/src/rp2_common/pico_stdio_usb/stdio_usb_descriptors.c.obj
                0x1000b048                tud_descriptor_configuration_cb
 .text.tud_descriptor_string_cb
                0x1000b050       0x70 CMakeFiles/main.dir/__/pico-sdk/src/rp2_common/pico_stdio_usb/stdio_usb_descriptors.c.obj
                0x1000b050                tud_descriptor_string_cb
 .text.dcd_rp2040_irq
                0x1000b0c0      0x21c CMakeFiles/main.dir/__/pico-sdk/lib/tinyusb/src/portable/raspberrypi/rp2040/dcd_rp2040.c.obj
 .text.dcd_int_enable
                0x1000b2dc        0xc CMakeFiles/main.dir/__/pico-sdk/lib/tinyusb/src/portable/raspberrypi/rp2040/dcd_rp2040.c.obj
                0x1000b2dc                dcd_int_enable
 .text.dcd_set_address
                0x1000b2e8       0x14 CMakeFiles/main.dir/__/pico-sdk/lib/tinyusb/src/portable/raspberrypi/rp2040/dcd_rp2040.c.obj
                0x1000b2e8                dcd_set_address
 .text.dcd_connect
                0x1000b2fc       0x10 CMakeFiles/main.dir/__/pico-sdk/lib/tinyusb/src/portable/raspberrypi/rp2040/dcd_rp2040.c.obj
                0x1000b2fc                dcd_connect
 .text.dcd_init
                0x1000b30c      0x144 CMakeFiles/main.dir/__/pico-sdk/lib/tinyusb/src/portable/raspberrypi/rp2040/dcd_rp2040.c.obj
                0x1000b30c                dcd_init
 .text.dcd_edpt0_status_complete
                0x1000b450       0x1c CMakeFiles/main.dir/__/pico-sdk/lib/tinyusb/src/portable/raspberrypi/rp2040/dcd_rp2040.c.obj
                0x1000b450                dcd_edpt0_status_complete
 .text.dcd_edpt_open
                0x1000b46c       0xf0 CMakeFiles/main.dir/__/pico-sdk/lib/tinyusb/src/portable/raspberrypi/rp2040/dcd_rp2040.c.obj
                0x1000b46c                dcd_edpt_open
 .text.dcd_edpt_close_all
                0x1000b55c       0xbc CMakeFiles/main.dir/__/pico-sdk/lib/tinyusb/src/portable/raspberrypi/rp2040/dcd_rp2040.c.obj
                0x1000b55c                dcd_edpt_close_all
 .text.dcd_edpt_xfer
                0x1000b618       0x24 CMakeFiles/main.dir/__/pico-sdk/lib/tinyusb/src/portable/raspberrypi/rp2040/dcd_rp2040.c.obj
                0x1000b618                dcd_edpt_xfer
 .text.dcd_edpt_stall
                0x1000b63c       0x34 CMakeFiles/main.dir/__/pico-sdk/lib/tinyusb/src/portable/raspberrypi/rp2040/dcd_rp2040.c.obj
                0x1000b63c                dcd_edpt_stall
 .text.dcd_edpt_clear_stall
                0x1000b670       0x2c CMakeFiles/main.dir/__/pico-sdk/lib/tinyusb/src/portable/raspberrypi/rp2040/dcd_rp2040.c.obj
                0x1000b670                dcd_edpt_clear_stall
 .text.rp2040_usb_init
                0x1000b69c       0x4c CMakeFiles/main.dir/__/pico-sdk/lib/tinyusb/src/portable/raspberrypi/rp2040/rp2040_usb.c.obj
                0x1000b69c                rp2040_usb_init
 .text.hw_endpoint_reset_transfer
                0x1000b6e8        0xc CMakeFiles/main.dir/__/pico-sdk/lib/tinyusb/src/portable/raspberrypi/rp2040/rp2040_usb.c.obj
                0x1000b6e8                hw_endpoint_reset_transfer
 .text._hw_endpoint_buffer_control_update32
                0x1000b6f4       0x58 CMakeFiles/main.dir/__/pico-sdk/lib/tinyusb/src/portable/raspberrypi/rp2040/rp2040_usb.c.obj
                0x1000b6f4                _hw_endpoint_buffer_control_update32
 .text.hw_endpoint_xfer_start
                0x1000b74c      0x14c CMakeFiles/main.dir/__/pico-sdk/lib/tinyusb/src/portable/raspberrypi/rp2040/rp2040_usb.c.obj
                0x1000b74c                hw_endpoint_xfer_start
 .text.hw_endpoint_xfer_continue
                0x1000b898      0x200 CMakeFiles/main.dir/__/pico-sdk/lib/tinyusb/src/portable/raspberrypi/rp2040/rp2040_usb.c.obj
                0x1000b898                hw_endpoint_xfer_continue
 .text.tud_mounted
                0x1000ba98       0x10 CMakeFiles/main.dir/__/pico-sdk/lib/tinyusb/src/device/usbd.c.obj
                0x1000ba98                tud_mounted
 .text.tud_suspended
                0x1000baa8       0x10 CMakeFiles/main.dir/__/pico-sdk/lib/tinyusb/src/device/usbd.c.obj
                0x1000baa8                tud_suspended
 .text.tud_inited
                0x1000bab8        0xc CMakeFiles/main.dir/__/pico-sdk/lib/tinyusb/src/device/usbd.c.obj
                0x1000bab8                tud_inited
 .text.tud_init
                0x1000bac4       0xdc CMakeFiles/main.dir/__/pico-sdk/lib/tinyusb/src/device/usbd.c.obj
                0x1000bac4                tud_init
 .text.tud_task
                0x1000bba0      0x938 CMakeFiles/main.dir/__/pico-sdk/lib/tinyusb/src/device/usbd.c.obj
                0x1000bba0                tud_task
 .text.dcd_event_bus_signal
                0x1000c4d8      0x124 CMakeFiles/main.dir/__/pico-sdk/lib/tinyusb/src/device/usbd.c.obj
                0x1000c4d8                dcd_event_bus_signal
 .text.dcd_event_bus_reset
                0x1000c5fc       0x58 CMakeFiles/main.dir/__/pico-sdk/lib/tinyusb/src/device/usbd.c.obj
                0x1000c5fc                dcd_event_bus_reset
 .text.dcd_event_setup_received
                0x1000c654       0x50 CMakeFiles/main.dir/__/pico-sdk/lib/tinyusb/src/device/usbd.c.obj
                0x1000c654                dcd_event_setup_received
 .text.dcd_event_xfer_complete
                0x1000c6a4       0x68 CMakeFiles/main.dir/__/pico-sdk/lib/tinyusb/src/device/usbd.c.obj
                0x1000c6a4                dcd_event_xfer_complete
 .text.usbd_open_edpt_pair
                0x1000c70c       0xa4 CMakeFiles/main.dir/__/pico-sdk/lib/tinyusb/src/device/usbd.c.obj
                0x1000c70c                usbd_open_edpt_pair
 .text.usbd_edpt_open
                0x1000c7b0       0x30 CMakeFiles/main.dir/__/pico-sdk/lib/tinyusb/src/device/usbd.c.obj
                0x1000c7b0                usbd_edpt_open
 .text.usbd_edpt_claim
                0x1000c7e0       0x5c CMakeFiles/main.dir/__/pico-sdk/lib/tinyusb/src/device/usbd.c.obj
                0x1000c7e0                usbd_edpt_claim
 .text.usbd_edpt_release
                0x1000c83c       0x4c CMakeFiles/main.dir/__/pico-sdk/lib/tinyusb/src/device/usbd.c.obj
                0x1000c83c                usbd_edpt_release
 .text.usbd_edpt_xfer
                0x1000c888       0x48 CMakeFiles/main.dir/__/pico-sdk/lib/tinyusb/src/device/usbd.c.obj
                0x1000c888                usbd_edpt_xfer
 .text.tud_control_status
                0x1000c8d0       0x30 CMakeFiles/main.dir/__/pico-sdk/lib/tinyusb/src/device/usbd_control.c.obj
                0x1000c8d0                tud_control_status
 .text.tud_control_xfer
                0x1000c900       0xb4 CMakeFiles/main.dir/__/pico-sdk/lib/tinyusb/src/device/usbd_control.c.obj
                0x1000c900                tud_control_xfer
 .text.usbd_control_reset
                0x1000c9b4       0x14 CMakeFiles/main.dir/__/pico-sdk/lib/tinyusb/src/device/usbd_control.c.obj
                0x1000c9b4                usbd_control_reset
 .text.usbd_control_set_complete_callback
                0x1000c9c8        0xc CMakeFiles/main.dir/__/pico-sdk/lib/tinyusb/src/device/usbd_control.c.obj
                0x1000c9c8                usbd_control_set_complete_callback
 .text.usbd_control_set_request
                0x1000c9d4       0x1c CMakeFiles/main.dir/__/pico-sdk/lib/tinyusb/src/device/usbd_control.c.obj
                0x1000c9d4                usbd_control_set_request
 .text.usbd_control_xfer_cb
                0x1000c9f0       0xfc CMakeFiles/main.dir/__/pico-sdk/lib/tinyusb/src/device/usbd_control.c.obj
                0x1000c9f0                usbd_control_xfer_cb
 .text.tud_cdc_n_connected
                0x1000caec       0x30 CMakeFiles/main.dir/__/pico-sdk/lib/tinyusb/src/class/cdc/cdc_device.c.obj
                0x1000caec                tud_cdc_n_connected
 .text.tud_cdc_n_available
                0x1000cb1c       0x1c CMakeFiles/main.dir/__/pico-sdk/lib/tinyusb/src/class/cdc/cdc_device.c.obj
                0x1000cb1c                tud_cdc_n_available
 .text.tud_cdc_n_read
                0x1000cb38       0x70 CMakeFiles/main.dir/__/pico-sdk/lib/tinyusb/src/class/cdc/cdc_device.c.obj
                0x1000cb38                tud_cdc_n_read
 .text.tud_cdc_n_write
                0x1000cba8       0x90 CMakeFiles/main.dir/__/pico-sdk/lib/tinyusb/src/class/cdc/cdc_device.c.obj
                0x1000cba8                tud_cdc_n_write
 .text.tud_cdc_n_write_flush
                0x1000cc38       0x78 CMakeFiles/main.dir/__/pico-sdk/lib/tinyusb/src/class/cdc/cdc_device.c.obj
                0x1000cc38                tud_cdc_n_write_flush
 .text.tud_cdc_n_write_available
                0x1000ccb0       0x1c CMakeFiles/main.dir/__/pico-sdk/lib/tinyusb/src/class/cdc/cdc_device.c.obj
                0x1000ccb0                tud_cdc_n_write_available
 .text.cdcd_init
                0x1000cccc       0x7c CMakeFiles/main.dir/__/pico-sdk/lib/tinyusb/src/class/cdc/cdc_device.c.obj
                0x1000cccc                cdcd_init
 .text.cdcd_reset
                0x1000cd48       0x2c CMakeFiles/main.dir/__/pico-sdk/lib/tinyusb/src/class/cdc/cdc_device.c.obj
                0x1000cd48                cdcd_reset
 .text.cdcd_open
                0x1000cd74       0xe4 CMakeFiles/main.dir/__/pico-sdk/lib/tinyusb/src/class/cdc/cdc_device.c.obj
                0x1000cd74                cdcd_open
 .text.cdcd_control_xfer_cb
                0x1000ce58       0xe4 CMakeFiles/main.dir/__/pico-sdk/lib/tinyusb/src/class/cdc/cdc_device.c.obj
                0x1000ce58                cdcd_control_xfer_cb
 .text.cdcd_xfer_cb
                0x1000cf3c      0x198 CMakeFiles/main.dir/__/pico-sdk/lib/tinyusb/src/class/cdc/cdc_device.c.obj
                0x1000cf3c                cdcd_xfer_cb
 .text.tusb_init
                0x1000d0d4        0xc CMakeFiles/main.dir/__/pico-sdk/lib/tinyusb/src/tusb.c.obj
                0x1000d0d4                tusb_init
 .text.tusb_inited
                0x1000d0e0        0x8 CMakeFiles/main.dir/__/pico-sdk/lib/tinyusb/src/tusb.c.obj
                0x1000d0e0                tusb_inited
 .text.tu_edpt_validate
                0x1000d0e8       0x78 CMakeFiles/main.dir/__/pico-sdk/lib/tinyusb/src/tusb.c.obj
                0x1000d0e8                tu_edpt_validate
 .text.tu_edpt_bind_driver
                0x1000d160       0x2c CMakeFiles/main.dir/__/pico-sdk/lib/tinyusb/src/tusb.c.obj
                0x1000d160                tu_edpt_bind_driver
 .text.tu_fifo_config
                0x1000d18c       0x78 CMakeFiles/main.dir/__/pico-sdk/lib/tinyusb/src/common/tusb_fifo.c.obj
                0x1000d18c                tu_fifo_config
 .text.tu_fifo_count
                0x1000d204       0x24 CMakeFiles/main.dir/__/pico-sdk/lib/tinyusb/src/common/tusb_fifo.c.obj
                0x1000d204                tu_fifo_count
 .text.tu_fifo_empty
                0x1000d228       0x10 CMakeFiles/main.dir/__/pico-sdk/lib/tinyusb/src/common/tusb_fifo.c.obj
                0x1000d228                tu_fifo_empty
 .text.tu_fifo_remaining
                0x1000d238       0x20 CMakeFiles/main.dir/__/pico-sdk/lib/tinyusb/src/common/tusb_fifo.c.obj
                0x1000d238                tu_fifo_remaining
 .text.tu_fifo_read
                0x1000d258       0x9c CMakeFiles/main.dir/__/pico-sdk/lib/tinyusb/src/common/tusb_fifo.c.obj
                0x1000d258                tu_fifo_read
 .text.tu_fifo_read_n
                0x1000d2f4       0xf0 CMakeFiles/main.dir/__/pico-sdk/lib/tinyusb/src/common/tusb_fifo.c.obj
                0x1000d2f4                tu_fifo_read_n
 .text.tu_fifo_write
                0x1000d3e4       0x80 CMakeFiles/main.dir/__/pico-sdk/lib/tinyusb/src/common/tusb_fifo.c.obj
                0x1000d3e4                tu_fifo_write
 .text.tu_fifo_write_n
                0x1000d464       0xe8 CMakeFiles/main.dir/__/pico-sdk/lib/tinyusb/src/common/tusb_fifo.c.obj
                0x1000d464                tu_fifo_write_n
 .text.tu_fifo_clear
                0x1000d54c       0x4c CMakeFiles/main.dir/__/pico-sdk/lib/tinyusb/src/common/tusb_fifo.c.obj
                0x1000d54c                tu_fifo_clear
 .text.tu_fifo_set_overwritable
                0x1000d598       0x3c CMakeFiles/main.dir/__/pico-sdk/lib/tinyusb/src/common/tusb_fifo.c.obj
                0x1000d598                tu_fifo_set_overwritable
 .text.startup._retrieve_unique_id_on_boot
                0x1000d5d4       0x10 CMakeFiles/main.dir/__/pico-sdk/src/rp2_common/pico_unique_id/unique_id.c.obj
 .text.pico_get_unique_board_id_string
                0x1000d5e4      0x1cc CMakeFiles/main.dir/__/pico-sdk/src/rp2_common/pico_unique_id/unique_id.c.obj
                0x1000d5e4                pico_get_unique_board_id_string
 .text.flash_get_unique_id
                0x1000d7b0       0x3c CMakeFiles/main.dir/__/pico-sdk/src/rp2_common/hardware_flash/flash.c.obj
                0x1000d7b0                flash_get_unique_id
 .text.spi_init
                0x1000d7ec       0xec CMakeFiles/main.dir/__/pico-sdk/src/rp2_common/hardware_spi/spi.c.obj
                0x1000d7ec                spi_init
 .text.i2c_write_blocking_internal
                0x1000d8d8      0x17c CMakeFiles/main.dir/__/pico-sdk/src/rp2_common/hardware_i2c/i2c.c.obj
 .text.i2c_read_blocking_internal
                0x1000da54       0xe8 CMakeFiles/main.dir/__/pico-sdk/src/rp2_common/hardware_i2c/i2c.c.obj
 .text.i2c_init
                0x1000db3c      0x108 CMakeFiles/main.dir/__/pico-sdk/src/rp2_common/hardware_i2c/i2c.c.obj
                0x1000db3c                i2c_init
 .text.i2c_write_blocking_until
                0x1000dc44       0x44 CMakeFiles/main.dir/__/pico-sdk/src/rp2_common/hardware_i2c/i2c.c.obj
                0x1000dc44                i2c_write_blocking_until
 .text.i2c_read_blocking_until
                0x1000dc88       0x44 CMakeFiles/main.dir/__/pico-sdk/src/rp2_common/hardware_i2c/i2c.c.obj
                0x1000dc88                i2c_read_blocking_until
 .text._ZN5Print17availableForWriteEv
                0x1000dccc        0x4 libLoRa_pico_lib.a(LoRa-RP2040.cpp.obj)
                0x1000dccc                Print::availableForWrite()
 .text._ZN9LoRaClass5flushEv
                0x1000dcd0        0x4 libLoRa_pico_lib.a(LoRa-RP2040.cpp.obj)
                0x1000dcd0                LoRaClass::flush()
 .text._ZN9LoRaClass9availableEv
                0x1000dcd4       0x64 libLoRa_pico_lib.a(LoRa-RP2040.cpp.obj)
                0x1000dcd4                LoRaClass::available()
 .text._ZN9LoRaClass5writeEh
                0x1000dd38       0xf4 libLoRa_pico_lib.a(LoRa-RP2040.cpp.obj)
                0x1000dd38                LoRaClass::write(unsigned char)
 .text._ZN9LoRaClass4readEv
                0x1000de2c       0xbc libLoRa_pico_lib.a(LoRa-RP2040.cpp.obj)
                0x1000de2c                LoRaClass::read()
 .text._ZN9LoRaClass5writeEPKhj
                0x1000dee8      0x118 libLoRa_pico_lib.a(LoRa-RP2040.cpp.obj)
                0x1000dee8                LoRaClass::write(unsigned char const*, unsigned int)
 .text._ZN9LoRaClass4peekEv
                0x1000e000      0x12c libLoRa_pico_lib.a(LoRa-RP2040.cpp.obj)
                0x1000e000                LoRaClass::peek()
 .text._ZN9LoRaClass5beginEl
                0x1000e12c      0x37c libLoRa_pico_lib.a(LoRa-RP2040.cpp.obj)
                0x1000e12c                LoRaClass::begin(long)
 .text._ZN9LoRaClass11beginPacketEi
                0x1000e4a8      0x218 libLoRa_pico_lib.a(LoRa-RP2040.cpp.obj)
                0x1000e4a8                LoRaClass::beginPacket(int)
 .text._ZN9LoRaClass9endPacketEb
                0x1000e6c0      0x150 libLoRa_pico_lib.a(LoRa-RP2040.cpp.obj)
                0x1000e6c0                LoRaClass::endPacket(bool)
 .text._ZN9LoRaClass11parsePacketEi
                0x1000e810      0x320 libLoRa_pico_lib.a(LoRa-RP2040.cpp.obj)
                0x1000e810                LoRaClass::parsePacket(int)
 .text._ZN9LoRaClass10packetRssiEv
                0x1000eb30       0x7c libLoRa_pico_lib.a(LoRa-RP2040.cpp.obj)
                0x1000eb30                LoRaClass::packetRssi()
 .text._ZN9LoRaClass7receiveEi
                0x1000ebac      0x170 libLoRa_pico_lib.a(LoRa-RP2040.cpp.obj)
                0x1000ebac                LoRaClass::receive(int)
 .text._ZN9LoRaClass10setTxPowerEii
                0x1000ed1c      0x17c libLoRa_pico_lib.a(LoRa-RP2040.cpp.obj)
                0x1000ed1c                LoRaClass::setTxPower(int, int)
 .text._ZN9LoRaClass18setSpreadingFactorEi
                0x1000ee98      0x2ac libLoRa_pico_lib.a(LoRa-RP2040.cpp.obj)
                0x1000ee98                LoRaClass::setSpreadingFactor(int)
 .text._ZN9LoRaClass18setSignalBandwidthEl
                0x1000f144      0x2a0 libLoRa_pico_lib.a(LoRa-RP2040.cpp.obj)
                0x1000f144                LoRaClass::setSignalBandwidth(long)
 .text._ZN9LoRaClass14setCodingRate4Ei
                0x1000f3e4       0xa4 libLoRa_pico_lib.a(LoRa-RP2040.cpp.obj)
                0x1000f3e4                LoRaClass::setCodingRate4(int)
 .text._ZN9LoRaClass17setPreambleLengthEl
                0x1000f488       0x90 libLoRa_pico_lib.a(LoRa-RP2040.cpp.obj)
                0x1000f488                LoRaClass::setPreambleLength(long)
 .text._ZN9LoRaClass9enableCrcEv
                0x1000f518       0x94 libLoRa_pico_lib.a(LoRa-RP2040.cpp.obj)
                0x1000f518                LoRaClass::enableCrc()
 .text.startup._GLOBAL__sub_I__ZN9LoRaClassC2Ev
                0x1000f5ac       0x34 libLoRa_pico_lib.a(LoRa-RP2040.cpp.obj)
 .text          0x1000f5e0      0xa6c libKISS.a(kiss.cpp.obj)
                0x1000f5e0                KissClass::EncodeFrame(aprs_frame*, ax25_frame*)
                0x1000fac8                KissClass::DecodeFrame(unsigned char*, kiss_tx_frame*)
                0x1000ffa0                KissClass::EncodeCall(unsigned char*)
 .text._Z10initAM2315v
                0x1001004c      0x15c libi2c_sensor.a(i2c_sensor.cpp.obj)
                0x1001004c                initAM2315()
 .text._Z10ReadAM2315PsS_
                0x100101a8      0x154 libi2c_sensor.a(i2c_sensor.cpp.obj)
                0x100101a8                ReadAM2315(short*, short*)
 .text          0x100102fc       0x10 /usr/lib/gcc/arm-none-eabi/7.3.1/../../../arm-none-eabi/lib/thumb/v6-m/libc.a(lib_a-abort.o)
                0x100102fc                abort
 .text          0x1001030c      0x570 /usr/lib/gcc/arm-none-eabi/7.3.1/../../../arm-none-eabi/lib/thumb/v6-m/libc.a(lib_a-mallocr.o)
                0x1001030c                _malloc_r
 .text          0x1001087c        0x8 /usr/lib/gcc/arm-none-eabi/7.3.1/../../../arm-none-eabi/lib/thumb/v6-m/libc.a(lib_a-mlock.o)
                0x1001087c                __malloc_lock
                0x10010880                __malloc_unlock
 .text          0x10010884       0x24 /usr/lib/gcc/arm-none-eabi/7.3.1/../../../arm-none-eabi/lib/thumb/v6-m/libc.a(lib_a-sbrkr.o)
                0x10010884                _sbrk_r
 .text          0x100108a8      0x190 /usr/lib/gcc/arm-none-eabi/7.3.1/../../../arm-none-eabi/lib/thumb/v6-m/libc.a(lib_a-signal.o)
                0x100108d4                _init_signal_r
                0x100108f0                _signal_r
                0x1001092c                _raise_r
                0x10010988                __sigtramp_r
                0x100109d8                raise
                0x100109ec                signal
                0x10010a04                _init_signal
                0x10010a24                __sigtramp
 .text          0x10010a38       0x30 /usr/lib/gcc/arm-none-eabi/7.3.1/../../../arm-none-eabi/lib/thumb/v6-m/libc.a(lib_a-signalr.o)
                0x10010a38                _kill_r
                0x10010a60                _getpid_r
 .text          0x10010a68       0x88 /usr/lib/gcc/arm-none-eabi/7.3.1/../../../arm-none-eabi/lib/thumb/v6-m/libc.a(lib_a-strcmp.o)
                0x10010a68                strcmp
 .text          0x10010af0       0x64 /usr/lib/gcc/arm-none-eabi/7.3.1/../../../arm-none-eabi/lib/thumb/v6-m/libc.a(lib_a-strlen-stub.o)
                0x10010af0                strlen
 .text          0x10010b54      0x274 /usr/lib/gcc/arm-none-eabi/7.3.1/../../../arm-none-eabi/lib/thumb/v6-m/libc.a(lib_a-freer.o)
                0x10010b54                _malloc_trim_r
                0x10010bf4                _free_r
 .text          0x10010dc8       0x10 /usr/lib/gcc/arm-none-eabi/7.3.1/../../../arm-none-eabi/lib/thumb/v6-m/libnosys.a(getpid.o)
                0x10010dc8                _getpid
 .text          0x10010dd8       0x10 /usr/lib/gcc/arm-none-eabi/7.3.1/../../../arm-none-eabi/lib/thumb/v6-m/libnosys.a(kill.o)
                0x10010dd8                _kill
 *(.fini)
 .fini          0x10010de8        0x4 /usr/lib/gcc/arm-none-eabi/7.3.1/thumb/v6-m/crti.o
                0x10010de8                _fini
 *fill*         0x10010dec        0x4 
 .fini.__stub   0x10010df0       0xc0 linker stubs
 *crtbegin.o(.ctors)
 *crtbegin?.o(.ctors)
 *(EXCLUDE_FILE(*crtend.o *crtend?.o) .ctors)
 *(SORT_BY_NAME(.ctors.*))
 *(.ctors)
 *crtbegin.o(.dtors)
 *crtbegin?.o(.dtors)
 *(EXCLUDE_FILE(*crtend.o *crtend?.o) .dtors)
 *(SORT_BY_NAME(.dtors.*))
 *(.dtors)
 *(.eh_frame*)
 .eh_frame      0x10010eb0        0x0 /usr/lib/gcc/arm-none-eabi/7.3.1/thumb/v6-m/crtbegin.o
                0x10010eb0                . = ALIGN (0x4)

.glue_7         0x10010eb0        0x0
 .glue_7        0x10010eb0        0x0 linker stubs

.glue_7t        0x10010eb0        0x0
 .glue_7t       0x10010eb0        0x0 linker stubs

.vfp11_veneer   0x10010eb0        0x0
 .vfp11_veneer  0x10010eb0        0x0 linker stubs

.v4_bx          0x10010eb0        0x0
 .v4_bx         0x10010eb0        0x0 linker stubs

.iplt           0x10010eb0        0x0
 .iplt          0x10010eb0        0x0 /usr/lib/gcc/arm-none-eabi/7.3.1/thumb/v6-m/crtbegin.o

.rodata         0x10010eb0      0xe94
 *(EXCLUDE_FILE(*libm.a: *libc.a:*lib_a-mem*.o *libgcc.a:) .rodata*)
 .rodata.main   0x10010eb0       0x98 CMakeFiles/main.dir/main.cpp.obj
 .rodata        0x10010f48       0x80 CMakeFiles/main.dir/main.cpp.obj
 .rodata._Z10print_helpv.str1.4
                0x10010fc8      0x135 CMakeFiles/main.dir/main.cpp.obj
 *fill*         0x100110fd        0x3 
 .rodata._Z12ShowSettingsv.str1.4
                0x10011100      0x1e0 CMakeFiles/main.dir/main.cpp.obj
 .rodata._Z13ReadUSBSerialv.str1.4
                0x100112e0        0x3 CMakeFiles/main.dir/main.cpp.obj
                                  0x6 (size before relaxing)
 *fill*         0x100112e3        0x1 
 .rodata._Z13decode_packetv.str1.4
                0x100112e4       0x9b CMakeFiles/main.dir/main.cpp.obj
 .rodata._Z16ComposeAprsFramePh.str1.4
                0x1001137f       0x9b CMakeFiles/main.dir/main.cpp.obj
                                  0x4 (size before relaxing)
 *fill*         0x1001137f        0x1 
 .rodata._Z18ProcessSerialInputPc.part.0.str1.4
                0x10011380      0x28c CMakeFiles/main.dir/main.cpp.obj
 .rodata._Z19SaveSettingsToFlashv.str1.4
                0x1001160c       0x3d CMakeFiles/main.dir/main.cpp.obj
 *fill*         0x10011649        0x3 
 .rodata._Z21ReadSettingsFromFlashv.str1.4
                0x1001164c       0x63 CMakeFiles/main.dir/main.cpp.obj
 *fill*         0x100116af        0x1 
 .rodata._Z24ComposeAprsFrameFromKissv.str1.4
                0x100116b0       0x1d CMakeFiles/main.dir/main.cpp.obj
 *fill*         0x100116cd        0x3 
 .rodata._Z5setupv.str1.4
                0x100116d0       0x94 CMakeFiles/main.dir/main.cpp.obj
 .rodata._Z7log_outPKcz.str1.4
                0x10011764        0x3 CMakeFiles/main.dir/main.cpp.obj
 *fill*         0x10011767        0x1 
 .rodata.main.str1.4
                0x10011768       0x7b CMakeFiles/main.dir/main.cpp.obj
 *fill*         0x100117e3        0x1 
 .rodata.spin_lock_claim_unused.str1.4
                0x100117e4       0x1b CMakeFiles/main.dir/__/pico-sdk/src/rp2_common/hardware_sync/sync.c.obj
 *fill*         0x100117ff        0x1 
 .rodata.hardware_alarm_claim.str1.4
                0x10011800       0x22 CMakeFiles/main.dir/__/pico-sdk/src/rp2_common/hardware_timer/timer.c.obj
 *fill*         0x10011822        0x2 
 .rodata.hard_assertion_failure.str1.4
                0x10011824        0xc CMakeFiles/main.dir/__/pico-sdk/src/rp2_common/pico_runtime/runtime.c.obj
 .rodata.panic.str1.4
                0x10011830       0x10 CMakeFiles/main.dir/__/pico-sdk/src/rp2_common/pico_runtime/runtime.c.obj
                                 0x12 (size before relaxing)
 .rodata._vsnprintf
                0x10011840      0x1e0 CMakeFiles/main.dir/__/pico-sdk/src/rp2_common/pico_printf/printf.c.obj
 .rodata._etoa.part.0.str1.4
                0x10011a20        0x9 CMakeFiles/main.dir/__/pico-sdk/src/rp2_common/pico_printf/printf.c.obj
 *fill*         0x10011a29        0x3 
 .rodata._ftoa.str1.4
                0x10011a2c        0xc CMakeFiles/main.dir/__/pico-sdk/src/rp2_common/pico_printf/printf.c.obj
 .rodata.pow10.5382
                0x10011a38       0x50 CMakeFiles/main.dir/__/pico-sdk/src/rp2_common/pico_printf/printf.c.obj
 .rodata.__bi_44
                0x10011a88        0xc CMakeFiles/main.dir/__/pico-sdk/src/rp2_common/pico_standard_link/binary_info.c.obj
 .rodata.__bi_75
                0x10011a94        0xc CMakeFiles/main.dir/__/pico-sdk/src/rp2_common/pico_standard_link/binary_info.c.obj
 .rodata.__bi_81
                0x10011aa0        0xc CMakeFiles/main.dir/__/pico-sdk/src/rp2_common/pico_standard_link/binary_info.c.obj
 .rodata.str1.4
                0x10011aac       0x3c CMakeFiles/main.dir/__/pico-sdk/src/rp2_common/pico_standard_link/binary_info.c.obj
 .rodata.crlf_str.5851
                0x10011ae8        0x2 CMakeFiles/main.dir/__/pico-sdk/src/rp2_common/pico_stdio/stdio.c.obj
 *fill*         0x10011aea        0x2 
 .rodata._resetd_driver
                0x10011aec       0x18 CMakeFiles/main.dir/__/pico-sdk/src/rp2_common/pico_stdio_usb/reset_interface.c.obj
 .rodata.__bi_93.7129
                0x10011b04        0xc CMakeFiles/main.dir/__/pico-sdk/src/rp2_common/pico_stdio_usb/stdio_usb.c.obj
 .rodata.str1.4
                0x10011b10       0x13 CMakeFiles/main.dir/__/pico-sdk/src/rp2_common/pico_stdio_usb/stdio_usb.c.obj
 *fill*         0x10011b23        0x1 
 .rodata.str1.4
                0x10011b24       0x2a CMakeFiles/main.dir/__/pico-sdk/src/rp2_common/pico_stdio_usb/stdio_usb_descriptors.c.obj
 *fill*         0x10011b4e        0x2 
 .rodata.usbd_desc_cfg
                0x10011b50       0x54 CMakeFiles/main.dir/__/pico-sdk/src/rp2_common/pico_stdio_usb/stdio_usb_descriptors.c.obj
 .rodata.usbd_desc_device
                0x10011ba4       0x12 CMakeFiles/main.dir/__/pico-sdk/src/rp2_common/pico_stdio_usb/stdio_usb_descriptors.c.obj
 *fill*         0x10011bb6        0x2 
 .rodata.usbd_desc_str
                0x10011bb8       0x18 CMakeFiles/main.dir/__/pico-sdk/src/rp2_common/pico_stdio_usb/stdio_usb_descriptors.c.obj
 .rodata.dcd_rp2040_irq.str1.4
                0x10011bd0       0x14 CMakeFiles/main.dir/__/pico-sdk/lib/tinyusb/src/portable/raspberrypi/rp2040/dcd_rp2040.c.obj
 .rodata._hw_endpoint_buffer_control_update32.str1.4
                0x10011be4       0x1f CMakeFiles/main.dir/__/pico-sdk/lib/tinyusb/src/portable/raspberrypi/rp2040/rp2040_usb.c.obj
 *fill*         0x10011c03        0x1 
 .rodata.hw_endpoint_xfer_continue.str1.4
                0x10011c04       0x29 CMakeFiles/main.dir/__/pico-sdk/lib/tinyusb/src/portable/raspberrypi/rp2040/rp2040_usb.c.obj
 *fill*         0x10011c2d        0x3 
 .rodata.str1.4
                0x10011c30        0x7 CMakeFiles/main.dir/__/pico-sdk/lib/tinyusb/src/portable/raspberrypi/rp2040/rp2040_usb.c.obj
 *fill*         0x10011c37        0x1 
 .rodata.tud_task
                0x10011c38       0x8c CMakeFiles/main.dir/__/pico-sdk/lib/tinyusb/src/device/usbd.c.obj
 .rodata._usbd_driver
                0x10011cc4       0x18 CMakeFiles/main.dir/__/pico-sdk/lib/tinyusb/src/device/usbd.c.obj
 .rodata.CSWTCH.43
                0x10011cdc       0x28 libLoRa_pico_lib.a(LoRa-RP2040.cpp.obj)
 .rodata._ZTV9LoRaClass
                0x10011d04       0x24 libLoRa_pico_lib.a(LoRa-RP2040.cpp.obj)
                0x10011d04                vtable for LoRaClass
 .rodata._ZZN9LoRaClass5beginElE8__bi_131
                0x10011d28        0x8 libLoRa_pico_lib.a(LoRa-RP2040.cpp.obj)
 .rodata._ZZN9LoRaClass5beginElE8__bi_138
                0x10011d30        0xc libLoRa_pico_lib.a(LoRa-RP2040.cpp.obj)
 .rodata.str1.4
                0x10011d3c        0x8 libLoRa_pico_lib.a(LoRa-RP2040.cpp.obj)
                                  0x7 (size before relaxing)
                0x10011d44                . = ALIGN (0x4)
 *(SORT_BY_ALIGNMENT(SORT_BY_NAME(.flashdata*)))
                0x10011d44                . = ALIGN (0x4)

.ARM.extab      0x10011d44      0x150
 *(.ARM.extab* .gnu.linkonce.armextab.*)
 .ARM.extab.text._ZN12aprssettingsC2Ev
                0x10011d44        0x0 CMakeFiles/main.dir/main.cpp.obj
 .ARM.extab.text._ZN6statusC2Ev
                0x10011d44        0x0 CMakeFiles/main.dir/main.cpp.obj
 .ARM.extab.text._Z7log_outPKcz
                0x10011d44        0xc CMakeFiles/main.dir/main.cpp.obj
 .ARM.extab.text._Z13decode_packetv
                0x10011d50        0xc CMakeFiles/main.dir/main.cpp.obj
 .ARM.extab.text._Z24ComposeAprsFrameFromKissv
                0x10011d5c        0xc CMakeFiles/main.dir/main.cpp.obj
 .ARM.extab.text.startup.main
                0x10011d68        0xc CMakeFiles/main.dir/main.cpp.obj
 .ARM.extab.text._ZN5Print17availableForWriteEv
                0x10011d74        0x0 libLoRa_pico_lib.a(LoRa-RP2040.cpp.obj)
 .ARM.extab.text._ZN9LoRaClass9availableEv
                0x10011d74        0xc libLoRa_pico_lib.a(LoRa-RP2040.cpp.obj)
 .ARM.extab.text._ZN9LoRaClass5writeEh
                0x10011d80        0xc libLoRa_pico_lib.a(LoRa-RP2040.cpp.obj)
 .ARM.extab.text._ZN9LoRaClass4readEv
                0x10011d8c        0xc libLoRa_pico_lib.a(LoRa-RP2040.cpp.obj)
 .ARM.extab.text._ZN9LoRaClass5writeEPKhj
                0x10011d98        0xc libLoRa_pico_lib.a(LoRa-RP2040.cpp.obj)
 .ARM.extab.text._ZN9LoRaClass4peekEv
                0x10011da4        0xc libLoRa_pico_lib.a(LoRa-RP2040.cpp.obj)
 .ARM.extab.text._ZN9LoRaClass5beginEl
                0x10011db0        0xc libLoRa_pico_lib.a(LoRa-RP2040.cpp.obj)
 .ARM.extab.text._ZN9LoRaClass11beginPacketEi
                0x10011dbc        0xc libLoRa_pico_lib.a(LoRa-RP2040.cpp.obj)
 .ARM.extab.text._ZN9LoRaClass9endPacketEb
                0x10011dc8        0xc libLoRa_pico_lib.a(LoRa-RP2040.cpp.obj)
 .ARM.extab.text._ZN9LoRaClass11parsePacketEi
                0x10011dd4        0xc libLoRa_pico_lib.a(LoRa-RP2040.cpp.obj)
 .ARM.extab.text._ZN9LoRaClass10packetRssiEv
                0x10011de0        0xc libLoRa_pico_lib.a(LoRa-RP2040.cpp.obj)
 .ARM.extab.text._ZN9LoRaClass7receiveEi
                0x10011dec        0xc libLoRa_pico_lib.a(LoRa-RP2040.cpp.obj)
 .ARM.extab.text._ZN9LoRaClass10setTxPowerEii
                0x10011df8        0xc libLoRa_pico_lib.a(LoRa-RP2040.cpp.obj)
 .ARM.extab.text._ZN9LoRaClass18setSpreadingFactorEi
                0x10011e04        0xc libLoRa_pico_lib.a(LoRa-RP2040.cpp.obj)
 .ARM.extab.text._ZN9LoRaClass18setSignalBandwidthEl
                0x10011e10        0xc libLoRa_pico_lib.a(LoRa-RP2040.cpp.obj)
 .ARM.extab.text._ZN9LoRaClass14setCodingRate4Ei
                0x10011e1c        0xc libLoRa_pico_lib.a(LoRa-RP2040.cpp.obj)
 .ARM.extab.text._ZN9LoRaClass17setPreambleLengthEl
                0x10011e28        0xc libLoRa_pico_lib.a(LoRa-RP2040.cpp.obj)
 .ARM.extab.text._ZN9LoRaClass9enableCrcEv
                0x10011e34        0xc libLoRa_pico_lib.a(LoRa-RP2040.cpp.obj)
 .ARM.extab     0x10011e40        0xc libKISS.a(kiss.cpp.obj)
 .ARM.extab.text._Z10initAM2315v
                0x10011e4c        0xc libi2c_sensor.a(i2c_sensor.cpp.obj)
 .ARM.extab.text._Z10ReadAM2315PsS_
                0x10011e58        0xc libi2c_sensor.a(i2c_sensor.cpp.obj)
 .ARM.extab     0x10011e64       0x24 /usr/lib/gcc/arm-none-eabi/7.3.1/thumb/v6-m/libgcc.a(unwind-arm.o)
 .ARM.extab     0x10011e88        0xc /usr/lib/gcc/arm-none-eabi/7.3.1/thumb/v6-m/libgcc.a(pr-support.o)
                0x10011e94                __exidx_start = .

.ARM.exidx      0x10011e94      0x1e8
 *(.ARM.exidx* .gnu.linkonce.armexidx.*)
 .ARM.exidx.text._ZN12aprssettingsC2Ev
                0x10011e94        0x8 CMakeFiles/main.dir/main.cpp.obj
 .ARM.exidx.text._ZN6statusC2Ev
                0x10011e9c        0x0 CMakeFiles/main.dir/main.cpp.obj
                                  0x8 (size before relaxing)
 .ARM.exidx.text._Z7log_outPKcz
                0x10011e9c        0x8 CMakeFiles/main.dir/main.cpp.obj
 .ARM.exidx.text._Z12ShowSettingsv
                0x10011ea4        0x8 CMakeFiles/main.dir/main.cpp.obj
 .ARM.exidx.text._Z5setupv
                0x10011eac        0x8 CMakeFiles/main.dir/main.cpp.obj
 .ARM.exidx.text._Z10print_helpv
                0x10011eb4        0x8 CMakeFiles/main.dir/main.cpp.obj
 .ARM.exidx.text._Z10startRadiov
                0x10011ebc        0x8 CMakeFiles/main.dir/main.cpp.obj
 .ARM.exidx.text._Z18ProcessSerialInputPc.part.0
                0x10011ec4        0x8 CMakeFiles/main.dir/main.cpp.obj
 .ARM.exidx.text._Z16ComposeAprsFramePh
                0x10011ecc        0x8 CMakeFiles/main.dir/main.cpp.obj
 .ARM.exidx.text._Z13decode_packetv
                0x10011ed4        0x8 CMakeFiles/main.dir/main.cpp.obj
 .ARM.exidx.text._Z24ComposeAprsFrameFromKissv
                0x10011edc        0x8 CMakeFiles/main.dir/main.cpp.obj
 .ARM.exidx.text._Z13ReadUSBSerialv
                0x10011ee4        0x8 CMakeFiles/main.dir/main.cpp.obj
 .ARM.exidx.text.startup._GLOBAL__sub_I_lastRssi
                0x10011eec        0x8 CMakeFiles/main.dir/main.cpp.obj
 .ARM.exidx.text.startup.main
                0x10011ef4       0x10 CMakeFiles/main.dir/main.cpp.obj
                                  0x8 (size before relaxing)
 .ARM.exidx.text._ZN5Print17availableForWriteEv
                0x10011f04        0x0 libLoRa_pico_lib.a(LoRa-RP2040.cpp.obj)
                                  0x8 (size before relaxing)
 .ARM.exidx.text._ZN9LoRaClass5flushEv
                0x10011f04        0x0 libLoRa_pico_lib.a(LoRa-RP2040.cpp.obj)
                                  0x8 (size before relaxing)
 .ARM.exidx.text._ZN9LoRaClass9availableEv
                0x10011f04        0x8 libLoRa_pico_lib.a(LoRa-RP2040.cpp.obj)
 .ARM.exidx.text._ZN9LoRaClass5writeEh
                0x10011f0c        0x8 libLoRa_pico_lib.a(LoRa-RP2040.cpp.obj)
 .ARM.exidx.text._ZN9LoRaClass4readEv
                0x10011f14        0x8 libLoRa_pico_lib.a(LoRa-RP2040.cpp.obj)
 .ARM.exidx.text._ZN9LoRaClass5writeEPKhj
                0x10011f1c        0x8 libLoRa_pico_lib.a(LoRa-RP2040.cpp.obj)
 .ARM.exidx.text._ZN9LoRaClass4peekEv
                0x10011f24        0x8 libLoRa_pico_lib.a(LoRa-RP2040.cpp.obj)
 .ARM.exidx.text._ZN9LoRaClass5beginEl
                0x10011f2c        0x8 libLoRa_pico_lib.a(LoRa-RP2040.cpp.obj)
 .ARM.exidx.text._ZN9LoRaClass11beginPacketEi
                0x10011f34        0x8 libLoRa_pico_lib.a(LoRa-RP2040.cpp.obj)
 .ARM.exidx.text._ZN9LoRaClass9endPacketEb
                0x10011f3c        0x8 libLoRa_pico_lib.a(LoRa-RP2040.cpp.obj)
 .ARM.exidx.text._ZN9LoRaClass11parsePacketEi
                0x10011f44        0x8 libLoRa_pico_lib.a(LoRa-RP2040.cpp.obj)
 .ARM.exidx.text._ZN9LoRaClass10packetRssiEv
                0x10011f4c        0x8 libLoRa_pico_lib.a(LoRa-RP2040.cpp.obj)
 .ARM.exidx.text._ZN9LoRaClass7receiveEi
                0x10011f54        0x8 libLoRa_pico_lib.a(LoRa-RP2040.cpp.obj)
 .ARM.exidx.text._ZN9LoRaClass10setTxPowerEii
                0x10011f5c        0x8 libLoRa_pico_lib.a(LoRa-RP2040.cpp.obj)
 .ARM.exidx.text._ZN9LoRaClass18setSpreadingFactorEi
                0x10011f64        0x8 libLoRa_pico_lib.a(LoRa-RP2040.cpp.obj)
 .ARM.exidx.text._ZN9LoRaClass18setSignalBandwidthEl
                0x10011f6c        0x8 libLoRa_pico_lib.a(LoRa-RP2040.cpp.obj)
 .ARM.exidx.text._ZN9LoRaClass14setCodingRate4Ei
                0x10011f74        0x8 libLoRa_pico_lib.a(LoRa-RP2040.cpp.obj)
 .ARM.exidx.text._ZN9LoRaClass17setPreambleLengthEl
                0x10011f7c        0x8 libLoRa_pico_lib.a(LoRa-RP2040.cpp.obj)
 .ARM.exidx.text._ZN9LoRaClass9enableCrcEv
                0x10011f84        0x8 libLoRa_pico_lib.a(LoRa-RP2040.cpp.obj)
 .ARM.exidx.text.startup._GLOBAL__sub_I__ZN9LoRaClassC2Ev
                0x10011f8c        0x8 libLoRa_pico_lib.a(LoRa-RP2040.cpp.obj)
 .ARM.exidx     0x10011f94       0x10 libKISS.a(kiss.cpp.obj)
                                 0x18 (size before relaxing)
 .ARM.exidx.text._Z10initAM2315v
                0x10011fa4        0x8 libi2c_sensor.a(i2c_sensor.cpp.obj)
 .ARM.exidx.text._Z10ReadAM2315PsS_
                0x10011fac       0x10 libi2c_sensor.a(i2c_sensor.cpp.obj)
                                  0x8 (size before relaxing)
 .ARM.exidx     0x10011fbc       0x90 /usr/lib/gcc/arm-none-eabi/7.3.1/thumb/v6-m/libgcc.a(unwind-arm.o)
                                 0xd8 (size before relaxing)
 .ARM.exidx     0x1001204c       0x30 /usr/lib/gcc/arm-none-eabi/7.3.1/thumb/v6-m/libgcc.a(pr-support.o)
                                 0x48 (size before relaxing)
                0x1001207c                __exidx_end = .

.rel.dyn        0x1001207c        0x0
 .rel.iplt      0x1001207c        0x0 /usr/lib/gcc/arm-none-eabi/7.3.1/thumb/v6-m/crtbegin.o
                0x1001207c                . = ALIGN (0x4)
                0x1001207c                __binary_info_start = .

.binary_info    0x1001207c       0x28
 *(.binary_info.keep.*)
 .binary_info.keep.__bi_ptr22
                0x1001207c        0x4 CMakeFiles/main.dir/__/pico-sdk/src/rp2_common/pico_standard_link/binary_info.c.obj
 .binary_info.keep.__bi_ptr30
                0x10012080        0x4 CMakeFiles/main.dir/__/pico-sdk/src/rp2_common/pico_standard_link/binary_info.c.obj
 .binary_info.keep.__bi_ptr38
                0x10012084        0x4 CMakeFiles/main.dir/__/pico-sdk/src/rp2_common/pico_standard_link/binary_info.c.obj
 .binary_info.keep.__bi_ptr44
                0x10012088        0x4 CMakeFiles/main.dir/__/pico-sdk/src/rp2_common/pico_standard_link/binary_info.c.obj
 .binary_info.keep.__bi_ptr50
                0x1001208c        0x4 CMakeFiles/main.dir/__/pico-sdk/src/rp2_common/pico_standard_link/binary_info.c.obj
 .binary_info.keep.__bi_ptr75
                0x10012090        0x4 CMakeFiles/main.dir/__/pico-sdk/src/rp2_common/pico_standard_link/binary_info.c.obj
 .binary_info.keep.__bi_ptr81
                0x10012094        0x4 CMakeFiles/main.dir/__/pico-sdk/src/rp2_common/pico_standard_link/binary_info.c.obj
 .binary_info.keep.__bi_ptr131
                0x10012098        0x4 libLoRa_pico_lib.a(LoRa-RP2040.cpp.obj)
 .binary_info.keep.__bi_ptr138
                0x1001209c        0x4 libLoRa_pico_lib.a(LoRa-RP2040.cpp.obj)
 *(.binary_info.*)
 .binary_info.__bi_ptr93
                0x100120a0        0x4 CMakeFiles/main.dir/__/pico-sdk/src/rp2_common/pico_stdio_usb/stdio_usb.c.obj
                0x100120a4                __binary_info_end = .
                0x100120a4                . = ALIGN (0x4)
                0x100120a4                __etext = .

.ram_vector_table
                0x20000000       0xc0
 *(.ram_vector_table)
 .ram_vector_table
                0x20000000       0xc0 CMakeFiles/main.dir/__/pico-sdk/src/rp2_common/pico_runtime/runtime.c.obj
                0x20000000                ram_vector_table

.data           0x200000c0     0x1d58 load address 0x100120a4
                0x200000c0                __data_start__ = .
 *(vtable)
 *(.time_critical*)
 .time_critical.mutex_enter_blocking
                0x200000c0       0x48 CMakeFiles/main.dir/__/pico-sdk/src/common/pico_sync/mutex.c.obj
                0x200000c0                mutex_enter_blocking
 .time_critical.mutex_try_enter
                0x20000108       0x48 CMakeFiles/main.dir/__/pico-sdk/src/common/pico_sync/mutex.c.obj
                0x20000108                mutex_try_enter
 .time_critical.mutex_enter_timeout_ms
                0x20000150       0x98 CMakeFiles/main.dir/__/pico-sdk/src/common/pico_sync/mutex.c.obj
                0x20000150                mutex_enter_timeout_ms
 .time_critical.mutex_exit
                0x200001e8       0x28 CMakeFiles/main.dir/__/pico-sdk/src/common/pico_sync/mutex.c.obj
                0x200001e8                mutex_exit
 .time_critical.flash_init_boot2_copyout
                0x20000210       0x34 CMakeFiles/main.dir/__/pico-sdk/src/rp2_common/hardware_flash/flash.c.obj
 .time_critical.flash_enable_xip_via_boot2
                0x20000244       0x10 CMakeFiles/main.dir/__/pico-sdk/src/rp2_common/hardware_flash/flash.c.obj
 .time_critical.flash_cs_force
                0x20000254       0x38 CMakeFiles/main.dir/__/pico-sdk/src/rp2_common/hardware_flash/flash.c.obj
 .time_critical.flash_range_erase
                0x2000028c       0x7c CMakeFiles/main.dir/__/pico-sdk/src/rp2_common/hardware_flash/flash.c.obj
                0x2000028c                flash_range_erase
 .time_critical.flash_range_program
                0x20000308       0x80 CMakeFiles/main.dir/__/pico-sdk/src/rp2_common/hardware_flash/flash.c.obj
                0x20000308                flash_range_program
 .time_critical.flash_do_cmd
                0x20000388       0xac CMakeFiles/main.dir/__/pico-sdk/src/rp2_common/hardware_flash/flash.c.obj
                0x20000388                flash_do_cmd
 .time_critical.spi_write_read_blocking
                0x20000434       0x58 CMakeFiles/main.dir/__/pico-sdk/src/rp2_common/hardware_spi/spi.c.obj
                0x20000434                spi_write_read_blocking
 .time_critical.spi_write_blocking
                0x2000048c       0x4c CMakeFiles/main.dir/__/pico-sdk/src/rp2_common/hardware_spi/spi.c.obj
                0x2000048c                spi_write_blocking
 *(.text*)
 .text          0x200004d8        0x4 /usr/lib/gcc/arm-none-eabi/7.3.1/thumb/v6-m/libgcc.a(_dvmd_tls.o)
                0x200004d8                __aeabi_ldiv0
                0x200004d8                __aeabi_idiv0
 .text          0x200004dc      0xa08 /usr/lib/gcc/arm-none-eabi/7.3.1/thumb/v6-m/libgcc.a(unwind-arm.o)
                0x20000798                _Unwind_GetCFA
                0x2000079c                __gnu_Unwind_RaiseException
                0x200007f0                __gnu_Unwind_ForcedUnwind
                0x20000804                __gnu_Unwind_Resume
                0x2000084c                __gnu_Unwind_Resume_or_Rethrow
                0x20000868                _Unwind_Complete
                0x2000086c                _Unwind_DeleteException
                0x2000087c                _Unwind_VRS_Get
                0x200008c4                _Unwind_VRS_Set
                0x2000090c                __gnu_Unwind_Backtrace
                0x20000c5c                __aeabi_unwind_cpp_pr0
                0x20000c68                __aeabi_unwind_cpp_pr1
                0x20000c74                __aeabi_unwind_cpp_pr2
                0x20000c80                _Unwind_VRS_Pop
 .text          0x20000ee4      0x144 /usr/lib/gcc/arm-none-eabi/7.3.1/thumb/v6-m/libgcc.a(libunwind.o)
                0x20000ee4                __restore_core_regs
                0x20000ee4                restore_core_regs
                0x20000f10                __gnu_Unwind_Restore_VFP
                0x20000f14                __gnu_Unwind_Save_VFP
                0x20000f18                __gnu_Unwind_Restore_VFP_D
                0x20000f1c                __gnu_Unwind_Save_VFP_D
                0x20000f20                __gnu_Unwind_Restore_VFP_D_16_to_31
                0x20000f24                __gnu_Unwind_Save_VFP_D_16_to_31
                0x20000f28                __gnu_Unwind_Restore_WMMXD
                0x20000f2c                __gnu_Unwind_Save_WMMXD
                0x20000f30                __gnu_Unwind_Restore_WMMXC
                0x20000f34                __gnu_Unwind_Save_WMMXC
                0x20000f38                ___Unwind_RaiseException
                0x20000f38                _Unwind_RaiseException
                0x20000f68                ___Unwind_Resume
                0x20000f68                _Unwind_Resume
                0x20000f98                _Unwind_Resume_or_Rethrow
                0x20000f98                ___Unwind_Resume_or_Rethrow
                0x20000fc8                ___Unwind_ForcedUnwind
                0x20000fc8                _Unwind_ForcedUnwind
                0x20000ff8                _Unwind_Backtrace
                0x20000ff8                ___Unwind_Backtrace
 .text          0x20001028      0x39c /usr/lib/gcc/arm-none-eabi/7.3.1/thumb/v6-m/libgcc.a(pr-support.o)
                0x2000107c                __gnu_unwind_execute
                0x2000136c                __gnu_unwind_frame
                0x20001394                _Unwind_GetRegionStart
                0x200013a0                _Unwind_GetLanguageSpecificData
                0x200013b4                _Unwind_GetDataRelBase
                0x200013bc                _Unwind_GetTextRelBase
 .text          0x200013c4       0x9c /usr/lib/gcc/arm-none-eabi/7.3.1/../../../arm-none-eabi/lib/thumb/v6-m/libc.a(lib_a-memmove.o)
                0x200013c4                memmove
 .text.__stub   0x20001460       0x60 linker stubs
                0x200014c0                . = ALIGN (0x4)
 *(.rodata*)
                0x200014c0                . = ALIGN (0x4)
 *(.data*)
 .data.flash_target_contents
                0x200014c0        0x4 CMakeFiles/main.dir/main.cpp.obj
                0x200014c0                flash_target_contents
 .data.striped_spin_lock_num
                0x200014c4        0x1 CMakeFiles/main.dir/__/pico-sdk/src/rp2_common/hardware_sync/sync.c.obj
 *fill*         0x200014c5        0x3 
 .data.default_alarm_pool
                0x200014c8       0x18 CMakeFiles/main.dir/__/pico-sdk/src/common/pico_time/time.c.obj
 .data.default_alarm_pool_heap
                0x200014e0       0x10 CMakeFiles/main.dir/__/pico-sdk/src/common/pico_time/time.c.obj
 .data          0x200014f0       0x48 CMakeFiles/main.dir/__/pico-sdk/src/rp2_common/hardware_irq/irq_handler_chain.S.obj
                0x200014f0                irq_handler_chain_slots
                0x20001520                irq_handler_chain_first_slot
                0x2000152a                irq_handler_chain_remove_tail
 *fill*         0x20001538        0x8 
 .data.aeabi_bits_funcs
                0x20001540       0x10 CMakeFiles/main.dir/__/pico-sdk/src/rp2_common/pico_bit_ops/bit_ops_aeabi.S.obj
                0x20001540                aeabi_bits_funcs
                0x20001550                aeabi_bits_funcs_end
 .data.aeabi_mem_funcs
                0x20001550       0x10 CMakeFiles/main.dir/__/pico-sdk/src/rp2_common/pico_mem_ops/mem_ops_aeabi.S.obj
                0x20001550                aeabi_mem_funcs
                0x20001560                aeabi_mem_funcs_end
 .data.stdio_usb
                0x20001560       0x14 CMakeFiles/main.dir/__/pico-sdk/src/rp2_common/pico_stdio_usb/stdio_usb.c.obj
                0x20001560                stdio_usb
 .data.ep_dir_string
                0x20001574        0x8 CMakeFiles/main.dir/__/pico-sdk/lib/tinyusb/src/portable/raspberrypi/rp2040/rp2040_usb.c.obj
                0x20001574                ep_dir_string
 .data._usbd_qdef
                0x2000157c       0x24 CMakeFiles/main.dir/__/pico-sdk/lib/tinyusb/src/device/usbd.c.obj
                0x2000157c                _usbd_qdef
 .data.i2c0_inst
                0x200015a0        0x8 CMakeFiles/main.dir/__/pico-sdk/src/rp2_common/hardware_i2c/i2c.c.obj
                0x200015a0                i2c0_inst
 .data.i2c1_inst
                0x200015a8        0x8 CMakeFiles/main.dir/__/pico-sdk/src/rp2_common/hardware_i2c/i2c.c.obj
                0x200015a8                i2c1_inst
 .data          0x200015b0      0x430 /usr/lib/gcc/arm-none-eabi/7.3.1/../../../arm-none-eabi/lib/thumb/v6-m/libc.a(lib_a-impure.o)
                0x200015b0                _impure_ptr
 .data          0x200019e0      0x410 /usr/lib/gcc/arm-none-eabi/7.3.1/../../../arm-none-eabi/lib/thumb/v6-m/libc.a(lib_a-mallocr.o)
                0x200019e0                __malloc_sbrk_base
                0x200019e4                __malloc_trim_threshold
                0x200019e8                __malloc_av_
                0x20001df0                . = ALIGN (0x4)
 *(.after_data.*)
                0x20001df0                . = ALIGN (0x4)
                0x20001df0                PROVIDE (__mutex_array_start = .)
 *(SORT_BY_NAME(.mutex_array.*))
 *(.mutex_array)
 .mutex_array   0x20001df0        0x8 CMakeFiles/main.dir/__/pico-sdk/src/rp2_common/pico_stdio/stdio.c.obj
                0x20001df8                PROVIDE (__mutex_array_end = .)
                0x20001df8                . = ALIGN (0x4)
                0x20001df8                PROVIDE (__preinit_array_start = .)
 *(SORT_BY_NAME(.preinit_array.*))
 .preinit_array.00001
                0x20001df8        0x4 CMakeFiles/main.dir/__/pico-sdk/src/rp2_common/pico_mem_ops/mem_ops_aeabi.S.obj
 .preinit_array.00010
                0x20001dfc        0x4 CMakeFiles/main.dir/__/pico-sdk/src/rp2_common/pico_bit_ops/bit_ops_aeabi.S.obj
 .preinit_array.00020
                0x20001e00        0x4 CMakeFiles/main.dir/__/pico-sdk/src/rp2_common/pico_double/double_aeabi.S.obj
 .preinit_array.00020
                0x20001e04        0x4 CMakeFiles/main.dir/__/pico-sdk/src/rp2_common/pico_float/float_aeabi.S.obj
 *(.preinit_array)
                0x20001e08                PROVIDE (__preinit_array_end = .)
                0x20001e08                . = ALIGN (0x4)
                0x20001e08                PROVIDE (__init_array_start = .)
 *(SORT_BY_NAME(.init_array.*))
 *(.init_array)
 .init_array    0x20001e08        0x4 /usr/lib/gcc/arm-none-eabi/7.3.1/thumb/v6-m/crtbegin.o
 .init_array    0x20001e0c        0x4 CMakeFiles/main.dir/main.cpp.obj
 .init_array    0x20001e10        0x4 CMakeFiles/main.dir/__/pico-sdk/src/rp2_common/pico_unique_id/unique_id.c.obj
 .init_array    0x20001e14        0x4 libLoRa_pico_lib.a(LoRa-RP2040.cpp.obj)
                0x20001e18                PROVIDE (__init_array_end = .)
                0x20001e18                . = ALIGN (0x4)
                0x20001e18                PROVIDE (__fini_array_start = .)
 *(SORT_BY_NAME(.fini_array.*))
 *(.fini_array)
                0x20001e18                PROVIDE (__fini_array_end = .)
 *(.jcr)
                0x20001e18                . = ALIGN (0x4)
                0x20001e18                __data_end__ = .

.tm_clone_table
                0x20001e18        0x0 load address 0x10013dfc
 .tm_clone_table
                0x20001e18        0x0 /usr/lib/gcc/arm-none-eabi/7.3.1/thumb/v6-m/crtbegin.o
 .tm_clone_table
                0x20001e18        0x0 /usr/lib/gcc/arm-none-eabi/7.3.1/thumb/v6-m/crtend.o

.igot.plt       0x20001e18        0x0 load address 0x10013dfc
 .igot.plt      0x20001e18        0x0 /usr/lib/gcc/arm-none-eabi/7.3.1/thumb/v6-m/crtbegin.o

.uninitialized_data
                0x20001e18        0x0 load address 0x10013dfc
                0x20001e18                . = ALIGN (0x4)
 *(.uninitialized_data*)

.scratch_x      0x20040000        0x0 load address 0x10013dfc
                0x20040000                __scratch_x_start__ = .
 *(.scratch_x.*)
                0x20040000                . = ALIGN (0x4)
                0x20040000                __scratch_x_end__ = .
                0x10013dfc                __scratch_x_source__ = LOADADDR (.scratch_x)

.scratch_y      0x20041000        0x0 load address 0x10013dfc
                0x20041000                __scratch_y_start__ = .
 *(.scratch_y.*)
                0x20041000                . = ALIGN (0x4)
                0x20041000                __scratch_y_end__ = .
                0x10013dfc                __scratch_y_source__ = LOADADDR (.scratch_y)

.bss            0x20001e18     0x225c
                0x20001e18                . = ALIGN (0x4)
                0x20001e18                __bss_start__ = .
 *(SORT_BY_ALIGNMENT(SORT_BY_NAME(.bss*)))
 .bss.AprsSettings
                0x20001e18      0x100 CMakeFiles/main.dir/main.cpp.obj
                0x20001e18                AprsSettings
 .bss.default_alarm_pool_entries
                0x20001f18      0x100 CMakeFiles/main.dir/__/pico-sdk/src/common/pico_time/time.c.obj
 .bss.last_avail_time.7108
                0x20002018        0x8 CMakeFiles/main.dir/__/pico-sdk/src/rp2_common/pico_stdio_usb/stdio_usb.c.obj
 .bss           0x20002020       0x1c /usr/lib/gcc/arm-none-eabi/7.3.1/thumb/v6-m/crtbegin.o
 .bss           0x2000203c        0x7 libKISS.a(kiss.cpp.obj)
 *fill*         0x20002043        0x1 
 .bss           0x20002044       0x34 /usr/lib/gcc/arm-none-eabi/7.3.1/../../../arm-none-eabi/lib/thumb/v6-m/libc.a(lib_a-mallocr.o)
                0x20002044                __malloc_top_pad
                0x20002048                __malloc_current_mallinfo
                0x20002070                __malloc_max_sbrked_mem
                0x20002074                __malloc_max_total_mem
 .bss.AX25Frame
                0x20002078      0x604 CMakeFiles/main.dir/main.cpp.obj
                0x20002078                AX25Frame
 .bss.AprsFrame
                0x2000267c      0x472 CMakeFiles/main.dir/main.cpp.obj
                0x2000267c                AprsFrame
 *fill*         0x20002aee        0x2 
 .bss.Kiss      0x20002af0        0x1 CMakeFiles/main.dir/main.cpp.obj
                0x20002af0                Kiss
 *fill*         0x20002af1        0x3 
 .bss.KissTxFrame
                0x20002af4      0x472 CMakeFiles/main.dir/main.cpp.obj
                0x20002af4                KissTxFrame
 *fill*         0x20002f66        0x2 
 .bss.LoRa      0x20002f68       0x2c libLoRa_pico_lib.a(LoRa-RP2040.cpp.obj)
                0x20002f68                LoRa
 .bss.Status    0x20002f94       0x74 CMakeFiles/main.dir/main.cpp.obj
                0x20002f94                Status
 .bss._ZZ13ReadUSBSerialvE2lp
                0x20003008        0x4 CMakeFiles/main.dir/main.cpp.obj
 .bss._ZZ13ReadUSBSerialvE4strg
                0x2000300c      0x200 CMakeFiles/main.dir/main.cpp.obj
 .bss._app_driver
                0x2000320c        0x4 CMakeFiles/main.dir/__/pico-sdk/lib/tinyusb/src/device/usbd.c.obj
 .bss._cdcd_itf
                0x20003210      0x2d8 CMakeFiles/main.dir/__/pico-sdk/lib/tinyusb/src/class/cdc/cdc_device.c.obj
 .bss._ctrl_xfer
                0x200034e8       0x14 CMakeFiles/main.dir/__/pico-sdk/lib/tinyusb/src/device/usbd_control.c.obj
 .bss._ubsd_mutexdef
                0x200034fc        0x8 CMakeFiles/main.dir/__/pico-sdk/lib/tinyusb/src/device/usbd.c.obj
 .bss._usbd_ctrl_buf
                0x20003504       0x40 CMakeFiles/main.dir/__/pico-sdk/lib/tinyusb/src/device/usbd_control.c.obj
 .bss._usbd_dev
                0x20003544       0x53 CMakeFiles/main.dir/__/pico-sdk/lib/tinyusb/src/device/usbd.c.obj
 *fill*         0x20003597        0x1 
 .bss._usbd_mutex
                0x20003598        0x4 CMakeFiles/main.dir/__/pico-sdk/lib/tinyusb/src/device/usbd.c.obj
 .bss._usbd_q   0x2000359c        0x4 CMakeFiles/main.dir/__/pico-sdk/lib/tinyusb/src/device/usbd.c.obj
 .bss.alarm_callbacks
                0x200035a0       0x10 CMakeFiles/main.dir/__/pico-sdk/src/rp2_common/hardware_timer/timer.c.obj
 .bss.boot2_copyout
                0x200035b0      0x100 CMakeFiles/main.dir/__/pico-sdk/src/rp2_common/hardware_flash/flash.c.obj
 .bss.claimed   0x200036b0        0x4 CMakeFiles/main.dir/__/pico-sdk/src/rp2_common/hardware_sync/sync.c.obj
 .bss.configured_freq
                0x200036b4       0x28 CMakeFiles/main.dir/__/pico-sdk/src/rp2_common/hardware_clocks/clocks.c.obj
 .bss.default_alarm_pool_entry_ids_high
                0x200036dc       0x10 CMakeFiles/main.dir/__/pico-sdk/src/common/pico_time/time.c.obj
 .bss.default_alarm_pool_heap_nodes
                0x200036ec       0x30 CMakeFiles/main.dir/__/pico-sdk/src/common/pico_time/time.c.obj
 .bss.desc_str.7007
                0x2000371c       0x28 CMakeFiles/main.dir/__/pico-sdk/src/rp2_common/pico_stdio_usb/stdio_usb_descriptors.c.obj
 .bss.drivers   0x20003744        0x4 CMakeFiles/main.dir/__/pico-sdk/src/rp2_common/pico_stdio/stdio.c.obj
 .bss.filter    0x20003748        0x4 CMakeFiles/main.dir/__/pico-sdk/src/rp2_common/pico_stdio/stdio.c.obj
 .bss.heap_end.5793
                0x2000374c        0x4 CMakeFiles/main.dir/__/pico-sdk/src/rp2_common/pico_runtime/runtime.c.obj
 .bss.hw_endpoints
                0x20003750      0x400 CMakeFiles/main.dir/__/pico-sdk/lib/tinyusb/src/portable/raspberrypi/rp2040/dcd_rp2040.c.obj
 .bss.lazy_vsnprintf
                0x20003b50        0x4 CMakeFiles/main.dir/__/pico-sdk/src/rp2_common/pico_printf/printf.c.obj
 .bss.load_value
                0x20003b54        0x4 CMakeFiles/main.dir/__/pico-sdk/src/rp2_common/hardware_watchdog/watchdog.c.obj
 .bss.next_buffer_ptr
                0x20003b58        0x4 CMakeFiles/main.dir/__/pico-sdk/lib/tinyusb/src/portable/raspberrypi/rp2040/dcd_rp2040.c.obj
 .bss.pools     0x20003b5c       0x10 CMakeFiles/main.dir/__/pico-sdk/src/common/pico_time/time.c.obj
 .bss.retrieved_id
                0x20003b6c        0x8 CMakeFiles/main.dir/__/pico-sdk/src/rp2_common/pico_unique_id/unique_id.c.obj
 .bss.rxBuffer  0x20003b74       0xff CMakeFiles/main.dir/main.cpp.obj
                0x20003b74                rxBuffer
 *fill*         0x20003c73        0x1 
 .bss.sf_clz_func
                0x20003c74        0x4 CMakeFiles/main.dir/__/pico-sdk/src/rp2_common/pico_double/double_init_rom.c.obj
                0x20003c74                sf_clz_func
 .bss.sleep_notifier
                0x20003c78        0x4 CMakeFiles/main.dir/__/pico-sdk/src/common/pico_time/time.c.obj
 .bss.stdio_usb_mutex
                0x20003c7c        0x8 CMakeFiles/main.dir/__/pico-sdk/src/rp2_common/pico_stdio_usb/stdio_usb.c.obj
 .bss.target_hi
                0x20003c84       0x10 CMakeFiles/main.dir/__/pico-sdk/src/rp2_common/hardware_timer/timer.c.obj
 .bss.txBuffer  0x20003c94       0xff CMakeFiles/main.dir/main.cpp.obj
                0x20003c94                txBuffer
 *fill*         0x20003d93        0x1 
 .bss.usbd_serial_str
                0x20003d94       0x11 CMakeFiles/main.dir/__/pico-sdk/src/rp2_common/pico_stdio_usb/stdio_usb_descriptors.c.obj
 .bss.NO_I2C_AVAILABLE
                0x20003da5        0x1 CMakeFiles/main.dir/main.cpp.obj
                0x20003da5                NO_I2C_AVAILABLE
 .bss.TransmitRequest
                0x20003da6        0x1 CMakeFiles/main.dir/main.cpp.obj
                0x20003da6                TransmitRequest
 .bss._app_driver_count
                0x20003da7        0x1 CMakeFiles/main.dir/__/pico-sdk/lib/tinyusb/src/device/usbd.c.obj
 .bss._usbd_initialized
                0x20003da8        0x1 CMakeFiles/main.dir/__/pico-sdk/lib/tinyusb/src/device/usbd.c.obj
 .bss.boot2_copyout_valid
                0x20003da9        0x1 CMakeFiles/main.dir/__/pico-sdk/src/rp2_common/hardware_flash/flash.c.obj
 .bss.claimed   0x20003daa        0x1 CMakeFiles/main.dir/__/pico-sdk/src/rp2_common/hardware_timer/timer.c.obj
 .bss.irq_hander_chain_free_slot_head
                0x20003dab        0x1 CMakeFiles/main.dir/__/pico-sdk/src/rp2_common/hardware_irq/irq.c.obj
 .bss.itf_num   0x20003dac        0x1 CMakeFiles/main.dir/__/pico-sdk/src/rp2_common/pico_stdio_usb/reset_interface.c.obj
 .bss.timer_callbacks_pending
                0x20003dad        0x1 CMakeFiles/main.dir/__/pico-sdk/src/rp2_common/hardware_timer/timer.c.obj
 *(COMMON)
 *fill*         0x20003dae        0x2 
 COMMON         0x20003db0      0x100 CMakeFiles/main.dir/__/pico-sdk/src/rp2_common/pico_double/double_init_rom.c.obj
                0x20003db0                sd_table
 COMMON         0x20003eb0      0x100 CMakeFiles/main.dir/__/pico-sdk/src/rp2_common/pico_float/float_init_rom.c.obj
                0x20003eb0                sf_table
 COMMON         0x20003fb0       0xc0 CMakeFiles/main.dir/__/pico-sdk/lib/tinyusb/src/device/usbd.c.obj
                0x20003fb0                _usbd_qdef_buf
 COMMON         0x20004070        0x4 /usr/lib/gcc/arm-none-eabi/7.3.1/../../../arm-none-eabi/lib/thumb/v6-m/libc.a(lib_a-reent.o)
                0x20004070                errno
                0x20004074                . = ALIGN (0x4)
                0x20004074                __bss_end__ = .

.heap           0x20004074      0x800
                0x20004074                __end__ = .
                0x20004074                end = __end__
 *(.heap*)
 .heap          0x20004074      0x800 CMakeFiles/main.dir/__/pico-sdk/src/rp2_common/pico_standard_link/crt0.S.obj
                0x20004874                __HeapLimit = .

.stack1_dummy   0x20040000        0x0
 *(.stack1*)

.stack_dummy    0x20041000      0x800
 *(.stack*)
 .stack         0x20041000      0x800 CMakeFiles/main.dir/__/pico-sdk/src/rp2_common/pico_standard_link/crt0.S.obj

.flash_end      0x10013dfc        0x0
                0x10013dfc                __flash_binary_end = .
                0x20040000                __StackLimit = (ORIGIN (RAM) + LENGTH (RAM))
                0x20041000                __StackOneTop = (ORIGIN (SCRATCH_X) + LENGTH (SCRATCH_X))
                0x20042000                __StackTop = (ORIGIN (SCRATCH_Y) + LENGTH (SCRATCH_Y))
                0x20041000                __StackOneBottom = (__StackOneTop - SIZEOF (.stack1_dummy))
                0x20041800                __StackBottom = (__StackTop - SIZEOF (.stack_dummy))
                0x20042000                PROVIDE (__stack = __StackTop)
                0x00000001                ASSERT ((__StackLimit >= __HeapLimit), region RAM overflowed)
                0x00000001                ASSERT (((__binary_info_header_end - __logical_binary_start) <= 0x100), Binary info must be in first 256 bytes of the binary)
LOAD CMakeFiles/main.dir/main.cpp.obj
LOAD CMakeFiles/main.dir/__/pico-sdk/src/rp2_common/pico_stdlib/stdlib.c.obj
LOAD CMakeFiles/main.dir/__/pico-sdk/src/rp2_common/hardware_gpio/gpio.c.obj
LOAD CMakeFiles/main.dir/__/pico-sdk/src/rp2_common/hardware_claim/claim.c.obj
LOAD CMakeFiles/main.dir/__/pico-sdk/src/rp2_common/pico_platform/platform.c.obj
LOAD CMakeFiles/main.dir/__/pico-sdk/src/rp2_common/hardware_sync/sync.c.obj
LOAD CMakeFiles/main.dir/__/pico-sdk/src/rp2_common/hardware_uart/uart.c.obj
LOAD CMakeFiles/main.dir/__/pico-sdk/src/rp2_common/hardware_divider/divider.S.obj
LOAD CMakeFiles/main.dir/__/pico-sdk/src/common/pico_time/time.c.obj
LOAD CMakeFiles/main.dir/__/pico-sdk/src/common/pico_time/timeout_helper.c.obj
LOAD CMakeFiles/main.dir/__/pico-sdk/src/rp2_common/hardware_timer/timer.c.obj
LOAD CMakeFiles/main.dir/__/pico-sdk/src/common/pico_sync/sem.c.obj
LOAD CMakeFiles/main.dir/__/pico-sdk/src/common/pico_sync/lock_core.c.obj
LOAD CMakeFiles/main.dir/__/pico-sdk/src/common/pico_sync/mutex.c.obj
LOAD CMakeFiles/main.dir/__/pico-sdk/src/common/pico_sync/critical_section.c.obj
LOAD CMakeFiles/main.dir/__/pico-sdk/src/common/pico_util/datetime.c.obj
LOAD CMakeFiles/main.dir/__/pico-sdk/src/common/pico_util/pheap.c.obj
LOAD CMakeFiles/main.dir/__/pico-sdk/src/common/pico_util/queue.c.obj
LOAD CMakeFiles/main.dir/__/pico-sdk/src/rp2_common/pico_runtime/runtime.c.obj
LOAD CMakeFiles/main.dir/__/pico-sdk/src/rp2_common/hardware_clocks/clocks.c.obj
LOAD CMakeFiles/main.dir/__/pico-sdk/src/rp2_common/hardware_irq/irq.c.obj
LOAD CMakeFiles/main.dir/__/pico-sdk/src/rp2_common/hardware_irq/irq_handler_chain.S.obj
LOAD CMakeFiles/main.dir/__/pico-sdk/src/rp2_common/hardware_pll/pll.c.obj
LOAD CMakeFiles/main.dir/__/pico-sdk/src/rp2_common/hardware_vreg/vreg.c.obj
LOAD CMakeFiles/main.dir/__/pico-sdk/src/rp2_common/hardware_watchdog/watchdog.c.obj
LOAD CMakeFiles/main.dir/__/pico-sdk/src/rp2_common/hardware_xosc/xosc.c.obj
LOAD CMakeFiles/main.dir/__/pico-sdk/src/rp2_common/pico_printf/printf.c.obj
LOAD CMakeFiles/main.dir/__/pico-sdk/src/rp2_common/pico_bit_ops/bit_ops_aeabi.S.obj
LOAD CMakeFiles/main.dir/__/pico-sdk/src/rp2_common/pico_bootrom/bootrom.c.obj
LOAD CMakeFiles/main.dir/__/pico-sdk/src/rp2_common/pico_divider/divider.S.obj
LOAD CMakeFiles/main.dir/__/pico-sdk/src/rp2_common/pico_double/double_aeabi.S.obj
LOAD CMakeFiles/main.dir/__/pico-sdk/src/rp2_common/pico_double/double_init_rom.c.obj
LOAD CMakeFiles/main.dir/__/pico-sdk/src/rp2_common/pico_double/double_math.c.obj
LOAD CMakeFiles/main.dir/__/pico-sdk/src/rp2_common/pico_double/double_v1_rom_shim.S.obj
LOAD CMakeFiles/main.dir/__/pico-sdk/src/rp2_common/pico_int64_ops/pico_int64_ops_aeabi.S.obj
LOAD CMakeFiles/main.dir/__/pico-sdk/src/rp2_common/pico_float/float_aeabi.S.obj
LOAD CMakeFiles/main.dir/__/pico-sdk/src/rp2_common/pico_float/float_init_rom.c.obj
LOAD CMakeFiles/main.dir/__/pico-sdk/src/rp2_common/pico_float/float_math.c.obj
LOAD CMakeFiles/main.dir/__/pico-sdk/src/rp2_common/pico_float/float_v1_rom_shim.S.obj
LOAD CMakeFiles/main.dir/__/pico-sdk/src/rp2_common/pico_malloc/pico_malloc.c.obj
LOAD CMakeFiles/main.dir/__/pico-sdk/src/rp2_common/pico_mem_ops/mem_ops_aeabi.S.obj
LOAD CMakeFiles/main.dir/__/pico-sdk/src/rp2_common/pico_standard_link/crt0.S.obj
LOAD CMakeFiles/main.dir/__/pico-sdk/src/rp2_common/pico_standard_link/new_delete.cpp.obj
LOAD CMakeFiles/main.dir/__/pico-sdk/src/rp2_common/pico_standard_link/binary_info.c.obj
LOAD CMakeFiles/main.dir/__/pico-sdk/src/rp2_common/pico_stdio/stdio.c.obj
LOAD CMakeFiles/main.dir/__/pico-sdk/src/rp2_common/pico_stdio_usb/reset_interface.c.obj
LOAD CMakeFiles/main.dir/__/pico-sdk/src/rp2_common/pico_stdio_usb/stdio_usb.c.obj
LOAD CMakeFiles/main.dir/__/pico-sdk/src/rp2_common/pico_stdio_usb/stdio_usb_descriptors.c.obj
LOAD CMakeFiles/main.dir/__/pico-sdk/lib/tinyusb/src/portable/raspberrypi/rp2040/dcd_rp2040.c.obj
LOAD CMakeFiles/main.dir/__/pico-sdk/lib/tinyusb/src/portable/raspberrypi/rp2040/rp2040_usb.c.obj
LOAD CMakeFiles/main.dir/__/pico-sdk/lib/tinyusb/src/device/usbd.c.obj
LOAD CMakeFiles/main.dir/__/pico-sdk/lib/tinyusb/src/device/usbd_control.c.obj
LOAD CMakeFiles/main.dir/__/pico-sdk/lib/tinyusb/src/class/audio/audio_device.c.obj
LOAD CMakeFiles/main.dir/__/pico-sdk/lib/tinyusb/src/class/cdc/cdc_device.c.obj
LOAD CMakeFiles/main.dir/__/pico-sdk/lib/tinyusb/src/class/dfu/dfu_device.c.obj
LOAD CMakeFiles/main.dir/__/pico-sdk/lib/tinyusb/src/class/dfu/dfu_rt_device.c.obj
LOAD CMakeFiles/main.dir/__/pico-sdk/lib/tinyusb/src/class/hid/hid_device.c.obj
LOAD CMakeFiles/main.dir/__/pico-sdk/lib/tinyusb/src/class/midi/midi_device.c.obj
LOAD CMakeFiles/main.dir/__/pico-sdk/lib/tinyusb/src/class/msc/msc_device.c.obj
LOAD CMakeFiles/main.dir/__/pico-sdk/lib/tinyusb/src/class/net/ecm_rndis_device.c.obj
LOAD CMakeFiles/main.dir/__/pico-sdk/lib/tinyusb/src/class/net/ncm_device.c.obj
LOAD CMakeFiles/main.dir/__/pico-sdk/lib/tinyusb/src/class/usbtmc/usbtmc_device.c.obj
LOAD CMakeFiles/main.dir/__/pico-sdk/lib/tinyusb/src/class/vendor/vendor_device.c.obj
LOAD CMakeFiles/main.dir/__/pico-sdk/lib/tinyusb/src/class/video/video_device.c.obj
LOAD CMakeFiles/main.dir/__/pico-sdk/lib/tinyusb/src/tusb.c.obj
LOAD CMakeFiles/main.dir/__/pico-sdk/lib/tinyusb/src/common/tusb_fifo.c.obj
LOAD CMakeFiles/main.dir/__/pico-sdk/src/rp2_common/pico_fix/rp2040_usb_device_enumeration/rp2040_usb_device_enumeration.c.obj
LOAD CMakeFiles/main.dir/__/pico-sdk/src/rp2_common/pico_unique_id/unique_id.c.obj
LOAD CMakeFiles/main.dir/__/pico-sdk/src/rp2_common/hardware_flash/flash.c.obj
LOAD CMakeFiles/main.dir/__/pico-sdk/src/rp2_common/hardware_spi/spi.c.obj
LOAD CMakeFiles/main.dir/__/pico-sdk/src/rp2_common/hardware_interp/interp.c.obj
LOAD CMakeFiles/main.dir/__/pico-sdk/src/rp2_common/hardware_i2c/i2c.c.obj
LOAD libLoRa_pico_lib.a
LOAD libLoRa_print.a
LOAD libKISS.a
LOAD libi2c_sensor.a
LOAD /tmp/ccWYemgR.o
LOAD /usr/lib/gcc/arm-none-eabi/7.3.1/../../../arm-none-eabi/lib/thumb/v6-m/libstdc++.a
LOAD /usr/lib/gcc/arm-none-eabi/7.3.1/../../../arm-none-eabi/lib/thumb/v6-m/libm.a
START GROUP
LOAD /usr/lib/gcc/arm-none-eabi/7.3.1/thumb/v6-m/libgcc.a
LOAD /usr/lib/gcc/arm-none-eabi/7.3.1/../../../arm-none-eabi/lib/thumb/v6-m/libc.a
END GROUP
START GROUP
LOAD /usr/lib/gcc/arm-none-eabi/7.3.1/thumb/v6-m/libgcc.a
LOAD /usr/lib/gcc/arm-none-eabi/7.3.1/../../../arm-none-eabi/lib/thumb/v6-m/libc.a
LOAD /usr/lib/gcc/arm-none-eabi/7.3.1/../../../arm-none-eabi/lib/thumb/v6-m/libnosys.a
END GROUP
LOAD /usr/lib/gcc/arm-none-eabi/7.3.1/thumb/v6-m/crtend.o
LOAD /usr/lib/gcc/arm-none-eabi/7.3.1/thumb/v6-m/crtn.o
OUTPUT(main.elf elf32-littlearm)

.ARM.attributes
                0x00000000       0x28
 .ARM.attributes
                0x00000000       0x1e /usr/lib/gcc/arm-none-eabi/7.3.1/thumb/v6-m/crti.o
 .ARM.attributes
                0x0000001e       0x2c /usr/lib/gcc/arm-none-eabi/7.3.1/thumb/v6-m/crtbegin.o
 .ARM.attributes
                0x0000004a       0x32 CMakeFiles/main.dir/main.cpp.obj
 .ARM.attributes
                0x0000007c       0x32 CMakeFiles/main.dir/__/pico-sdk/src/rp2_common/hardware_gpio/gpio.c.obj
 .ARM.attributes
                0x000000ae       0x32 CMakeFiles/main.dir/__/pico-sdk/src/rp2_common/hardware_claim/claim.c.obj
 .ARM.attributes
                0x000000e0       0x32 CMakeFiles/main.dir/__/pico-sdk/src/rp2_common/pico_platform/platform.c.obj
 .ARM.attributes
                0x00000112       0x32 CMakeFiles/main.dir/__/pico-sdk/src/rp2_common/hardware_sync/sync.c.obj
 .ARM.attributes
                0x00000144       0x32 CMakeFiles/main.dir/__/pico-sdk/src/common/pico_time/time.c.obj
 .ARM.attributes
                0x00000176       0x32 CMakeFiles/main.dir/__/pico-sdk/src/common/pico_time/timeout_helper.c.obj
 .ARM.attributes
                0x000001a8       0x32 CMakeFiles/main.dir/__/pico-sdk/src/rp2_common/hardware_timer/timer.c.obj
 .ARM.attributes
                0x000001da       0x32 CMakeFiles/main.dir/__/pico-sdk/src/common/pico_sync/lock_core.c.obj
 .ARM.attributes
                0x0000020c       0x32 CMakeFiles/main.dir/__/pico-sdk/src/common/pico_sync/mutex.c.obj
 .ARM.attributes
                0x0000023e       0x32 CMakeFiles/main.dir/__/pico-sdk/src/common/pico_sync/critical_section.c.obj
 .ARM.attributes
                0x00000270       0x32 CMakeFiles/main.dir/__/pico-sdk/src/common/pico_util/pheap.c.obj
 .ARM.attributes
                0x000002a2       0x32 CMakeFiles/main.dir/__/pico-sdk/src/rp2_common/pico_runtime/runtime.c.obj
 .ARM.attributes
                0x000002d4       0x32 CMakeFiles/main.dir/__/pico-sdk/src/rp2_common/hardware_clocks/clocks.c.obj
 .ARM.attributes
                0x00000306       0x32 CMakeFiles/main.dir/__/pico-sdk/src/rp2_common/hardware_irq/irq.c.obj
 .ARM.attributes
                0x00000338       0x22 CMakeFiles/main.dir/__/pico-sdk/src/rp2_common/hardware_irq/irq_handler_chain.S.obj
 .ARM.attributes
                0x0000035a       0x32 CMakeFiles/main.dir/__/pico-sdk/src/rp2_common/hardware_pll/pll.c.obj
 .ARM.attributes
                0x0000038c       0x32 CMakeFiles/main.dir/__/pico-sdk/src/rp2_common/hardware_watchdog/watchdog.c.obj
 .ARM.attributes
                0x000003be       0x32 CMakeFiles/main.dir/__/pico-sdk/src/rp2_common/hardware_xosc/xosc.c.obj
 .ARM.attributes
                0x000003f0       0x32 CMakeFiles/main.dir/__/pico-sdk/src/rp2_common/pico_printf/printf.c.obj
 .ARM.attributes
                0x00000422       0x22 CMakeFiles/main.dir/__/pico-sdk/src/rp2_common/pico_bit_ops/bit_ops_aeabi.S.obj
 .ARM.attributes
                0x00000444       0x32 CMakeFiles/main.dir/__/pico-sdk/src/rp2_common/pico_bootrom/bootrom.c.obj
 .ARM.attributes
                0x00000476       0x22 CMakeFiles/main.dir/__/pico-sdk/src/rp2_common/pico_divider/divider.S.obj
 .ARM.attributes
                0x00000498       0x22 CMakeFiles/main.dir/__/pico-sdk/src/rp2_common/pico_double/double_aeabi.S.obj
 .ARM.attributes
                0x000004ba       0x32 CMakeFiles/main.dir/__/pico-sdk/src/rp2_common/pico_double/double_init_rom.c.obj
 .ARM.attributes
                0x000004ec       0x22 CMakeFiles/main.dir/__/pico-sdk/src/rp2_common/pico_double/double_v1_rom_shim.S.obj
 .ARM.attributes
                0x0000050e       0x22 CMakeFiles/main.dir/__/pico-sdk/src/rp2_common/pico_int64_ops/pico_int64_ops_aeabi.S.obj
 .ARM.attributes
                0x00000530       0x22 CMakeFiles/main.dir/__/pico-sdk/src/rp2_common/pico_float/float_aeabi.S.obj
 .ARM.attributes
                0x00000552       0x32 CMakeFiles/main.dir/__/pico-sdk/src/rp2_common/pico_float/float_init_rom.c.obj
 .ARM.attributes
                0x00000584       0x22 CMakeFiles/main.dir/__/pico-sdk/src/rp2_common/pico_float/float_v1_rom_shim.S.obj
 .ARM.attributes
                0x000005a6       0x22 CMakeFiles/main.dir/__/pico-sdk/src/rp2_common/pico_mem_ops/mem_ops_aeabi.S.obj
 .ARM.attributes
                0x000005c8       0x22 CMakeFiles/main.dir/__/pico-sdk/src/rp2_common/pico_standard_link/crt0.S.obj
 .ARM.attributes
                0x000005ea       0x32 CMakeFiles/main.dir/__/pico-sdk/src/rp2_common/pico_standard_link/binary_info.c.obj
 .ARM.attributes
                0x0000061c       0x32 CMakeFiles/main.dir/__/pico-sdk/src/rp2_common/pico_stdio/stdio.c.obj
 .ARM.attributes
                0x0000064e       0x32 CMakeFiles/main.dir/__/pico-sdk/src/rp2_common/pico_stdio_usb/reset_interface.c.obj
 .ARM.attributes
                0x00000680       0x32 CMakeFiles/main.dir/__/pico-sdk/src/rp2_common/pico_stdio_usb/stdio_usb.c.obj
 .ARM.attributes
                0x000006b2       0x32 CMakeFiles/main.dir/__/pico-sdk/src/rp2_common/pico_stdio_usb/stdio_usb_descriptors.c.obj
 .ARM.attributes
                0x000006e4       0x32 CMakeFiles/main.dir/__/pico-sdk/lib/tinyusb/src/portable/raspberrypi/rp2040/dcd_rp2040.c.obj
 .ARM.attributes
                0x00000716       0x32 CMakeFiles/main.dir/__/pico-sdk/lib/tinyusb/src/portable/raspberrypi/rp2040/rp2040_usb.c.obj
 .ARM.attributes
                0x00000748       0x32 CMakeFiles/main.dir/__/pico-sdk/lib/tinyusb/src/device/usbd.c.obj
 .ARM.attributes
                0x0000077a       0x32 CMakeFiles/main.dir/__/pico-sdk/lib/tinyusb/src/device/usbd_control.c.obj
 .ARM.attributes
                0x000007ac       0x32 CMakeFiles/main.dir/__/pico-sdk/lib/tinyusb/src/class/cdc/cdc_device.c.obj
 .ARM.attributes
                0x000007de       0x32 CMakeFiles/main.dir/__/pico-sdk/lib/tinyusb/src/tusb.c.obj
 .ARM.attributes
                0x00000810       0x32 CMakeFiles/main.dir/__/pico-sdk/lib/tinyusb/src/common/tusb_fifo.c.obj
 .ARM.attributes
                0x00000842       0x32 CMakeFiles/main.dir/__/pico-sdk/src/rp2_common/pico_unique_id/unique_id.c.obj
 .ARM.attributes
                0x00000874       0x32 CMakeFiles/main.dir/__/pico-sdk/src/rp2_common/hardware_flash/flash.c.obj
 .ARM.attributes
                0x000008a6       0x32 CMakeFiles/main.dir/__/pico-sdk/src/rp2_common/hardware_spi/spi.c.obj
 .ARM.attributes
                0x000008d8       0x32 CMakeFiles/main.dir/__/pico-sdk/src/rp2_common/hardware_i2c/i2c.c.obj
 .ARM.attributes
                0x0000090a       0x32 libLoRa_pico_lib.a(LoRa-RP2040.cpp.obj)
 .ARM.attributes
                0x0000093c       0x32 libKISS.a(kiss.cpp.obj)
 .ARM.attributes
                0x0000096e       0x32 libi2c_sensor.a(i2c_sensor.cpp.obj)
 .ARM.attributes
                0x000009a0       0x22 /tmp/ccWYemgR.o
 .ARM.attributes
                0x000009c2       0x1e /usr/lib/gcc/arm-none-eabi/7.3.1/thumb/v6-m/libgcc.a(_dvmd_tls.o)
 .ARM.attributes
                0x000009e0       0x2c /usr/lib/gcc/arm-none-eabi/7.3.1/../../../arm-none-eabi/lib/thumb/v6-m/libc.a(lib_a-memmove.o)
 .ARM.attributes
                0x00000a0c       0x1b /usr/lib/gcc/arm-none-eabi/7.3.1/../../../arm-none-eabi/lib/thumb/v6-m/libc.a(lib_a-strcmp.o)
 .ARM.attributes
                0x00000a27       0x2c /usr/lib/gcc/arm-none-eabi/7.3.1/../../../arm-none-eabi/lib/thumb/v6-m/libc.a(lib_a-strlen-stub.o)
 .ARM.attributes
                0x00000a53       0x2c /usr/lib/gcc/arm-none-eabi/7.3.1/thumb/v6-m/crtend.o

.comment        0x00000000       0xae
 .comment       0x00000000       0x57 /usr/lib/gcc/arm-none-eabi/7.3.1/thumb/v6-m/crtbegin.o
                                 0x58 (size before relaxing)
 .comment       0x00000057       0x58 CMakeFiles/main.dir/main.cpp.obj
 .comment       0x00000057       0x58 CMakeFiles/main.dir/__/pico-sdk/src/rp2_common/hardware_gpio/gpio.c.obj
 .comment       0x00000057       0x58 CMakeFiles/main.dir/__/pico-sdk/src/rp2_common/hardware_claim/claim.c.obj
 .comment       0x00000057       0x58 CMakeFiles/main.dir/__/pico-sdk/src/rp2_common/pico_platform/platform.c.obj
 .comment       0x00000057       0x58 CMakeFiles/main.dir/__/pico-sdk/src/rp2_common/hardware_sync/sync.c.obj
 .comment       0x00000057       0x58 CMakeFiles/main.dir/__/pico-sdk/src/common/pico_time/time.c.obj
 .comment       0x00000057       0x58 CMakeFiles/main.dir/__/pico-sdk/src/common/pico_time/timeout_helper.c.obj
 .comment       0x00000057       0x58 CMakeFiles/main.dir/__/pico-sdk/src/rp2_common/hardware_timer/timer.c.obj
 .comment       0x00000057       0x58 CMakeFiles/main.dir/__/pico-sdk/src/common/pico_sync/lock_core.c.obj
 .comment       0x00000057       0x58 CMakeFiles/main.dir/__/pico-sdk/src/common/pico_sync/mutex.c.obj
 .comment       0x00000057       0x58 CMakeFiles/main.dir/__/pico-sdk/src/common/pico_sync/critical_section.c.obj
 .comment       0x00000057       0x58 CMakeFiles/main.dir/__/pico-sdk/src/common/pico_util/pheap.c.obj
 .comment       0x00000057       0x58 CMakeFiles/main.dir/__/pico-sdk/src/rp2_common/pico_runtime/runtime.c.obj
 .comment       0x00000057       0x58 CMakeFiles/main.dir/__/pico-sdk/src/rp2_common/hardware_clocks/clocks.c.obj
 .comment       0x00000057       0x58 CMakeFiles/main.dir/__/pico-sdk/src/rp2_common/hardware_irq/irq.c.obj
 .comment       0x00000057       0x58 CMakeFiles/main.dir/__/pico-sdk/src/rp2_common/hardware_pll/pll.c.obj
 .comment       0x00000057       0x58 CMakeFiles/main.dir/__/pico-sdk/src/rp2_common/hardware_watchdog/watchdog.c.obj
 .comment       0x00000057       0x58 CMakeFiles/main.dir/__/pico-sdk/src/rp2_common/hardware_xosc/xosc.c.obj
 .comment       0x00000057       0x58 CMakeFiles/main.dir/__/pico-sdk/src/rp2_common/pico_printf/printf.c.obj
 .comment       0x00000057       0x58 CMakeFiles/main.dir/__/pico-sdk/src/rp2_common/pico_bootrom/bootrom.c.obj
 .comment       0x00000057       0x58 CMakeFiles/main.dir/__/pico-sdk/src/rp2_common/pico_double/double_init_rom.c.obj
 .comment       0x00000057       0x58 CMakeFiles/main.dir/__/pico-sdk/src/rp2_common/pico_float/float_init_rom.c.obj
 .comment       0x00000057       0x58 CMakeFiles/main.dir/__/pico-sdk/src/rp2_common/pico_standard_link/binary_info.c.obj
 .comment       0x00000057       0x58 CMakeFiles/main.dir/__/pico-sdk/src/rp2_common/pico_stdio/stdio.c.obj
 .comment       0x00000057       0x58 CMakeFiles/main.dir/__/pico-sdk/src/rp2_common/pico_stdio_usb/reset_interface.c.obj
 .comment       0x00000057       0x58 CMakeFiles/main.dir/__/pico-sdk/src/rp2_common/pico_stdio_usb/stdio_usb.c.obj
 .comment       0x00000057       0x58 CMakeFiles/main.dir/__/pico-sdk/src/rp2_common/pico_stdio_usb/stdio_usb_descriptors.c.obj
 .comment       0x00000057       0x58 CMakeFiles/main.dir/__/pico-sdk/lib/tinyusb/src/portable/raspberrypi/rp2040/dcd_rp2040.c.obj
 .comment       0x00000057       0x58 CMakeFiles/main.dir/__/pico-sdk/lib/tinyusb/src/portable/raspberrypi/rp2040/rp2040_usb.c.obj
 .comment       0x00000057       0x58 CMakeFiles/main.dir/__/pico-sdk/lib/tinyusb/src/device/usbd.c.obj
 .comment       0x00000057       0x58 CMakeFiles/main.dir/__/pico-sdk/lib/tinyusb/src/device/usbd_control.c.obj
 .comment       0x00000057       0x58 CMakeFiles/main.dir/__/pico-sdk/lib/tinyusb/src/class/cdc/cdc_device.c.obj
 .comment       0x00000057       0x58 CMakeFiles/main.dir/__/pico-sdk/lib/tinyusb/src/tusb.c.obj
 .comment       0x00000057       0x58 CMakeFiles/main.dir/__/pico-sdk/lib/tinyusb/src/common/tusb_fifo.c.obj
 .comment       0x00000057       0x58 CMakeFiles/main.dir/__/pico-sdk/src/rp2_common/pico_unique_id/unique_id.c.obj
 .comment       0x00000057       0x58 CMakeFiles/main.dir/__/pico-sdk/src/rp2_common/hardware_flash/flash.c.obj
 .comment       0x00000057       0x58 CMakeFiles/main.dir/__/pico-sdk/src/rp2_common/hardware_spi/spi.c.obj
 .comment       0x00000057       0x58 CMakeFiles/main.dir/__/pico-sdk/src/rp2_common/hardware_i2c/i2c.c.obj
 .comment       0x00000057       0x58 libLoRa_pico_lib.a(LoRa-RP2040.cpp.obj)
 .comment       0x00000057       0x58 libKISS.a(kiss.cpp.obj)
 .comment       0x00000057       0x58 libi2c_sensor.a(i2c_sensor.cpp.obj)
 .comment       0x00000057       0x57 /usr/lib/gcc/arm-none-eabi/7.3.1/../../../arm-none-eabi/lib/thumb/v6-m/libc.a(lib_a-memmove.o)
                                 0x58 (size before relaxing)
 .comment       0x000000ae       0x58 /usr/lib/gcc/arm-none-eabi/7.3.1/../../../arm-none-eabi/lib/thumb/v6-m/libc.a(lib_a-strlen-stub.o)
 .comment       0x000000ae       0x58 /usr/lib/gcc/arm-none-eabi/7.3.1/thumb/v6-m/crtend.o

.debug_line     0x00000000      0x401
 .debug_line    0x00000000       0x5d /usr/lib/gcc/arm-none-eabi/7.3.1/thumb/v6-m/libgcc.a(_dvmd_tls.o)
 .debug_line    0x0000005d      0x1b1 /usr/lib/gcc/arm-none-eabi/7.3.1/../../../arm-none-eabi/lib/thumb/v6-m/libc.a(lib_a-memmove.o)
 .debug_line    0x0000020e       0xad /usr/lib/gcc/arm-none-eabi/7.3.1/../../../arm-none-eabi/lib/thumb/v6-m/libc.a(lib_a-strcmp.o)
 .debug_line    0x000002bb      0x146 /usr/lib/gcc/arm-none-eabi/7.3.1/../../../arm-none-eabi/lib/thumb/v6-m/libc.a(lib_a-strlen-stub.o)

.debug_info     0x00000000     0x175f
 .debug_info    0x00000000       0x26 /usr/lib/gcc/arm-none-eabi/7.3.1/thumb/v6-m/libgcc.a(_dvmd_tls.o)
 .debug_info    0x00000026      0xe31 /usr/lib/gcc/arm-none-eabi/7.3.1/../../../arm-none-eabi/lib/thumb/v6-m/libc.a(lib_a-memmove.o)
 .debug_info    0x00000e57       0x26 /usr/lib/gcc/arm-none-eabi/7.3.1/../../../arm-none-eabi/lib/thumb/v6-m/libc.a(lib_a-strcmp.o)
 .debug_info    0x00000e7d      0x8e2 /usr/lib/gcc/arm-none-eabi/7.3.1/../../../arm-none-eabi/lib/thumb/v6-m/libc.a(lib_a-strlen-stub.o)

.debug_abbrev   0x00000000      0x3c3
 .debug_abbrev  0x00000000       0x14 /usr/lib/gcc/arm-none-eabi/7.3.1/thumb/v6-m/libgcc.a(_dvmd_tls.o)
 .debug_abbrev  0x00000014      0x1e3 /usr/lib/gcc/arm-none-eabi/7.3.1/../../../arm-none-eabi/lib/thumb/v6-m/libc.a(lib_a-memmove.o)
 .debug_abbrev  0x000001f7       0x14 /usr/lib/gcc/arm-none-eabi/7.3.1/../../../arm-none-eabi/lib/thumb/v6-m/libc.a(lib_a-strcmp.o)
 .debug_abbrev  0x0000020b      0x1b8 /usr/lib/gcc/arm-none-eabi/7.3.1/../../../arm-none-eabi/lib/thumb/v6-m/libc.a(lib_a-strlen-stub.o)

.debug_aranges  0x00000000       0x80
 .debug_aranges
                0x00000000       0x20 /usr/lib/gcc/arm-none-eabi/7.3.1/thumb/v6-m/libgcc.a(_dvmd_tls.o)
 .debug_aranges
                0x00000020       0x20 /usr/lib/gcc/arm-none-eabi/7.3.1/../../../arm-none-eabi/lib/thumb/v6-m/libc.a(lib_a-memmove.o)
 .debug_aranges
                0x00000040       0x20 /usr/lib/gcc/arm-none-eabi/7.3.1/../../../arm-none-eabi/lib/thumb/v6-m/libc.a(lib_a-strcmp.o)
 .debug_aranges
                0x00000060       0x20 /usr/lib/gcc/arm-none-eabi/7.3.1/../../../arm-none-eabi/lib/thumb/v6-m/libc.a(lib_a-strlen-stub.o)

.debug_str      0x00000000      0x952
 .debug_str     0x00000000       0x9d /usr/lib/gcc/arm-none-eabi/7.3.1/thumb/v6-m/libgcc.a(_dvmd_tls.o)
 .debug_str     0x0000009d      0x7d0 /usr/lib/gcc/arm-none-eabi/7.3.1/../../../arm-none-eabi/lib/thumb/v6-m/libc.a(lib_a-memmove.o)
                                0x8d0 (size before relaxing)
 .debug_str     0x0000086d       0x8d /usr/lib/gcc/arm-none-eabi/7.3.1/../../../arm-none-eabi/lib/thumb/v6-m/libc.a(lib_a-strcmp.o)
                                 0x9b (size before relaxing)
 .debug_str     0x000008fa       0x58 /usr/lib/gcc/arm-none-eabi/7.3.1/../../../arm-none-eabi/lib/thumb/v6-m/libc.a(lib_a-strlen-stub.o)
                                0x5ad (size before relaxing)

.debug_loc      0x00000000      0x42b
 .debug_loc     0x00000000      0x397 /usr/lib/gcc/arm-none-eabi/7.3.1/../../../arm-none-eabi/lib/thumb/v6-m/libc.a(lib_a-memmove.o)
 .debug_loc     0x00000397       0x94 /usr/lib/gcc/arm-none-eabi/7.3.1/../../../arm-none-eabi/lib/thumb/v6-m/libc.a(lib_a-strlen-stub.o)

.debug_frame    0x00000000       0x78
 .debug_frame   0x00000000       0x30 /usr/lib/gcc/arm-none-eabi/7.3.1/../../../arm-none-eabi/lib/thumb/v6-m/libc.a(lib_a-memmove.o)
 .debug_frame   0x00000030       0x20 /usr/lib/gcc/arm-none-eabi/7.3.1/../../../arm-none-eabi/lib/thumb/v6-m/libc.a(lib_a-strcmp.o)
 .debug_frame   0x00000050       0x28 /usr/lib/gcc/arm-none-eabi/7.3.1/../../../arm-none-eabi/lib/thumb/v6-m/libc.a(lib_a-strlen-stub.o)

.stabstr        0x00000000       0x76
 .stabstr       0x00000000       0x76 /usr/lib/gcc/arm-none-eabi/7.3.1/../../../arm-none-eabi/lib/thumb/v6-m/libnosys.a(getpid.o)
